:08000000F07F0020F56F010004
:100400000000000000000000FFFFFFFFBE03FFFF31
:1004100007B5002069460246022315F049FC6846EC
:10042000064906220AF0A7F820B1054869460622C7
:1004300009F00DFF03B05DF804FB00BF38AB01000D
:10044000F382FF1F012808B50FD10422074809F0E5
:10045000FEFE074B05481B68064A93F82210BDE8CC
:10046000084001F0010111F081B808BDE082FF1FD2
:10047000EC82FF1FF90900000149182209F0E7BECC
:100480008B72010038B51C4C1C4D216848F21C00D1
:100490001831B4220BF0B2FD002817DA21681C20B5
:1004A0001831B4220BF0AAFD002812DA2068144992
:1004B0001830B42209F0CBFEB5F90030002B16DB62
:1004C0002846FFF7D9FFFFF7A3FF10E04FF40044E1
:1004D00000E00024B5F90030002B0BDB074918229F
:1004E00044F004000BF08AFDFFF792FF02E04FF4A6
:1004F000804038BD204638BDEC82FF1FF182FF1FCF
:10050000C872010038B5054C0546206821300AF054
:1005100061F828702068213038BD00BFE482FF1FD9
:1005200008B5144B202818800BD002D8E0B1082859
:1005300005E0802818D0B0F5807F0AD0402818D177
:1005400012E0612043F698210622BDE808400AF037
:1005500059BA0622612040F6B8310AF053FA064B28
:100560001A78064B1A7008BD6120BDE808400AF0F1
:10057000ADBA08BD9083FF1FE882FF1F3782FF1FBF
:100580000A46002109F05BBE10B548F204000C4990
:100590000B4C18220BF032FD002809DA042021460A
:1005A00018220BF02BFD002802DA2046FFF764FF2B
:1005B000FFF72EFF238843F00403238010BD00BF04
:1005C000F182FF1F70B5012886B02C4D2C4E20D132
:1005D0002C491822684609F03AFEFFF753FF20F431
:1005E000804084B227492868182209F030FE336819
:1005F0005B899B0715D504A90422234809F027FE2F
:1006000003A90422214809F022FE214802A904225C
:1006100005E0FFF737FF1B4904462868182209F058
:1006200016FE1C482968182209F011FE2868037E6E
:100630001D2B05D018301849B42209F008FE0024FB
:10064000296830681831B42209F001FEB4F5004F72
:100650000BD11C20694601220BF0D0FC00280ADADD
:1006600002200BF0E3FC002006E0B4F5804F02D13D
:10067000002001F00BFA204606B070BDEC82FF1F8F
:10068000E482FF1FF182FF1F0183FF1FFD82FF1F16
:10069000F982FF1FC882FF1FC8720100024B186851
:1006A000021F5042504170470C83FF1F08B5054B95
:1006B000012261201A600AF009FAFA20BDE8084018
:1006C0000CF0D4BC0C83FF1F074B084A197811703B
:1006D00018B1022804D104F059BC054A127800E090
:1006E000FF221A70704700BF3782FF1F1982FF1F59
:1006F000E882FF1F024B1A78024B1A70704700BF46
:100700001982FF1F3782FF1F30B51F4B1F4D1B681B
:1007100085B093F824208DF80B208022ADF80420BA
:100720004FF4C062ADF8062061228DF80C2093F8DA
:100730004E208DF80E2093F84F20DB698DF80F20A6
:10074000002401460093204601236A468DF80840A4
:100750008DF80D3009F042FC287088B10521224641
:1007600009F05CFB009B59060AD540F20441224681
:10077000287809F053FB28788121224609F04EFBA6
:10078000287805B030BD00BFEC82FF1FE882FF1F54
:100790002DE9F043754C867B2568A1B0002D57D11B
:1007A00028460CF08DFCCC2009F042FF704F3860D9
:1007B000B42009F03DFF6F4B18602846FFF702FF99
:1007C000B0F5004F3D4608D1612041F2707103221F
:1007D0000AF018F90423236004E00123FA202360BF
:1007E0000CF044FC01F0DAFC6D2004210AF0D8F88A
:1007F0000320FFF789FF002800F0B5805E4B5F48BB
:100800001A785F4B1A7009F087FE2B685B8C98078B
:1008100003D56FF01E000EF097F803F053FB3C2059
:1008200001F09EFA03F04CFE2868393013F056FEB2
:1008300004F000FF002001464FF0FF3211F070FD80
:10084000752004210AF0ACF84D2004210AF0A8F824
:10085000494D464F30466946052209F0F9FA00280D
:1008600046D09DF803109DF8042011B101291AD03B
:1008700039E0062A0DD005D8032AEBD110460BF03B
:10088000D5FB03E0822A0AD0832AE3D116F074FB59
:10089000E0E728783B49162209F018FEDAE737200E
:1008A00010F00EF9D6E7D92A1AD006D8B72AD1D136
:1008B000084616F0F7FA34480FE0DC2A06D0DD2AA5
:1008C000C8D12368082BC5D13960C3E72F4809F088
:1008D00023FE2F4800F09AFE2E4809F01DFEB9E7CE
:1008E0000EF07AF8B6E73046694609F0B1FAB1E79A
:1008F000236813F0370F36D01F4D287809F0BCFA63
:1009000088B3DFF89880DFF898902F4628786946FA
:10091000402209F09DFA044628B3B8F8006006F4B6
:100920008046B6B26846214616B104F025FBEDE7D5
:1009300000F0B0FEB9F80020684621467AB902F00E
:1009400057FD0028E2D04FF4807001F0A5F902288D
:10095000DCD138781049172209F0B8FDD6E73246C5
:1009600002F046FDD2E721B0BDE8F0830C83FF1F03
:10097000EC82FF1FE482FF1FE882FF1F7C730100EF
:100980003782FF1FBD73010099730100AB73010033
:10099000F982FF1F3BAA0100A37201004684FF1FDA
:1009A0009083FF1F10B50E49044604220D4809F03C
:1009B000E2FD0D4B28B918680C49A6300EF028F856
:1009C00008E01B68074893F82210094A01F001016A
:1009D00010F0CCFD14B9074B02221A7010BD00BFF5
:1009E00024AB0100E082FF1FEC82FF1F45040000E2
:1009F000F9090000F082FF1F013808B5072823D845
:100A0000DFE800F0040E121416060A2F164808BD7F
:100A1000164B1868653008BD144B18687C3008BD4B
:100A2000124B1868873008BD114808BD114808BD31
:100A30000B88CC2B02D90020088008BD0E48C3F1DA
:100A4000CD020A80184408BD0C480D49042209F063
:100A5000FEFB0C4B187828B1013818700120FFF705
:100A6000A1FF002008BD00BFBA720100EC82FF1F89
:100A7000F081FF1F7E720100B0710100E082FF1F54
:100A800024AB0100F082FF1F7047013911F8013FCC
:100A900033B110F9012B5BB29A42F7D000207047B6
:100AA00090F90020202A07DC03461846013390F90C
:100AB0000020202AF9D070471846704730B50368E7
:100AC00002461946013391F90000202803D111682C
:100AD00001311160F5E700231846CC5C65B22F2D7B
:100AE00013DDE5B2A5F13004E4B2092C84BFA5F111
:100AF0003704E4B2000104F00F0480B2204314680C
:100B000001330134042B1460E7D130BD10B5036804
:100B100093F90020202A07D01A461346013293F990
:100B2000001031F02004F8D11A46013392F9001078
:100B30002029F9D0026092F90000D0F1010038BFFD
:100B4000002010BD83885BBA838003681BBA0360F2
:100B50007047000010B50C4609F0DEFC084809F0AB
:100B6000DBFC084B1B685B8C1C4004D0064809F07A
:100B7000D3FC012402E0054809F0CEFC204610BD5C
:100B8000A8A20100EC82FF1FF47B0100FE7B0100A4
:100B900010B50388DA0705D413F0020F0CBF022446
:100BA000012400E00024094809F0B6FC084B0520A8
:100BB00000FB043009F0B0FC064809F0ADFC064823
:100BC0000221BDE81040FFF7C5BF00BF097C01004E
:100BD000537B01003BAA0100147C010008B50548C5
:100BE00009F09AFC044809F097FC0448BDE8084065
:100BF00009F092BC207C0100C0920100337C01000E
:100C00002DE9F047DFF8D0902D4E99F800204FF0F5
:100C10000C0808FB02F2B31888B08246B5581F7959
:100C20005C7901A820211B2209F009FBBAF1000F11
:100C300004D054450FDD0C35013CFAE7214809F09A
:100C40006BFC99F8003008FB0366B06809F064FC9F
:100C50001D4809F061FC1D4E0C3554B3307800215D
:100C6000422209F033FC50B9184B4021187841F268
:100C70006D0209F0D3F8164B01201C601CE055F8FA
:100C80000C0C09F049FCB8420246307802DB01A99D
:100C9000012202E0BA1A01A992B209F017FC55F834
:100CA000080C09F039FC0B4809F036FC013C0C3506
:100CB000D3E7074B20461C6008B0BDE8F08700BFB3
:100CC000707B0100327C0100367C01003782FF1FFF
:100CD0001083FF1F337C01004484FF1F08B5094BBC
:100CE0001B78082B08D1084B1B681BB1186808B18A
:100CF00009F012FC054800E00548BDE8084009F08D
:100D00000BBC00BF4484FF1F1483FF1F9E93010090
:100D10007D820100B0F5000F08B505D34008002121
:100D200009F000FC054804E04002002109F0FAFB4C
:100D30000348BDE8084009F0EFBB00BF4E7C01004E
:100D4000567C01002DE9F04FADF5037D09280546DD
:100D5000019100F04282112800F03F82082800F043
:100D6000CF81152800F0F681A0F11D03DBB2012B25
:100D700040F2D2830B2800F01B839F4E306820B9CD
:100D80004FF4807108F0C4F8306031680C8F04F0C3
:100D90000204A4B24CB9204608F0DCF808B1974828
:100DA00073E2954B1A68964B1A60202D00F2B483BB
:100DB000DFE815F02600F50255024C020801080193
:100DC000B2038202A60113021302B2036102B2034C
:100DD000B203B203B20313021302B203B203D0018F
:100DE000C4022600B203F500B2032100F500B203ED
:100DF000B203B20326000023DDF80490019301E062
:100E00004FF000097F4F3C683CB901987C4908F0DD
:100E100043FA002801DA7C4837E27C4C0123A381A5
:100E20000DF108089023172DC4F80080238101D10B
:100E3000022302E01B2D02D10623237504E0202D9E
:100E400001D00023F9E725753B68C3B9704809F064
:100E500063FB3368186809F05FFB3368DB8E032B94
:100E600002D96C4809F058FB019820B190F9003084
:100E70000BB109F051FB684809F04EFB02E0614BF1
:100E800000221A60654EB34630780021932209F0A3
:100E90001DFB78B9614B4021187841F26D0208F0D2
:100EA000BDFF172D01D10423FCE0202D0CBF05232D
:100EB0000123F7E05248554907F09CFE63898246BA
:100EC000002B38D0172D03D1554809F025FB2CE015
:100ED0001B2D2AD10022023B19F9021031F0200EFD
:100EE000C2EB030001D00132F6E7F2B140444946BB
:100EF00009F041FBC8B9B4F80A904148A9F10209C8
:100F0000C14407F0EBFC10B14846464901E04649B0
:100F1000484609F055FB0D2303700A234370023045
:100F2000C8EB000060814FF000099BF80000628967
:100F3000414609F0CBFA1AF10F0FA5D10021608AC2
:100F400009F0F0FA394809F0E7FA0021606809F081
:100F5000E9FA374809F0E0FA0021208A09F0E2FABC
:100F6000344809F0D9FA00211822284809F067F915
:100F7000002008F0EBFD038B5E0709D5036B5D1CB9
:100F800006D090F82B005843FFF7C4FE2A48C1E270
:100F900003236D2100203B6008F066FD83E04CF2E6
:100FA000010344F201041C2D18BF23460198326846
:100FB00002A908F0FBFB002802DA204809F0ACFA8D
:100FC00002A89AE00F4F1E493A686D2381F83F301E
:100FD00040F61203042D18BF1123022A884602D1BD
:100FE000042D4CD12EE00198326808F0DFFB022876
:100FF00040F0B581F4E700BF1483FF1F5D7C010062
:101000004884FF1F9483FF1F707C01002083FF1F13
:10101000847C0100E5A201008F7C01003782FF1F64
:10102000937C0100977C0100B37C0100C07C01002F
:10103000CD7C0100D67C0100E57C0100ED7C010047
:101040004C83FF1FA34C4FF48072217802A809F053
:10105000F6F82378013323709F4C02A920464FF401
:10106000807208F093F9054608B19C482CE09C4832
:1010700009F052FAA068294609F054FA39E0994D6E
:10108000DFF854922E46287800214FF4807209F040
:101090001DFA50B9934B4021187841F26D0208F0C7
:1010A000BDFE02233B60012437E202AC00238A48E4
:1010B0003B6021464FF4807208F08CF818B9B9F8FB
:1010C0003C202E2303E0884809F026FA11E09042E4
:1010D00007DA215C0A39C9B2702988BF235401306C
:1010E000F5E73078214609F0F1F9B8F83C30FF2BEC
:1010F000C9D87E4809F010FA774808F02FF90BE2BA
:10110000019809F04EF80446794809F005FA20469E
:10111000842109F011FA2246002002A908F0D4FC2B
:10112000044608B17348F5E1704809F0F5F9254621
:1011300002AF00262F44B8599421043609F0FCF977
:10114000402EF8D16948403509F0E6F9B5F5007F41
:10115000EED1E2E1019809F024F8044601A8FFF776
:10116000D5FC20B9019809F01CF8C0B200E00020BD
:10117000002302ADC218B3F5007FD2B202D0EA5408
:101180000133F7E75C4809F0C7F92046842109F0EC
:10119000D3F95A4B40221A6001A8FFF7B7FC08B1F7
:1011A000012005E0019808F0FCFFC0B20028F7D04C
:1011B0000319DEB200202946224608F09FFC08B140
:1011C0004F4800E04F48013409F0A6F9E3B29E42CF
:1011D000F0D14A4B40221A609EE14B4809F09CF93D
:1011E000019B93F900202D2A16D193F90120312A71
:1011F00012D193F90230322B06D0362B0CD1434852
:1012000009F08AF9042203E0414809F085F9022235
:10121000019B0433019303E03E4809F07DF900226D
:101220000A2D01D0122D01D142F00102113DEDB283
:10123000012D98BF42F008020020019908F074FBCC
:10124000044608B1344865E134481EE0019831682D
:1012500008F026FB002800F05F8131485AE1019830
:10126000326802A940F2026308F0A0FA022800F0F6
:1012700053812C484EE1019A154612F8014B63B296
:10128000202B05D0002CF7D1274809F045F944E17F
:1012900000222A700198326802A908F087FA002813
:1012A00001DA224836E1681C02A908F009F8002892
:1012B00000F032811E482DE10198316808F092FA61
:1012C000441C01D11B4825E1002800F025811A4863
:1012D00020E100BF2882FF1F4C83FF1F087D010013
:1012E000157D01003782FF1F287D01003BAA010008
:1012F0004F7D01005F7D01006B7D01008CF00F4090
:101300007E7D0100957D01009D7D0100B07D010085
:10131000AC7D0100B47D0100B87D0100C77D0100F6
:10132000E67D0100F87D01000D7E0100207E0100B8
:101330002C7E01003C7E01004C7E0100019808F0EB
:101340004DFF0746019810F9012B202A0190F9D191
:1013500002A93268022308F029FA022801D0714854
:10136000D8E0002008F0F2FB3946046B0546002265
:1013700002A808F0E9F802A808F026FB68B96A4854
:1013800009F0CAF8286B001B00F0C380102109F097
:10139000C9F8664809F0C0F8BBE06548BAE00198B2
:1013A000316808F08BF8002800F0B6806148B1E0A1
:1013B000002008F0CBFB04465F4809F0ADF8238B12
:1013C00003F4807292B20AB15C48A3E0990601D49A
:1013D0005B480DE0134602A8E11891F84910195432
:1013E0000133202918BF1A460B2BF5D10023835453
:1013F00009F092F8534809F08FF82069FFF78AFC4A
:10140000514809F089F8238B5B0602D54F4809F053
:1014100083F84F4809F080F8238B9F060FD513F40B
:10142000C04F09D05E0402D54A4809F075F8238BF5
:101430009D0404D5484800E0484809F06DF8238B26
:10144000D80602D5464809F067F8464809F064F81E
:10145000238B990650D5444809F05EF81821208D59
:1014600009F060F8414809F057F894F82B30208DC6
:101470001821584309F056F83D4809F04DF89C21D1
:10148000606809F059F83B4809F046F89C21206A49
:1014900009F052F8384809F03FF89C21E06909F05A
:1014A0004BF8364809F038F8182194F82A0009F06A
:1014B00039F8334809F030F89C21A06809F03CF86D
:1014C000304809F029F89C21606A09F035F82E4867
:1014D00009F022F89C21E06A09F02EF82B4809F067
:1014E0001BF89C21206B09F027F8294809F014F813
:1014F000606B9C2109F020F8264809F00DF80025C2
:101500006319912193F83800013509F015F8102D71
:10151000F6D1144809F000F8002420460DF5037DAB
:10152000BDE8F08F3E7D01005C7E0100787E010009
:10153000887E01009C7E0100AB7E0100B67E01002A
:10154000C57E01008B940100FA8E0100D37E01005C
:10155000A77D0100D97E0100DC7E0100DF7E010055
:10156000E27E01003BAA0100F37E0100057F01003D
:10157000137F0100237F01002E7F0100387F0100CF
:10158000487F01004D7F01005D7F0100687F010001
:10159000777F0100827F010008B5802103466D221C
:1015A00005480FF038FB013004D10448BDE808407D
:1015B00008F0B2BF08BD00BF9883FF1F877F0100FE
:1015C00038B505460C460D48294608F0E3FF78B1CA
:1015D0000B48294608F0DEFF20B10A4808F09CFFBE
:1015E000012038BD084B1B685A8C22EA040403E032
:1015F000054B1B685A8C14435C8438BDA07F0100E6
:10160000A77F0100AF7F0100EC82FF1F1FB5694675
:101610000FF0B9FB684608F07FFF05B05DF804FBEA
:1016200010B5044686B0154808F076FF04F10800AE
:10163000FFF7ECFF124808F06FFF01A9A01C0FF0A4
:101640006BFB01A808F068FF0E4808F065FF04F185
:101650000C00FFF7DBFF0C4808F05EFF04F1100000
:10166000FFF7D4FF094808F057FF04F11400FFF713
:10167000CDFF074808F050FF06B010BDC27F010043
:10168000D47F0100E57F0100F67F01000B8001009F
:101690003BAA01000F4B1B88B3F5007F10B50A462B
:1016A00004460D4B10D00D49097805290CD102785C
:1016B0001878082A02D10A49032207E03A2A0CBF07
:1016C00021460849012201E018782146BDE8104072
:1016D00008F0FCBE1C83FF1FE882FF1F9283FF1FE0
:1016E000627B0100FBA501000E4B1B6837B55C8CCB
:1016F0000D4D04F01004A4B24CB1188C0B4B002219
:1017000000937821134612F087FA287007E095F9C4
:10171000000012F0FCFA064B1C80064B1C7003B054
:1017200030BD00BFEC82FF1F2082FF1F7D3600000E
:101730001C83FF1F9283FF1FF0B5544F847B97F9E2
:101740000030002B8BB001DAFFF7CEFF0DF1090658
:10175000204602A9052208F07BFB002800F09380B8
:101760009DF80B309DF80C20412B3CD0692B63D0A9
:10177000012B40F08380DD2A1CD1454B1B6893B1BF
:10178000012B02D1002001460BE0042B01D11720D0
:1017900006E0052B01D1202002E0022B03D1052019
:1017A0000021FFF7CFFA3B4B18680028D0D0FFF795
:1017B00027FACDE7BF2ACBD1354D2B68032BC7D1F4
:1017C000002008F0C3F9036B5A1C09D090F82B00D5
:1017D0005843FFF79FFA304808F09EFEFFF77EFA65
:1017E00000232B60B4E7204602A908F031FB9DF8E6
:1017F0000850042D1CD1314601220DF1070008F0DC
:1018000026FD264808F088FE9DF8070000F01F031B
:101810001D2B05DD1F2B9BD140B2FFF7BDFE97E7C7
:10182000002197F900000A462B4611F03EF88FE799
:10183000032D8DD11A481EE002A9204608F008FBAE
:101840000DF107003146012208F001FD9DF8083036
:10185000012B7FF47DAF9DF8073003F01F031F2B92
:1018600008D1104808F058FE0DF10A00FFF7CEFE2F
:101870000D4800E00D4808F04FFE69E7204602A938
:1018800008F0E6FA64E70BB0F0BD00BF2082FF1F4E
:101890009483FF1F1083FF1FE57C01001B80010064
:1018A0002C800100468001003BAA01005A80010003
:1018B00010B5094C2068FEF7DFFD206807490622B5
:1018C000023008F0C4FC206805491830B422BDE895
:1018D000104008F0BCBC00BFEC82FF1FF382FF1F6A
:1018E000C87201002DE9F7435B4D2B6806460C4694
:1018F000032B00F28B80DFE803F0022B2685574F85
:101900003B682BB94FF40070042108F0B9FE386031
:10191000534A00231360534A1360534B3A681A60CA
:1019200001232B6014E0514A5148083313600AF038
:10193000A9FB504B186002234F482B6008F0ECFDC8
:101940003846FFF7FFF83444454D1FFA84F954E058
:101950004548434902680B6840F2FF17BB4224D850
:1019600014B902600B6073E016F801CB0133013C3F
:10197000082B02F801CBA4B2F0D10B60374B026008
:101980001F683846FFF7DEF8BA8841F234239A42DE
:1019900001D03A4804E03B68B3F5003FC3D3384870
:1019A00008F0BAFD03232B6052E002600B60CAE727
:1019B000B3B299452AD02C4F3B685A1C01343A6087
:1019C00016F8012B2C60B4F5007F1A7015D12D4844
:1019D000DFF8888008F0A0FD264BD8F800101868C2
:1019E00022460AF0A7FB1F4B1A6802F500721A6024
:1019F00000232B60D8F800303B602C68B4F5007FE2
:101A0000D6D303E020BB19BB296021E0154B144954
:101A1000164A1B68096812681944914218D30621B6
:101A20009A428DF80710134C05D90C4920680968B3
:101A3000D21A0AF07FFB0DF1070120680AF036FC8C
:101A4000114808F069FD61206421832208F0DAFF63
:101A500003B0BDE8F08300BF1883FF1F3C83FF1F66
:101A60007484FF1F4083FF1F4084FF1F7C84FF1F7F
:101A7000AB8001003883FF1FAD800100778001003B
:101A800091800100FBA50100BB800100022838B550
:101A90000546184C1AD02168182248F204000AF0B2
:101AA0008BFA216848F21C001831B4220AF084FA3B
:101AB000012D1CD002200AF0B9FA0E4B19680E4B0A
:101AC00018311868B42208F0C2FB10E00A4B2068F5
:101AD0001B685A89438C5340990701D5012038BDB2
:101AE0000649182208F047FD0028D4D0F6E7002068
:101AF00038BD00BFEC82FF1FE482FF1FC882FF1FBA
:101B000038B50F4B1B68D9789C789D7901EB04247C
:101B1000597902460904D87901EB05210144187965
:101B200001EB0060022108F081FA2D23A4B20246E5
:101B300003700A2120460132BDE8384008F076BA29
:101B4000EC82FF1F7FB5064808F0E6FC01A8FFF70E
:101B5000D7FF01A808F0E0FC07B05DF804FB00BF68
:101B6000D68001007FB5831E0B2B44D8DFE803F03D
:101B700006431143434339341824182CFFF7E2FF7E
:101B8000FFF72CF81D4808F0C7FC1D4B18683930CA
:101B90001FE01B4B18681422393008F058FB2AE06C
:101BA00001A90C2814BF032004200BF0C9F801A8D8
:101BB00008F0B2FC13480CE010200BF0C1F81248FA
:101BC00008F0AAFC0C2013E0102000210BF0B8F85C
:101BD0000E4808F0A1FC0EE008200BF0B1F80C480C
:101BE00003E020200BF0ACF80A4808F095FC0A202E
:101BF0000021FFF7B7FF07B05DF804FBE8800100A4
:101C0000EC82FF1F3BAA010000810100108101004E
:101C1000208101002F81010008B5184B1B88B3F506
:101C2000807F03D12020FEF77BFC13E0144B1A8841
:101C3000B2F5006F05D14FF480521A8003F0A6F977
:101C400008E0104B04221A800F4B032193F9000087
:101C500012F010F8FFF776FFFEF7C0FF0B4808F010
:101C60005BFC0B4B1868393008F056FC094B002020
:101C70001870BDE80840FEF7C3BF00BF9083FF1F88
:101C80004684FF1F1C83FF1F2082FF1FE880010086
:101C9000EC82FF1F4484FF1FB0F5807F08B5034628
:101CA0000AD0B0F5006F0D4A0FD11288A2B90C4AC4
:101CB00012888AB90B4A0AE00A4B1B8863B9074BA2
:101CC0001B884BB9FEF72CFC02E04FF40073138025
:101CD000FFF7A2FF002008BD022008BD1C83FF1FE4
:101CE0009083FF1F4684FF1F38B503460846013125
:101CF00090F900202B2AF9D0042B16D0072B27D0DF
:101D0000032B2AD1154C256808F068FA236885F85A
:101D10004E0093F84E20632A01D9632202E0092A7B
:101D20001BD80A2283F84E2038BD0C4C256808F0D9
:101D300055FA236885F84F0093F84F20632A01D99C
:101D4000632202E0092A08D80A2283F84F2038BD0E
:101D5000024B1C6808F042FA208438BDEC82FF1F59
:101D6000054B1B68598C4B0703D5C1F3C0110DF00F
:101D700093BE0DF0D5BE00BFEC82FF1F1F4B204A63
:101D80001B681268D8695168884210B50BD1B3F846
:101D90004E00D18E884206D193F82440117B641AFC
:101DA00018BF012400E0012452895B8C53409BB290
:101DB00013F0280F18BF44F00204590748BF44F03D
:101DC0000404DA0648BF44F008040120FEF7FAFBD9
:101DD000E30702D50420FEF797FCA00701D502F027
:101DE00071F8610702D53C20FFF7BAFF220703D53F
:101DF000BDE81040FFF778BC10BD00BFEC82FF1FAC
:101E0000E482FF1F054B0A46014693F900001123A7
:101E100009B90349082310F048BD00BF2082FF1F05
:101E20007C740100313803283FD8DFE800F002114C
:101E3000202F1F4B1F491A6809681868043B1B684C
:101E400023EA000001EA02031843C0F34010704780
:101E5000174B18491A6809681868043B1B6823EA7D
:101E6000000001EA02031843C0F380107047104BD2
:101E700010491A6809681868043B1B6823EA0000C7
:101E800001EA02031843C0F3C0107047084B094928
:101E90001A6809681868043B1B6823EA000001EA15
:101EA00002031843C0F3002070470020704700BFB2
:101EB00094F00F4080F00F402DE9F843124B1A6860
:101EC00092F85070B2F852800125312000249946D2
:101ED000461C40B2F6B2FFF7A5FF00B12C436D00DF
:101EE000392EEDB201D0F0B2F2E7FFF747FFD9F893
:101EF000003083F8507083F85140A3F852800020DE
:101F0000BDE8F843FFF7C2BDEC82FF1F313803285C
:101F10001FD8DFE800F0020910170F4B186880F097
:101F20002000C0F3401070470B4B186880F0400051
:101F3000C0F380107047084B186880F08000C0F331
:101F4000C0107047044B186880F48070C0F3002004
:101F500070470020704700BF94F00F40303870B5D4
:101F6000032852D8DFE800F002090406202405E027
:101F7000802403E04FF4807400E04024642945B2DB
:101F80000AD002DC612940D003E0692904D06F291E
:101F90001FD04FF0FF3070BD14F0E00635D11C4B60
:101FA0001A6842F400621A601A4B1A6822EA0402A4
:101FB0001A60022040F20312214614F057F8164B23
:101FC0001B68012093F8502000FA05F522EA050568
:101FD00019E014F0E00618D10D4B1A6842F40062C3
:101FE0001A60022021464FF4827214F03FF8094B28
:101FF0001A6814431C60084B1B68012093F850209A
:1020000000FA05F5154383F85050002070BD00BF5D
:102010003880044094F00F40EC82FF1F61380F2895
:102020004DD8DFE800F0080D12171C1E20222429CD
:102030002E33383D4247234B1868C0F300207047C9
:10204000204B1868C0F3402070471E4B1868C0F33F
:10205000802070471B4B1868C0F3C0207047194B95
:1020600006E0184B09E0174B0CE0164B0FE0164B3F
:102070001868C0F300307047134B1868C0F3403045
:102080007047114B1868C0F3803070470E4B1868CA
:10209000C0F3C03070470B4B1868C0F3C0007047E6
:1020A000084B1868C0F300107047074B1868C0F35E
:1020B00080407047044B1868C0F3C0407047002050
:1020C000704700BFC0F00F4080F00F4061380F280C
:1020D00039D8DFE800F0080B0F1215181B1E212459
:1020E000272A2D2F31344FF4807201E04FF4007213
:1020F0001B4B27E04FF48062FAE74FF40062F7E7EA
:102100004FF48052F4E74FF40052F1E74FF480426D
:10211000EEE74FF40042EBE74FF4805211E04FF44A
:1021200000520EE04FF480420BE04FF4004208E012
:102130000822DDE71022DBE74FF4802201E04FF4B4
:102140000022084B1A60084B1B68012202FA00F0BB
:10215000B3F852205040A3F852000020704700BF4F
:10216000CCF00F408CF00F40EC82FF1F21B1094BE7
:102170001A6842F400621A60074B1A6810F0080FE0
:1021800014BF4FF48071002122F4F0720A431A60E8
:10219000704700BF3880044080F00F402DE9F84FB1
:1021A000BB4E336893F8510093F85050284083F8A1
:1021B00051000121FFF7DAFF01243020B0462C4204
:1021C00000F1010614BF6F216921F6B240B2FFF79A
:1021D000C5FE6400382EE4B201D03046EFE7AD4CC6
:1021E000AD4EAE4D61235F1C5BB2623BFFB20E2B66
:1021F00010D8DFE813F01E002D003D004C005B00FE
:102200006A00790088009700A600B500E200E200AD
:10221000C400D300236843F48053236003204FF4A9
:1022200080714FF4827213F021FF2B6843F48073A6
:102230001CE0236843F48053236003204FF40071B3
:102240004FF4827213F012FF2B6843F400730DE019
:10225000236843F48053236003204FF480614FF4DC
:10226000827213F003FF2B6843F480632B60A4E0B9
:10227000236843F48053236003204FF400614FF43C
:10228000827213F0F3FE2B6843F40063EEE72368D9
:1022900043F48053236003204FF480514FF4827243
:1022A00013F0E4FE2B6843F48053DFE7236843F424
:1022B0008053236003204FF400514FF4827213F0D7
:1022C000D5FE2B6843F40053D0E7236843F48053D2
:1022D000236003204FF480414FF4827213F0C6FE56
:1022E0002B6843F48043C1E7236843F480532360A1
:1022F00003204FF400414FF4827213F0B7FE2B68B5
:1023000043F40043B2E7236843F4006323600220F0
:102310004FF480514FF4827213F0A8FE336843F4F7
:10232000805349E0236843F40063236002204FF4A4
:1023300000514FF4827213F099FE336843F4005356
:102340003AE0236843F40063236002204FF48041A5
:102350004FF4827213F08AFE336843F480432BE01B
:10236000236843F40063236002204FF400414FF4DC
:10237000827213F07BFE336843F400431CE0236851
:1023800043F40063236002204FF480214FF48272F3
:1023900013F06CFE336843F480230DE0236843F4AC
:1023A0000063236002204FF400214FF4827213F087
:1023B0005DFE336843F400233360712F01D0FBB21C
:1023C00011E7D8F80030364A36483749374CB3F869
:1023D00052A0102501234FF400462F464FF4802CC5
:1023E0004FF400284FF0080913EA0A0F6FD0802B32
:1023F0004CD016D8082B3ED009D8022B35D0042B50
:1024000036D0012B40F0BF804FF4807B3BE0202B87
:1024100034D0402B35D0102B40F0B5804FF4805B8A
:1024200031E0B3F5006F4BD00CD8B3F5007F3FD04F
:10243000B3F5806F3FD0B3F5807F40F0A4804FF4B8
:10244000805B3AE0B3F5005F3CD005D8B3F5805F20
:1024500008BFC1F8009096E0B3F5804F34D0B3F5D3
:10246000004F08BFC4F800808DE04FF4007B0AE005
:102470004FF4806B07E04FF4006B04E04FF4005B17
:1024800001E04FF4804BC1F800B07CE00E607AE0D0
:10249000EC82FF1F3880044094F00F40D4F00F40CE
:1024A000C8F00F4088F00F40C4F00F4084F00F4098
:1024B0004FF4005B01E04FF4804BC4F800B062E0E1
:1024C000266060E00F605EE0C4F800C05BE0802B37
:1024D00049D014D8082B3BD008D8022B32D0042B7B
:1024E00033D0012B4FD14FF4807B39E0202B32D0F9
:1024F000402B33D0102B46D14FF4805B30E0B3F546
:10250000006F3AD00BD8B3F5007F2ED0B3F5806FB3
:102510002ED0B3F5807F36D14FF4805B2AE0B3F53F
:10252000005F2CD005D8B3F5805F08BFC2F80090DB
:1025300029E0B3F5804F24D0B3F5004F08BFC0F8B1
:10254000008020E04FF4007B0AE04FF4806B07E04E
:102550004FF4006B04E04FF4005B01E04FF4804B5C
:10256000C2F800B00FE016600DE04FF4005B01E030
:102570004FF4804BC0F800B005E0066003E0176040
:1025800001E0C0F800C05B00013D9BB27FF42CAFBE
:10259000BDE8F88F10B52B4B1A78110604462FD4DE
:1025A0001A7892072ED41A7850072DD41A789106EB
:1025B0002CD41A781B78D20704D513F0400F224987
:1025C000224B1AE0580623D4214B1A78D10721D484
:1025D0001A78920720D41A7850071FD41B7819074D
:1025E0001ED41B4B1A78D2061CD41A7890061BD422
:1025F0001B78184913F0800F174B18BF194614E0C9
:10260000164912E0164910E016490EE016490CE092
:1026100016490AE0164908E0164906E0164904E0A2
:10262000164902E0164900E0164924B9084607F0A9
:1026300073FF204610BD204607F0C2FF001BC0B24A
:1026400010BD00BF00F00740447601007076010025
:1026500001F00740527601004B760100D47301006F
:102660009C780100767A0100EB750100667B010021
:10267000C4780100A57401009C740100DD730100A1
:10268000E47501007D74010038B514F0B3FB00243B
:102690000546631E082B06D8DFE803F007090B0D7B
:1026A0000F1113151700104810E010480EE01048E5
:1026B0000CE010480AE0104808E0104806E0104816
:1026C00004E0104802E0104800E0104807F024FF42
:1026D000A54202D10E4807F01FFF0E48013407F053
:1026E0001BFF0A2CD5D138BD3E8101004681010077
:1026F0004F81010058810100618101006A81010060
:10270000728101007C8101008681010090810100BD
:102710009A8101003BAA01002DE9F0470C468EB0DA
:1027200015460B2800F24E86DFE810F00C0045003D
:10273000E202FD0264036604AC05B105A7024C0683
:102740004C06C30209B9084605E0042908D1012254
:102750009E4B00201A70FEF753FA044600F033BE79
:10276000052908BF0222F3D0062908BF0322EFD0B3
:10277000072908BF0422EBD0092908BF0522E7D0AA
:102780000A2908BF0622E3D00E2908BF0722DFD09E
:102790000F2908BF0822DBD0102908BF0922D7D093
:1027A000112908BF0A22D3D0122940F00B86874B8B
:1027B00000201870CFE70292202900F20386DFE89C
:1027C00011F021003800CB000106B7007A000106A5
:1027D00001060106010659006300B3000106010667
:1027E000E500C901C901010601060106010601064D
:1027F0000106010601062500E500C901C9013E02E6
:102800002D00310014F0B8FB00F0DCBD704807F07B
:1028100083FE0020FFF7BEFE00F0D4BDFFF734FFBB
:1028200000F0D0BD92F90000303814F03BFB00F00E
:10283000C9BD684807F070FE674807F06DFE67483D
:1028400007F06AFE07F05CFF822107F075FE64481E
:1028500007F062FE07F048FF822107F06DFE614835
:1028600007F05AFE07F034FF822107F065FE5E484C
:1028700000F0A2BD04A80AF097FC002404705B4895
:1028800007F04AFE04A8F3E11378313BDBB2032BD7
:1028900002D9574800F090BD564807F03DFE029B14
:1028A00093F90000FFF732FB044608B95248DFE114
:1028B000524800F081BD1078A0F13103DBB2032B48
:1028C00002D94F4800F078BD40B2FFF71FFB044625
:1028D00010B14C4800F070BD054601263120471C60
:1028E00040B2FFB2FFF79EFA08B13543EDB2760071
:1028F000352FF6B201D0F8B2F1E7029807F051FC9B
:10290000C0B2461E02980123184403FA06F602904C
:1029100007F047FC01280CBF3543B543E8B200215E
:10292000FFF724FC00F04FBDFFF7C6FA00F04ABDE8
:102930001378313BDBB2032BC3D8334807F0ECFDEF
:10294000029B93F90000FFF76DFA044610B12F487F
:1029500000F032BD2E488BE10EAC104644F82C2D11
:1029600007F01FFC05462046FEF7D0F810B12948B5
:1029700000F022BD039B05F12F0040B293F9001037
:10298000FFF7ECFA002800F01D85F0E792F900301F
:102990000BB9102653E0104607F003FC1E4B1860DD
:1029A00002A8FEF7B3F8029B1A78002AF1D002F0D1
:1029B000DF0252B24C2A01D1042102E0572A2FD162
:1029C0000221164A0133116030E000BF4484FF1F2A
:1029D000A4810100B8810100397C0100CF81010090
:1029E00053800100DC810100337C0100EE81010095
:1029F000138201002582010038820100418201001A
:102A0000498201005882010068820100758201003C
:102A10005DA40100798201004483FF1F2482FF1F0F
:102A2000422A04D1A54A012111600B440293029865
:102A300090F90030002BACD007F0D0FB0646A04840
:102A4000DFF878A207F068FD20238DF810308DF8AC
:102A500011305746002E40F3B5849A4D84212868E2
:102A600007F06AFD984807F057FD0DF112084FF086
:102A70001009DAF80020022A06F1FF3617D0042ADE
:102A800028D0012A40F09E841B2C07D128680DF124
:102A9000060113F09BF99DF8063001E02B681B78C6
:102AA0003968039341F010019DF80C0020E01B2CC5
:102AB00007D128680DF1060113F088F9BDF806303A
:102AC00001E02B681B883968039341F01001BDF8C1
:102AD0000C000DE01B2C04D1286803A913F076F933
:102AE00002E02B681B6803933968039841F01001DA
:102AF000C9B207F021FD3B682A6803981A44022BEB
:102B00002A60C3EB090904D0042B0CBF1822002251
:102B100000E00822434498450ED020FA02F1A1F1CA
:102B2000200C5FFA8CFCBCF15A0F94BFC9B22E2165
:102B300008F8011B083AEEE716B1B9F1000F98D179
:102B40000D221A700A225A7000229A7004A807F007
:102B5000E3FC7FE792F90030002B00F0338410464D
:102B600007F01FFB112C054601D01D2C01D1574841
:102B700000E0574807F0D0FC02A8FDF7C7FF029B12
:102B80001A78002A00F01E8402F0DF0252B24C2AAA
:102B900001D1042102E0572A04D102214D4A013318
:102BA000116005E0422A04D14A4A012111600B4418
:102BB000029302A8FDF7AAFF029807F0F2FA049028
:102BC00002A8FDF7A3FF112C01D01D2C06D10298FD
:102BD00090F9003013B107F001FB00E001201C3C2C
:102BE000E4B23C4F012C8CBF002401240646B846B9
:102BF000002E40F3E7833A68022A0AD0042A13D051
:102C0000012A17D1049B14B18DF80C3005E02B700C
:102C100010E0049B34B1ADF80C30284603A913F042
:102C200083F807E02B8005E014B1284604A9F6E7F5
:102C3000049B2B60D8F80030013E1D44D8E792F980
:102C40000030002B00F0BE83104607F0AAFA0446BD
:102C500002A8FDF75BFF029890F9001011B107F090
:102C6000A0FA0146204613F045F8044618B91A4860
:102C700007F052FCA7E319489EE311B1012909D0DE
:102C8000A0E3174807F048FC164B1A8842F480422C
:102C90001A8098E3134C2388B3F5805F01D0124863
:102CA0008AE3124807F038FC238843F4005323805A
:102CB00088E308461146FEF745F84EE52482FF1FDB
:102CC000818201004483FF1F92A3010092820100D0
:102CD000998201001C82FF1FA1820100AA820100CB
:102CE000BA8201004684FF1FF282010010830100B6
:102CF00049B1032940F06683A24B10461C6807F0D7
:102D00006DFA20845EE3A04D2B88042B05D19F48EB
:102D100007F002FC10232B8055E39D4B08461980D9
:102D2000FDF7FEFB4FE30492072900F24B83DFE837
:102D300001F004284B5214575C3C04A8FDF7BEFE7A
:102D4000044604A8FDF7BAFE0EA9012201F82C0DD5
:102D5000204609F031F98F482EE304A8FDF7AEFEB6
:102D6000044604A8FDF7AAFE0EA9012201F82C0DC5
:102D70006FEA44406FEA504080B209F01DF986487E
:102D80001AE304A8FDF79AFE03A9012209F036F917
:102D9000002808DB814807F0BFFB9DF80C000921E3
:102DA00007F0CAFB0EE37E4806E3764C7D492068B7
:102DB000182207F04CFA20687B4B18301968B422AF
:102DC00007F045FA7948F7E2FEF772FD0020FEF7BA
:102DD0005DFE7748F0E2012009F028F97548EBE242
:102DE000022009F023F97448E6E20020FEF74EFEC7
:102DF0007248E1E2102900F2E582DFE811F01100EB
:102E0000190041004600630057007F00A000C00089
:102E10001E0052005F00E302E302E302E3024B0004
:102E2000104667490DF08DFF1F20FEF7B5FBC9E284
:102E3000544B19681046083130E062486249062256
:102E400007F099FB044608B16048B5E24D4E316881
:102E5000284602310DF037FF0028F5D031684FF0D9
:102E6000FF3304A802310622059307F0F0F904A904
:102E700022460223012012F01BFF14F07DF8A2E28B
:102E8000404B196810460C3108E03E4B196810465B
:102E9000103103E03B4B1968104614310DF051FF1F
:102EA00090E24048FEF7BCFB3E4804E0354C206809
:102EB000FEF7B6FB2068FDF76BFE83E200200AF008
:102EC0000BFE7FE24248434D07F026FB0024132609
:102ED000414807F021FB06FB045007F01DFB3F486B
:102EE00007F01AFBE0B200210AF0AEFD0134002128
:102EF00007F018FB122CEBD137485DE2214BDFF8CD
:102F0000F4801F6800264FF0050909FB068029465A
:102F100007F040FB044668B93B8823F003039BB2EB
:102F20002EB1012E40F0448243F0020340E243F010
:102F300001033DE20136032EE7D129483CE229484E
:102F400007F0EAFA002420460BF0E2F8054680B1CB
:102F5000254807F0E1FA05F10B00FEF757FB23487F
:102F600007F0DAFA681D04A90DF0D6FE04A807F0F0
:102F7000D3FA0134E4B2082CE5D11D481CE20BF071
:102F8000E3F81FE2EC82FF1F1C83FF1F2783010071
:102F90004684FF1F33830100458301005D830100E8
:102FA00072830100F182FF1FE482FF1F94830100FE
:102FB000B5830100D5830100F08301000D84010079
:102FC0009883FF1FF382FF1F24AB010025840100BB
:102FD00041840100207901003BAA010013A20100F5
:102FE000BC850100598401006F8401007E840100CA
:102FF0008D840100537B01001D2900F2E381DFE88D
:1030000011F01E006500320047008200E101E1017D
:10301000E101E101E101E101E101E101E101E101A0
:10302000E101E1019F00E101E101E101130113016F
:10303000E101E101E101E101E10127013B01A74BD0
:10304000A74F1E6800244FF0070808FB04702946AC
:1030500007F0A0FA10B986F82440B0E101340C2C36
:10306000F3D1A048A8E192F90030372B05D19B4B52
:103070001B68DA6942F0010206E0382B06D1974B53
:103080001B68DA6922F00102DA6198E1964893E15F
:10309000924B964F1E6800244FF0050808FB047001
:1030A000294607F077FA60B9F36923F006032CB1DB
:1030B000012C40F07F8143F002037BE143F00403E5
:1030C00078E10134032CE9D1894875E1834B894FBC
:1030D0001E68002407EB8400294607F05BFA68B9F4
:1030E000F369012C23F0180305D0022C40F0628113
:1030F00043F010035EE143F008035BE10134032C6D
:10310000E8D17D4858E1754B7C4F1E68002407EBE1
:10311000C400294607F03EFA68B9F369012C23F090
:10312000600305D0022C40F0458143F0200341E1CB
:1031300043F040033EE10134032CE8D170483BE109
:10314000664C704807F0E8F96F4807F0E5F9236826
:1031500093F824300B2B97BF614A6C48072000FB83
:10316000032007F0D9F96A4807F0D6F92368DB692C
:10317000DF074CBF6748684807F0CEF9674807F09B
:10318000CBF92368DB699E0705D413F0040F0CBF4D
:103190000223002300E00123544A052000FB032002
:1031A00007F0BAF95E4807F0B7F923685148DB69C0
:1031B000DD0654BFC3F3C003022300EB830007F016
:1031C000ABF9584807F0A8F92368DB69580605D41D
:1031D00013F0200F0CBF0025022500E00125524806
:1031E00007F09AF9454800EBC50007F095F9484803
:1031F00007F092F9002D00F0E5804C4807F08CF9BB
:103200002368002193F84E0007F08CF9484807F036
:1032100083F9484807F080F92368002193F84F00AC
:1032200007F080F94248C7E0104606F0D7FFC0B269
:10323000632803D8002808BF012000E06320274B43
:103240001B68152C0CBF83F84E0083F84F00B6E0C6
:10325000394807F061F9394807F05EF9012012F0AA
:10326000C1F8182107F05EF9354807F055F900203C
:1032700012F0B8F8182198E04FF0FF3012F0B2F8D1
:10328000304899E008461146FEF76CFC9AE00A299E
:1032900000F29880DFE801F00611145869611F966A
:1032A00096965B0010461021FEF78AF90446002826
:1032B00040F08880FEF718FA85E01046022149E0C8
:1032C00010460421FEF77CF9044600287AD13C2000
:1032D000FEF746FD77E0104640213BE0EC82FF1F01
:1032E000F0750100D285010095840100447B010046
:1032F000EB85010090740100FE85010078750100E6
:1033000014860100AD840100C6840100CE84010052
:103310003BAA010086950100D7840100D9840100F1
:10332000F4850100E1840100F0840100FE840100C5
:103330000A8501000E850100198501002E85010016
:103340003F850100508501001046082107E0104626
:103350004FF40071FEF734F934E010462021FEF7F7
:103360002FF978BB00F0AEFD2CE0194807F0D4F837
:1033700040211848FDF7EEFB04211748FDF7EAFB52
:1033800016480821FDF7E6FB18B115482021FDF786
:10339000E1FB14481021FDF7DDFB98B1124807F05E
:1033A000BBF8124B1B68188C082107F0BBF809E02A
:1033B0003B8008E0F36102E007F0AEF802E0042091
:1033C000FDF7A2F9002420460EB0BDE8F08700BF4B
:1033D0006B85010081850100DD8A01002C8B0100D5
:1033E000558B010095850100A3850100EC82FF1F2C
:1033F0002DE9F04F914E924C85B00546174689460F
:103400004FF00008B9F1000F00F013812A78082A64
:1034100009D1237823B1013B8A48237007F07CF857
:103420000023337000E11B2A04D05B2A05D13378D6
:103430001B2B02D132700135F6E033785B2B52D171
:10344000A2F14103032B4ED8DFE803F00E0E080271
:103450002378002B00F0E880013BE4E02378272B61
:1034600000F2E2800133DEE0DFF80CA2DFF8E4B125
:10347000DAF80020282000FB02B007F0ABF82A7829
:103480000390412ADAF8002007D10AB9032200E0AC
:10349000013ACAF800206C4806E00132032AC8BF8E
:1034A00000226A48CAF8002007F036F8039A32B1C1
:1034B0006748029207F030F8029A013AF7E763484A
:1034C00007F02AF8DAF80000282202FB00B0029286
:1034D00007F022F8DAF80000029A02FB00B007F0C9
:1034E00079F82070A0E00A2A00F09E80002A00F0FF
:1034F0009B80DFF884B194F800C0DBF800005549E8
:10350000282303FB00C00A542A780D2A7ED10A2200
:103510000A54384602910193FDF7D6F80299DBF878
:103520000020019B4C4803FB02134C492278097888
:103530004FF00C0E0EFB01F100EB010E0132D2B286
:1035400050F801809EF805E099180020CDF80CE0B5
:1035500001F8010C37B942490988002946D04905CC
:1035600006D543E0022F03D13E49098800293DD00A
:10357000002A38D04FF0000C039A624518461FD03D
:10358000D8F800100193CDF808C0FDF77EFADDF8F9
:1035900008C0019B0CF1010C024670B13248029246
:1035A00006F0BAFF98F8080098F80910029AFFF799
:1035B000B3F890B9FDF792FB0FE008F10C08DBE7D8
:1035C0002A49FDF762FA024668B104200921FFF793
:1035D000A3F810B9264806F09FFF3FB9204B188882
:1035E000FCF79EFF02E0234806F096FFFDF782F805
:1035F000DBF80010124B00221A7001311E4B032918
:10360000D4BF19601A604FF0010803E00CF1010CFF
:1036100084F800C00A49002333700B78272B05F18A
:10362000010501D92723237009F1FF391FFA89F910
:10363000E8E6404605B0BDE8F08F00BF8084FF1F7C
:103640007884FF1F637B01002D860100347C01001C
:1036500095A30100A083FF1F707B01004484FF1F1E
:103660009083FF1F4684FF1F3BAA010031860100A3
:103670007D820100798201009C83FF1F023970B5B1
:1036800006461446062961D8DFE801F0274157397C
:10369000326004002E4D2F4928680422253006F0A0
:1036A0006AFF28B92C4B1B8803F4917343B909E0D6
:1036B000286821462530042206F05DFF0028F1D05D
:1036C000022070BD254B1B8813F4C050F8D1244B49
:1036D00001221A80234B1E7070BD214B40221A809C
:1036E000204B002193F90000BDE8704010F0C2BAF1
:1036F0001D4B1A78FF2A02D11C4A12781A70184BF7
:10370000002018801A4B18701A4B187070BD144B9B
:10371000188840280CD1144A144910780870FF21E9
:1037200011704FF400721A80FEF776FA012070BD16
:1037300010280CBF0820002070BD20461946012229
:10374000FFF756FE003018BF012070BD002070BD8D
:10375000EC82FF1F24AB01009083FF1F4684FF1FF4
:103760001C83FF1F2082FF1F3782FF1F4883FF1F1C
:103770009283FF1F7884FF1F462810D005D8412868
:103780000FD044280FD102207047542805D0732849
:103790000BD0532807D140207047102070470420D9
:1037A00070472020704700207047012070470000BC
:1037B00048282ED00ED8372833D005D8312822D02B
:1037C000322838D110207047382824D0452832D1EB
:1037D00002207047522828D005D84E280DD04F28F7
:1037E00029D10420704758281DD06E2823D1134BAF
:1037F0001B68DB6913F0600F19E0104B1B68DB6975
:1038000013F0060F13E00D4B1B68DB6913F0180F64
:103810000DE008207047094B1B68DB6913F0010FAE
:1038200005E001207047202070474020704702D1FA
:1038300009B102230B700020704700BFEC82FF1F0C
:1038400044280BD002D841280AD014E0462803D0DF
:10385000532810D10120704702207047082070477C
:10386000064B1B68188810F0030004D111B1022325
:103870000B70704770470020704700BFEC82FF1F3D
:10388000F8B505461446002940F0B7810278413A60
:10389000342A00F2AE81DFE812F07B00AC01540064
:1038A000AC015F012401AC019301AC00AC0141000B
:1038B000AC0108013500AC01AC01AC01AC011B014D
:1038C000AC018A002001AC013B01AC01AC01AC01B0
:1038D000AC01AC01AC01AC01AC017000AC01AC01BD
:1038E000AC016501AC01AC01AC01AC01AC01AC01B7
:1038F000AC015A00AC01AC013201AC01AC013A00A0
:10390000AC019F009B4B9C4918680023D7E040788E
:1039100061380021C0B20AF097F816E0964897493E
:1039200006F04EFE95F90100FEF778FB10B19448C1
:10393000944901E09248944906F042FE1523238001
:10394000BEE1924B1868013018608B4D0DE1437851
:10395000682B07D0732B08D0662B40F0AF8106F0A0
:10396000CFFE04E006F0C0FE01E006F0B1FE8221C9
:10397000814A06F0CDFB0623E1E740786138C0B20A
:103980000AF0C6FB002800F034817B4D0B3088E044
:1039900040786138C0B20AF0BBFB002800F02981F2
:1039A000754D053029460DF0B7F9401B11E04378FD
:1039B000714D302B03D1284609F0F6FBF5E7322B89
:1039C00003D12846FEF7E6FD03E00320294609F06F
:1039D000B7F920802846F8BD664B186829300346A1
:1039E0001A46013392F900102629F9DC121A2280B6
:1039F000F8BD4378642B39D018D8472B46D004D86B
:103A0000363B012B40F2F58058E1532B45D0562B25
:103A100040F0548158484923037050234370762363
:103A200083703423C37004232380F8BD6D2B26D00C
:103A300008D8672B12D0692B40F040814D4B186895
:103A400008302DE0742B00F0D480762B0AD0732B35
:103A500040F03481474B18680C3021E0454B186822
:103A600010301DE04A4B18682D3019E0494B1B6897
:103A70005B89990713D4042323804748F8BD454B3D
:103A80001B685B899A07F6D5444809E0414B1B68DF
:103A90005B899B07EFD5424802E0424800E042487C
:103AA000354D29460DF06FF97FE74048324DB0F9AA
:103AB0000030002BA4BF2F4B1868023072E7C218E9
:103AC00092F839205A54002A3FF439AF0133F6E70F
:103AD000294D2846FEF714F867E708232380344869
:103AE000F8BD4378482B234B1B680CBF93F84E005E
:103AF00093F84F000021204A06F098FABCE0437882
:103B0000542B03D11B4B1B68188CF3E70020B3E048
:103B10004378303B042B18D8DFE803F00303070B8E
:103B20000F00144B1D68653512E0124B1D68873578
:103B30000EE0104B1D68A6350AE01E4B0E4A1868B1
:103B40000D4D002106F072FA02E000202080F8BD41
:103B5000284606F03FFD3CE7174806F03BFD208075
:103B60001548F8BD154B044D188800212A4606F06B
:103B70005DFA1AE7EC82FF1F9485FF1FB0930100E6
:103B8000A585FF1FC9920100AB9301008C85FF1F23
:103B9000D892FF1FE482FF1F24AB0100FD82FF1FAC
:103BA0000183FF1FE082FF1FF982FF1FF182FF1FC9
:103BB000C0920100248AFF1FF081FF1F8885FF1F2C
:103BC0009A682AB1937813B11088012202E01A464C
:103BD0000A2318466978312909D032298AD0302938
:103BE0006CD139480AB1394944E0394942E01846B4
:103BF00080E7042323803748F8BD28B99868294610
:103C0000042206F01CFBE5E60278302A39D19D68D3
:103C100025B9022283F84220002390E6AA7828885A
:103C2000504380B2814202D9002AF2D046E00139E5
:103C300089B291FBF2F602FB161297B20136B6B2C8
:103C400021483FB9012E0CBF2349244906F0B8FC96
:103C5000024606E0224906F0B3FC7B1C5E430246A6
:103C6000B6B20021304606F0E1F9AB78BB420CBF9A
:103C70001C491D4906F0A4FC134BC01A20801846AD
:103C8000F8BD312A1CD193F84220B1F5004F42F023
:103C9000080283F8422011D814480022125401323D
:103CA000B2F5807FFAD1B1F5004F22800AD193F8A6
:103CB000422042F0040283F8422003E00020F8BDD5
:103CC0000148F8BD0948F8BD9485FF1FD392010053
:103CD0000F930100CE920100429301007193010005
:103CE00063930100A0930100A59301008184FF1F4D
:103CF00037B500238DF807300378502B00F101040D
:103D00007FD013D8452B60D004D8422B47D0442B0A
:103D10003FD0BBE04D2B79D04F2B6BD0492B40F0DF
:103D2000B58090F90100FEF7F1F8ADE0622B1FD0ED
:103D300007D8552B3DD0612B0CD0532B40F0A680DB
:103D40004FE0642B1ED0C0F0A1806D3B012B40F2F0
:103D50009F809BE0504D514928680422253006F091
:103D60000AFC002800F0948028682146253001E0F4
:103D70004B492046042206F0FEFBD0F1010038BF7B
:103D8000002086E02046FFF7B3FF00287ED0032006
:103D90007FE02046FFF7ACFF0028F8D076E03E4BEE
:103DA00040781B6893F824304138C41A604260415F
:103DB0006FE0394B40781B680DF10701DC69FFF7B4
:103DC000F7FC20420AD0022063E0334B40781B68A6
:103DD0000DF107011C88FFF733FDF2E79DF807009E
:103DE00057E04078FFF7C8FC2B4B1B685B8C1842F0
:103DF000E9D14BE090F90100FEF788F80028E2D005
:103E000044E090F90100FEF70DF83DE090F9013033
:103E1000303B062B3AD8DFE803F0040C11191E27BB
:103E200031001D4B1D4918680622023006F0A3FB25
:103E300026E0194B1B491868083003E0164B1A4955
:103E400018680C30042206F096FB1DE0124B17494F
:103E500018681030F6E7104B1B681888144B1B8845
:103E6000C01A18BF01200FE0124B1A680A4B508984
:103E70001B685B8C5840C0F3400005E0FCF70EFC6B
:103E8000D0F1010038BF002000289CD1002000E0C4
:103E9000012003B030BD00BFEC82FF1F24AB010046
:103EA000C2930100D082FF1FD482FF1FD882FF1F60
:103EB000C882FF1FE482FF1F61206421832206F075
:103EC000A1BD0000104B1868438C1A0710B516D519
:103ED00013F0200F00F125000C494FF0040214BF2D
:103EE0000724032406F047FB08B144F008042346E6
:103EF00007480849084ABDE810400CF05DBDBDE820
:103F000010400CF0C9BD00BFEC82FF1F24AB0100C4
:103F10001D3F0000F13C0000813800005328F8B537
:103F20000C46154600F0B28030D8482800F0E081F9
:103F300014D8422800F0B28004D8002863D0412869
:103F400068D0FDE1452800F0C280462800F05A8183
:103F5000442840F0F5810AF0F7F8F1E14E2800F02E
:103F6000F08007D8492800F0FC804D2840F0E88117
:103F7000B04B54E1502800F02481C0F02E8152282B
:103F800040F0DE81002009F0A7FDD9E16F2800F0A4
:103F90001F8114D85A2800F0328106D8552800F025
:103FA0008480582800F08881CAE1652800F0988054
:103FB0006E2800F0FE80632840F0C281E9E0752899
:103FC0007CD00ED8702800F01281732840F0B881A0
:103FD000994B08781D68FFF7CFFB6B8C58406884BD
:103FE000AEE1FA28C0F0AC81FB2806D9FE2840F0EB
:103FF000A781002382F82230A2E1904B928A1878A0
:1040000006F064FA9CE18E4B18808E4B18608E4B44
:10401000187095E191F90130313B032B31D8DFE87D
:1040200003F01E02252E844B854A1B6811885A8C8A
:1040300041F0080102F002020A435A840220FDF70F
:1040400025FD20B10120FDF721FDFFF735FFFFF72A
:1040500039FF3C20FDF784FEFDF746FB70E1764B0F
:104060001B68002283F829200133FBE7FDF720FCC1
:104070000220FDF70BFD20B10120FDF707FDFFF742
:104080001BFFFDF77BFE00226D4B13E16C4D0878A2
:104090002E88FFF771FB3043288051E1664B4A7848
:1040A0001B68413A83F824204AE1664D88782E68DF
:1040B0000021FFF77DFB3043286041E15E4B1A6829
:1040C000604B1B680420D361FCF71EFB38E15E4D9A
:1040D00048782E780021FFF7B3FB304328702FE19A
:1040E00091F90030712B26D004DC532B35D06D2B89
:1040F00005D025E1722B21D0732B28D020E1FCF7CD
:10410000CDFA90B94C4B504A1B6811781A8822F0AE
:104110000B020A431A804A4A11885A8C41F008015E
:1041200002F055020A435A840AE1022007F07EFF9A
:10413000FCF7BCFA04E1FDF7BFFE01E1FDF71EFE4E
:10414000FEE03D4B18680131393010F00DF90220C6
:10415000FDF79CFC002800F0F3800120FDF796FCA1
:104160004DE091F90030692B08D0732B0AD0672BF2
:1041700040F0E680304B1968103106E02E4B19688C
:10418000083102E02C4B19680C31A01C0CF0D9FD51
:10419000D6E0294D2D4928680622023006F0EBF9B9
:1041A000002840F0CD802968601C02310CF08BFDA6
:1041B000C6E091F90030542B40F0C2800720023154
:1041C00026E091F9000091F90210FDF7C7FEB7E073
:1041D00091F90000FDF77AFFB2E091F90020184B49
:1041E0000121303A01FA02F219880A4362E0144CC4
:1041F00000212078FDF7BAFF00232380A0E0FFF71D
:104200005BFE9DE011F9023B482B0CBF032004200C
:10421000FDF76AFD94E0202A06D003F8011B14F88C
:10422000011F4AB2262AF6D100221A70084A01203C
:10423000131830E0F081FF1FEC82FF1F3782FF1F51
:104240008685FF1F9085FF1F8585FF1F24AB01001A
:10425000EF81FF1F252923D15E789D78A6F13001DB
:10426000C9B2092903F10207A5F13003DBB284BF0B
:10427000A6F13701C9B2092B84BFA5F13703DBB220
:1042800043EA011353703B4694F900200133402A5E
:1042900008BF002022461978541C0029DAD101E019
:1042A0005170F1E7217000284AD1FCF77BFB254BC8
:1042B0001A8801321A8043E091F90030303B032B19
:1042C0003ED8DFE803F002060A0E1F4B186865307F
:1042D0000AE01D4B18687C3006E01B4B18688730DD
:1042E00002E0194B1868A630A11C10F03DF827E039
:1042F00093681BB9042006F09BF9A86094F900307C
:10430000AD68312B0CD1A01C05F068FFC0B208B914
:10431000012303E00C28A87012D90C23AB700FE026
:10432000322B0DD1A01C05F059FF80B208B9012332
:1043300005E0B0F57A7F288002D94FF47A732B809C
:104340000020F8BD8885FF1FEC82FF1F10B594B0D8
:10435000169C2378452B40F0A18063784C2B40F0CD
:104360009D80A3785A2B40F09980E378452B40F04C
:1043700095802379542B40F091806379492B0AD0A2
:10438000532B40F08B80102203A8214605F05FFFDD
:10439000227801234AE005AC00213B22204605F0AB
:1043A0004EFF40490522204605F051FF41233E497A
:1043B0008DF8193004220DF11A0005F048FF0DF1B7
:1043C0001E003A49042205F042FF394B1B685B8C02
:1043D00003F002039BB203B1012306220DF1230077
:1043E00034498DF8223005F032FF0DF12900092102
:1043F000FCF7C6F856238DF8323031238DF8333070
:104400002D4A2E4992F900002E238DF8343037239F
:104410008DF835303B2200238DE80C008DF83630C6
:1044200040F23A5203AB0FF081FD35E0E15C01331D
:104430000F2B82EA0102F9D19DF81B309A422DD14F
:104440000DF112010422184805F001FF042217485B
:104450000DF1160105F0FBFE154B9DF81A201B68A7
:1044600042B15A8C42F002025A846FF01E000AF0E8
:104470006BFA0BE05A8C22F002025A8409F064FEB7
:10448000094861214FF0FF3209F0CCFD022007F00E
:10449000CDFD0020FDF7FAFA012000E0002014B065
:1044A00010BD00BFC6930100F982FF1FFD82FF1FF0
:1044B000EC82FF1FF382FF1F2982FF1F38AB010030
:1044C00010B5094C94F90030002B0BDA0749102085
:1044D00003220FF055FC207040F23A51BDE8104025
:1044E0000FF074BC10BD00BF2982FF1F4D430000B8
:1044F000022A2DE9F04704460D46164600F0B28028
:10450000042A02D0002A74D10AE00378832B40F0F9
:10451000AC80594B594918780D2205F0D7FFA4E01B
:10452000037823F08001212940F0A2808079E1798D
:10453000534F40EA012C13F0800FA7F800C06378B6
:1045400026D0FE2B3A8011D04CD8212B40F0908001
:104550006279237943EA02234A4A13605B1003F12C
:104560000A01C9B2752005F0F1FF3BE0A378002BEA
:104570007ED1E378002B7BD1012879D1002977D136
:10458000414B42491878012205F0A0FF00202AE0A3
:10459000202B1DD0222B6BD12379617943EA012195
:1045A000384B19603A4B1E78A3789B074CBF81218A
:1045B0008221304605F032FCA27812F0010230462A
:1045C0001ABF84210022882105F028FC03200AE07C
:1045D000304A13702379627943EA0222294B06207C
:1045E0001A6000E03046082D43D9083DADB20834CA
:1045F00000E00020224B1E889946002E39D0254B22
:104600001A78202A9A461ED11E4B1F68022397FB58
:10461000F3F7214B072E28BF0726072000FB0730A2
:10462000B54234BFA846B046C6F107031844214638
:10463000424605F00CFEB04505D307F11401752084
:10464000C9B205F083FFB9F800200D4B0021954257
:104650008AF8001001D3198007E0551B1D80062041
:10466000BDE8F0870020BDE8F0870320BDE8F087B3
:104670000420BDE8F08700BFF085FF1F2A82FF1FDE
:10468000D285FF1FE085FF1FFF87FF1FBD9401003C
:10469000E882FF1FD185FF1FF885FF1F2DE9F04736
:1046A000204D214F287800210A4605F00FFFB8461B
:1046B000044640F2FF1A3B6853B3544520D9DFF853
:1046C00078901A4E99F800003268002105F0FCF944
:1046D00080B999F80020164B287853F822304FF40F
:1046E0000072596905F0F2FE3368A4F500740133D5
:1046F000A4B23360D8F80030013BC8F80030DAE7E4
:104700002878402141F27502BDE8F04705F086BBEC
:104710000C2CF5D9287807490D22BDE8F04705F0A3
:10472000D5BE00BFF085FF1FEC85FF1FD885FF1F9A
:10473000F485FF1F2A82FF1FF185FF1F38B5364B16
:104740001B6804467BBB35482146042205F013FF55
:1047500028BB637B324A13700BBBA37B013BDBB2EC
:104760000F2B1CD894F90C30002BE37B2DDA232B74
:1047700023D016D9282B32D0A82B30D0252B1CD0F3
:10478000284D211D0422281D05F061FD05F10800BA
:1047900004F10801042205F05AFD01232B730420C3
:1047A00038BD122B01D1072038BD1A2B01D0032BA5
:1047B00030E0237C5B0929D0E2E71B4B1B681B8B95
:1047C00003F08803002BDBD0EDE71E2BEBD002D8E3
:1047D000002BE8D0D4E72A2B01D0AA2BD0D1124B42
:1047E0001A68138B03F08803002BC9D0A37C617C6B
:1047F0001B0443EA0163217D0B43E17C43EA01236F
:104800000A490B6012699342BAD2CCE7637C03F089
:104810003F033F2BB4D1C6E7D485FF1F2E94010080
:10482000F185FF1F2A82FF1FF485FF1FD885FF1F18
:104830002DE9F047B74E857B3378A6B01BB1B64C57
:104840000DF11D07A8E0B54BD3F8008008F1390041
:1048500005F0C0FEB24B44001A681ABFA71CFFB295
:10486000042799463AB9384605F0E2FE0323C9F811
:10487000000007704370D9F8003024B1023308F10A
:104880003801002002E09C70DC7008E011F8012F74
:10489000023322B103F8022C03F8010CF6E7A14B16
:1048A000002401274FF075082146019301AA062331
:1048B00005208DF81240ADF80E70ADF80A40ADF845
:1048C00008408DF814708DF815308DF8168005F0BD
:1048D00085FB4023ADF824301023214630708DF83D
:1048E00027708DF82670ADF822304FF400774FF422
:1048F00080734FF4806906AA05208DF82A800694FB
:10490000ADF81C30ADF81E90ADF8207005F066FBD8
:10491000854BADF8224018702146022306AA0520D7
:104920008DF826308DF827408DF82A400694ADF892
:104930001C40ADF81E4005F051FB7C4B8DF82A80E1
:10494000187003238DF827308DF82630784BADF89A
:104950001C702146052006AA0693ADF81E90ADF8FE
:10496000207005F03BFB734B734CDFF8F08118703F
:104970002778384605F0EAF8237848F8270001330D
:10498000DBB22370002BF3D059E79DF81B30012BCD
:104990000AD0752B00F01881284606A9052205F0DB
:1049A00057FA0028F1D126E19DF81C30CA2B3DD0E2
:1049B00005D80A2B00F0D680142B3DD0ECE7CC2B89
:1049C00005D01ED3DD2BE7D1FFF768FEE4E75B4B94
:1049D000DFF88C914FF00008C3F80080584BC4F802
:1049E0000080C3F80080B9F8003043B1554B1A7805
:1049F000554B40461A70FBF793FDA9F800805348C9
:104A0000F6E0DFF85C81B8F800304BB14D4B1A7816
:104A10004D4B00201A70FBF783FD0023A8F80030EF
:104A20000120002106F0E6FF4948E1E002200021D4
:104A300006F0E0FF4748DBE047498B7848780A7882
:104A40001B0443EA00231343CA7843EA0263B3F525
:104A5000613F23D8B3F5E13F22D8B3F5614F21D8A8
:104A6000B3F5164F20D8B3F5964F1FD8B3F5615F55
:104A70001ED8B3F5165F1DD8B3F5965F1CD8B3F5F5
:104A8000166F1BD8B3F5966F1AD8B3F5167F19D8E1
:104A9000B3F5967F94BF0023012314E00C2312E0AA
:104AA0000B2310E00A230EE009230CE008230AE0A0
:104AB000072308E0062306E0052304E0042302E0C0
:104AC000032300E002238A79D01F42424241487901
:104AD000012805D0022805D142F0020292B201E07D
:104AE00042F004020979012904D0022904D142F0DC
:104AF000100201E042F0080208490968C86981F81B
:104B0000243020F01F000243CA610420FBF7FCFDA3
:104B100042E700BFFF87FF1FD485FF1FEC82FF1F06
:104B2000DC85FF1FF1440000E485FF1FD085FF1FD7
:104B30003D470000F085FF1FF185FF1FEC85FF1F3B
:104B4000E885FF1FE882FF1F3782FF1F589401008E
:104B50006494010074940100F885FF1FF485FF1F21
:104B60004684FF1FBC4B1A6892F82430D2690C2B84
:104B70009CBFBA4951F82310B94B88BF4FF49641F6
:104B8000080A1970090C99700021D970D1074CBF1F
:104B90000721082158709007997101D5022103E07F
:104BA00012F0040118BF01215971110701D501222A
:104BB00003E012F0100218BF02221A713078A849DF
:104BC000072205F083FCE7E6284639469DF81C20BD
:104BD00005F03EF99DF81D30FE2B7FF4DDAEA148B7
:104BE00005F09AFC9DF81E00012105F09BFC9E48F3
:104BF00005F092FCD0E69D4E9D4FB046307805F012
:104C00003BF9002800F056813C68DFF864A2307858
:104C100044B3984C984D2168C1F5007292B2294472
:104C200005F016F93B681B1A3B6023681844B0F581
:104C3000007F206011DB914B1878914B1A68511C52
:104C40001960294604F05AFF002323603B6823B112
:104C50007520042105F0A4FE7EE1DAF80030002B77
:104C6000CCD120E1874DDFF8149206A9802205F00F
:104C7000EFF8042207A9281D05F0E9FA30782C7214
:104C800001216C72AC72EC722C7305F00BF99DF97A
:104C900024309DF82520002B89F800209DF827302E
:104CA00080F2AF80232B62D007D8122B2AD01A2B88
:104CB0002ED0032B40F0F78087E0282B3DD0A82B87
:104CC00042D0252B40F0EF806F4B307853F82220F4
:104CD00013698DF808408DF80940128D013B110AC7
:104CE0008DF80B201A0E8DF804201A0C8DF8052073
:104CF0001A0A8DF80A108DF806208DF8073001A9E0
:104D00000822CEE09DF828305B0900F0C78086E0DD
:104D10005E49042201A805F09AFA99F800205A4B3E
:104D200053F822301B8BD80644BF80238DF8063001
:104D300098F8000001A90422B3E09DF82E209DF808
:104D40002F3043EA02220DE09DF82E209DF82D30F1
:104D5000120442EA03629DF830301A439DF82F3066
:104D600042EA03224A4B1A60FFF798FC46E79DF897
:104D70002F309DF82E4047490C2201A843EA042415
:104D800005F065FA99F800203F4B53F82230198B53
:104D900011F0880F11D089064CBF022201228DF834
:104DA0000C201B691A0A8DF80B308DF80A201A0C9A
:104DB0001B0E8DF809208DF8083098F8000001A925
:104DC0000C2C34BF22460C226BE0122201A832497F
:104DD00005F03DFA99F800202B4B53F822301B8B3D
:104DE00003F0880343B970238DF8043002238DF853
:104DF00006303A238DF8103098F8000001A91222ED
:104E00004FE02A2B0ED0AA2B11D0002B4BD11E4BDA
:104E100053F822301B8B03F08803002B43D101236E
:104E20002B7340E09DF82E209DF82F300BE09DF86D
:104E30002E309DF82D201B0443EA02639DF830209C
:104E400013439DF82F2043EA02233B60DAF8003039
:104E50005B02CAF80030D1E6EC82FF1F34950100F6
:104E6000F885FF1F819401008E940100F085FF1FDB
:104E7000D485FF1FE885FF1FFF85FF1FF185FF1FFA
:104E8000D885FF1F2A82FF1FF485FF1FAF94010002
:104E9000EC85FF1FDC9401009294010030783049CA
:104EA000242205F013FB98F800002E490D2205F08E
:104EB0000DFBA3E62C4C2D4E2D4F207804F0DCFF8B
:104EC000002849D0338813F4C04F22D05A0416D595
:104ED00038780021402205F0F9FA40B106A94022B5
:104EE000207804F0B5FF06A9024638782EE0204B62
:104EF0004021187841F2750204F090FF2CE006A9D9
:104F00002078802204F0A4FF014606A8FCF7EAFC02
:104F1000D3E706A98022207804F09AFF054606A967
:104F20002A46207805F0D2FA338806A829460222BC
:104F30007BB9FEF75DFA0028BFD04FF40060FCF7A4
:104F4000ABFE0228B9D120780A49172205F0BEFA33
:104F5000B3E7FEF74DFAB0E726B0BDE8F08700BF33
:104F60000F9501002A82FF1FE485FF1F4684FF1F63
:104F7000E882FF1FF89401000A46034903460878B7
:104F8000194605F0A3BA00BFE485FF1F024B1A784B
:104F9000024B1A70704700BFE485FF1F3782FF1F66
:104FA000122303800048704732940100622303807B
:104FB00000487047CC930100052803460DD8094AE4
:104FC00052F82000027832B9032B08D1064B18683A
:104FD00003780B8070470A807047002070471046A6
:104FE000704700BFC0940100DC85FF1F042380F8D8
:104FF0006630024B03620020704700BF68950100D5
:10500000062380F86630024B03620020704700BF21
:1050100077950100064B1B6814225343432280F806
:1050200066206422B3FBF2F3C3610020704700BF27
:10503000248AFF1F042380F8663000230362184689
:105040007047042380F866300023036218467047D7
:10505000022380F866300123C3610020704790F876
:10506000642090F86B100244A12992F824300AD0F1
:10507000002B08BF0123022180F86610C36182F86B
:105080002430002070474FF0FF30704790F86420C4
:1050900090F86B100244A12992F824300BD004211F
:1050A00080F866100549002B08BF0123016282F8D1
:1050B0002430002070474FF0FF3070478895010082
:1050C00090F8642090F86B100244A12992F82430E3
:1050D0000BD0022180F86610002B08BF01230621A7
:1050E000C16182F82430002070474FF0FF307047D4
:1050F00090F8642090F86B100244A12992F82430B3
:105100000CD0022180F86610002B08BF012340F26A
:10511000DC51C16182F82430002070474FF0FF302D
:105120007047000090F8642090F86B100244A129A9
:1051300092F824300BD0422180F866100549002BEC
:1051400008BF0123C16182F82430002070474FF06E
:10515000FF30704700E1F50590F8642090F86B107F
:105160000244A12992F824300ED0012180F8661063
:105170000749002B08BF01230162062180F8671050
:1051800082F82430002070474FF0FF30704700BF96
:10519000F382FF1F90F8642090F86B100244A1295D
:1051A00092F824300BD0022180F86610002B08BF43
:1051B00001230121C16182F82430002070474FF0A3
:1051C000FF30704773B590F8683090F86420013371
:1051D0009A4204464FF0000516D0E21801A992F851
:1051E000242012F0800F05D00133E21892F8242019
:1051F00062F07F024A550135042D03F10103ECD121
:105200001F482A4605F0B7F994F86B30A12B32D02D
:10521000022384F866304BF68033E36194F86430FF
:105220002344002283F824200DB1002025E01548F6
:1052300081262B1894F864201B7A13F0800F03D179
:10524000224482F824300BE0511CC9B284F8641067
:105250002244214403F07F0382F8246081F8243043
:10526000032D04D094F86430013384F864300135A0
:10527000042DDED1D9E74FF0FF3002B070BD00BF82
:10528000F982FF1FF182FF1F73B590F8683090F824
:10529000642001339A4204464FF0000516D0E2180C
:1052A00001A992F8242012F0800F05D00133E218F2
:1052B00092F8242062F07F024A550135042D03F153
:1052C0000103ECD11E482A4605F055F994F86B30DD
:1052D000A12B31D0022384F866300123E36194F8D6
:1052E00064302344002283F824200DB1002025E0FF
:1052F000144881262B1894F864201B7A13F0800F31
:1053000003D1224482F824300BE0511CC9B284F846
:1053100064102244214403F07F0382F8246081F862
:105320002430032D04D094F86430013384F86430C1
:105330000135042DDED1D9E74FF0FF3002B070BD4A
:10534000F982FF1FF182FF1F73B590F8683090F863
:10535000642001339A4204464FF0000516D0E2184B
:1053600001A992F8242012F0800F05D00133E21831
:1053700092F8242062F07F024A550135042D03F192
:105380000103ECD11D482A4605F0F5F894F86B307E
:10539000A12B2ED0402384F86630194B23620423BE
:1053A00084F867300DB1002025E0164881262B18BF
:1053B00094F864201B7A13F0800F03D1224482F802
:1053C00024300BE0511CC9B284F8641022442144FB
:1053D00003F07F0382F8246081F82430032D04D089
:1053E00094F86430013384F864300135042DDED143
:1053F000D9E74FF0FF3002B070BD00BFF982FF1F48
:10540000FD82FF1FF182FF1F73B590F8683090F89E
:10541000642001339A4204464FF0000516D0E2188A
:1054200001A992F8242012F0800F05D00133E21870
:1054300092F8242062F07F024A550135042D03F1D1
:105440000103ECD11E482A4605F095F894F86B301C
:10545000A12B31D0022384F866300123E36194F854
:1054600064302344002283F824200DB1002025E07D
:10547000144881262B1894F864201B7A13F0800FAF
:1054800003D1224482F824300BE0511CC9B284F8C5
:1054900064102244214403F07F0382F8246081F8E1
:1054A0002430032D04D094F86430013384F8643040
:1054B0000135042DDED1D9E74FF0FF3002B070BDC9
:1054C000F982FF1FF182FF1F73B590F8683090F8E2
:1054D000642001339A4204464FF0000516D0E218CA
:1054E00001A992F8242012F0800F05D00133E218B0
:1054F00092F8242062F07F024A550135042D03F111
:105500000103ECD11D482A4605F035F894F86B30BC
:10551000A12B2ED0402384F86630184B236204233D
:1055200084F867300DB1002025E0154881262B183E
:1055300094F864201B7A13F0800F03D1224482F880
:1055400024300BE0511CC9B284F864102244214479
:1055500003F07F0382F8246081F82430032D04D007
:1055600094F86430013384F864300135042DDED1C1
:10557000D9E74FF0FF3002B070BD00BFF982FF1FC6
:10558000F182FF1F13B5042380F8663090F86B306A
:10559000A32B044606D1074B216818681522393021
:1055A0000CF09AFE0DF10700FAF7ACFF2062002024
:1055B00002B010BDEC82FF1F38B50C46154603281B
:1055C0002FD8DFE800F00F022721174805F002F876
:1055D000854216D1144821462A4604F0CCFF80B9F2
:1055E000012038BD114804F0F5FF854209D121465C
:1055F0002A460E4804F0BFFF003818BF6FF00000C5
:1056000038BD4FF0FF3038BD0846084904F0D8FFD8
:10561000001B38BD08460522054904F018FE052088
:1056200038BD002038BD00BF8F9501009C9501005A
:1056300097950100114910B500238B700B728B7385
:105640000B718B720B740323A82223244B7102234A
:10565000C0204A70CC70CA7163244A73CB72612235
:105660000123087088710873CA734C724B74044824
:10567000044ABDE810400CF00BB900BF0088FF1FC2
:10568000B9550000A4950100064B0A0E5A700A0C89
:105690009A700A0ADA700022187019715A71184645
:1056A000704700BFF489FF1F03688B4270B5044642
:1056B0000D461CD0038BDB070ED50E4E94F84830F8
:1056C000616956F823302268204698470130F5D0AA
:1056D000238B23F00103238394F84820064B256095
:1056E00053F82230626920462946984770BD002051
:1056F00070BD00BF008AFF1F1C88FF1F10B500236C
:105700001A46C45CD101C9B204EB5202013351FA0A
:1057100082F20B2BD2B2F4D1104610BD30B54468E2
:1057200085680B6804EBC505184C2C40002C03DA87
:10573000013C64F007040134072C25D8DFE804F0AD
:1057400004070A1215181E21C3F30B031CE0C3F350
:105750000B3319E01B0EBAB14A6802F00F0243EA9C
:1057600002230FE0C3F30B130EE0C3F30B430BE074
:105770001B0F4AB10A7943EA021303E0C3F30B2378
:1057800002E01B0D0022C260184630BD07000080F9
:1057900010B58468406800EBC4042D482040002800
:1057A00003DA013860F00700013007284DD8DFE840
:1057B00000F0040B132028303E46136823F47F6367
:1057C00023F00F0319433FE0136823F47F0323F40E
:1057D000704343EA013137E0106820F07F4040EA2F
:1057E000016010608BB3536823F00F0343EA11216B
:1057F0001BE0136823F47F4323F0F00343EA011115
:1058000022E0136823F07F6323F4702343EA01410D
:105810001AE0106820F0704040EA01701060A3B1F7
:10582000536823F0FF0343EA111151600DE0136840
:1058300023F47F2323F4706343EA012104E0136817
:10584000C3F3130343EA01511160002010BD00BFF0
:10585000070000802DE9F04F874B542404FB0134EE
:10586000ADF5057DA56894F82B30266A401BB0FB8A
:10587000F3F563681D44238B03F4C0438B4617463E
:105880003BB106EB15264FF6FF731F3DEDB20293B9
:1058900007E06FF0704C06EBD516CDF808C005F0A8
:1058A0007F05764B204653F82B30314604AA9847A3
:1058B000824618B90390DFF8C89148E06FF0030AF8
:1058C000D4E004A951F82530DDF808C003EA0C0142
:1058D000614549D061688B4246D9022FD4F82080B7
:1058E0007CD0002A00F0A48015F0010F4FEA550586
:1058F000EDB204A900F0948031F8250041F82500AC
:10590000DDF80CC00CF1010CCDF80CC0002A00F041
:10591000938008EB1328DDB2B04518D04FF0000C8F
:1059200094F82A30634500F28C8059F82B302046D9
:1059300004A9324698470130F7D0504B204653F81F
:105940002B30414604AA98470028B7D14646208B01
:1059500010F4C042B5D004A96B0851F82330E90710
:105960004CBF1B0C9BB2AFE7022F7FD09AB115F052
:10597000010F4FEA5505EDB205D004A931F82530E5
:1059800041F825300AE004AA52F825301B0C1B040C
:1059900042F8253002E004AB43F82520410707D543
:1059A000236B039F01333B4440F0020023632083B9
:1059B0000025334F284694F82A30AB420CD9E269CF
:1059C00057F82B3002FB0562204604A99847421C79
:1059D000F5D00135EDB2EEE7824647E0CAB115F0E9
:1059E000010F4FEA5505EDB209D004A830F8252083
:1059F0006FEA02426FEA124240F8252034E004A91F
:105A000051F825206FEA12426FEA024241F8252040
:105A10002AE004AF6FF0704147F8251017460BE0FD
:105A200051F82500010C04A8090440F8251067E787
:105A300004A941F8252063E708EBD31803F07F059C
:105A40006AE7E26959F82B30CDF804C002FB0C621A
:105A5000204604A998470130DDF804C0F1D00CF1CC
:105A6000010C5FFA8CFC5BE7002752E750460DF50E
:105A7000057DBDE8F08F00BF4488FF1F1C88FF1F15
:105A8000008AFF1F37B5BDF818401D19B5F5007F16
:105A90000568C4BFC3F50074A4B28D4207D1416943
:105AA00010461944224604F0D2FB002006E090F88C
:105AB00048500094024C54F82540A04703B030BD34
:105AC0003088FF1F304AF0B5304E314C4FF400356E
:105AD000FF27944615603760DCF800102A4B8903D5
:105AE000FAD52168C9B2FF29F4D14FF400321A6007
:105AF000264AFE2111601A689503FCD5244A2249E2
:105B0000224E13684FF4003500230F4614460D60F3
:105B1000C25C3260D7F800C01B4A1CF4003FF9D0C9
:105B20000133B3F5007FD4F800C0F0D14FF4003357
:105B30001360164BFF21196011460B68124A13F4CB
:105B4000003FFAD0124B19684FF4003111600F4931
:105B5000FF200860194610680B4B8403FBD50A68C8
:105B60004FF400321A60094AFF2111601A6890034D
:105B7000FCD5074B1B6803F01F03052B14BF6FF008
:105B800004000020F0BD00BF2CC0024034C0024021
:105B900038C0024008B5084B08481A8B42F008028A
:105BA0001A83074B32221A6004F0B6FC0548BDE8A0
:105BB000084004F0B1BC00BF4488FF1F70A0010082
:105BC000A488FF1F7FA0010010B50C4C0C4B94F86B
:105BD0004820216853F8223062692046984758B916
:105BE000636993F8FE21552A02D06FF0020010BDC0
:105BF00093F8FF31AA2BF8D110BD00BF4488FF1FD6
:105C00001C88FF1F38B50E4B0E4D4FF400521A6022
:105C10000D4B01221A600446FA214D20022204F0A5
:105C2000F1FE1CB14FF400732B8338BD074804F01C
:105C300073FC4FF480732B83054B1C6038BD00BF91
:105C400004F00F404488FF1FA488FF1F89A00100B3
:105C5000B088FF1F2DE9F74F594D01912B68594C22
:105C6000174644F620629342064605DD564804F086
:105C700053FC6FF001068BE0226812B1062A3CD07B
:105C800085E0524ADFF84891DFF848C115214FF40A
:105C900000384FF0FF0A9346013900F08680C2F8C1
:105CA0000080C9F800A0DBF800008003FBD5DCF819
:105CB0000000C0B2FF28EFD144492268DFF810C1CC
:105CC000DFF810914FF400308846052A0DDC08609B
:105CD00016F802A0CCF800A0D8F800A01AF4003FF3
:105CE000FAD0D9F800A00132EFE722602BB14D20A5
:105CF000002104F055FE00232B6023683349DFF8B0
:105D0000D090DFF8D0C001334FF400384FF0FF0AD5
:105D10008B465A1E1A2A009305DD2B6801332B602F
:105D20000623236043E0C1F80080C9F800A0DBF837
:105D300000209203FBD5DCF80020019802701006C9
:105D400003F10103E5D4009B236007B331781F4AB8
:105D50001F4EDFF880900023492914BF042112212F
:105D600023604FF400304FF0FF0C90468B420DDA69
:105D70001060C6F800C0D8F800A01AF4003FFAD0AE
:105D8000D9F800A007F803A00133EFE7236000264D
:105D90002B6833B14D20002104F002FE084B002295
:105DA0001A6000232360304607E001332B604D204A
:105DB000012104F0F5FD4FF0FF3003B0BDE8F08F96
:105DC0002888FF1FFC89FF1FA2A001002CC00240F1
:105DD00034C0024038C0024037B51D4C23680D4620
:105DE00013F0040101D069B92EE0018B490619496D
:105DF00043F004034FF4005008602360164B58BF73
:105E000052021A60144B58201968FFF73DFC0DF13F
:105E100007010022FFF71EFF104B1860A8B99DF87C
:105E200007304BB92846FFF74DFE28B10C4804F067
:105E300073FB6FF0040008E00A4B4FF400521A6045
:105E4000236823F004032360002003B030BD00BFAB
:105E5000B088FF1F08F00F40B888FF1F3488FF1F6D
:105E6000AFA0010004F00F402DE9F347434C444D2F
:105E70002368164613F0020201D06AB97AE0028B59
:105E80005006404A43F002034FF400501060236074
:105E90003D4B58BF490219603B4F39685120FFF70D
:105EA000F3FB00220DF10701FFF7D4FE421C28602E
:105EB000F3D0002808DA354B4FF400521A602368FB
:105EC00023F00203236056E09DF80730002B49D1F0
:105ED0002F4A304F30494FF400304FF0FF0C9046BE
:105EE0001060C7F800C0D8F800309B03FBD50B68E2
:105EF000DBB2FF2BF4D0FE2B31D12548DFF89480A4
:105F0000254F00234FF4003C4FF0FF098246C0F8B4
:105F100000C0C8F80090DAF800201D499203FAD5B5
:105F20003A68F2540133B3F5007FF0D14FF40033F7
:105F30000B60184BFF221A600B6813F4003F144BE0
:105F4000FAD0154A11684FF4003119601149FF2049
:105F5000086019688803FCD51368002301E06FF01E
:105F600003032B60094B4FF400521A60236823F09F
:105F700002032360286802B0BDE8F087B088FF1FE5
:105F8000AC88FF1F08F00F403C88FF1F04F00F4053
:105F90002CC0024034C0024038C002402DE9F74313
:105FA0005D4C25681F4615F00203164601D06BB9FB
:105FB000ADE0038B5806594B4FF400521A60584B12
:105FC00058BF490245F0020525601960DFF850818D
:105FD000544DD8F800105120FFF756FB0DF1070182
:105FE0000022FFF737FE411C2860F2D0002808DAB3
:105FF0004D4B4FF400521A60236823F002032360D4
:1060000086E09DF80730002B79D14849484D494B2F
:106010004FF400304FF0FF0C88460860C5F800C010
:10602000D8F800209203FBD51A68D2B2FF2AF4D028
:10603000FE2A09D13D4A3E4DDFF8F88000214FF499
:106040000030FF2394460AE03B4804F065FA56E02E
:10605000DCF8009019F4003FFAD0D8F80090B9426B
:1060600004D00131106089B22B60F1E70B46BDF816
:1060700028102E4A2E4DDFF8BC80194489B24FF407
:106080000030FF2794468B420DD2013310609BB243
:106090002F60DCF8009019F4003FFAD0D8F8009097
:1060A00006F8019BEFE72149214EDFF888C040F256
:1060B000FF104FF40035FF2783421C4A09D80133F3
:1060C0000D609BB237600A689203FCD5DCF80020B3
:1060D000F2E74FF400331360154BFF21196011688C
:1060E000124B8E03FBD5134A11684FF4003119602F
:1060F0000F49FF20086019688D03FCD513680A4B0F
:106100004FF400521A60236823F00203236000203A
:1061100003B0BDE8F08300BFB088FF1F08F00F4058
:106120002488FF1FE889FF1F04F00F402CC00240A5
:1061300034C0024038C00240BDA0010000B5174B7A
:10614000ADF5037D19685820FFF79EFA0DF10701A0
:106150000022FFF77FFD124B1860D8B99DF8071099
:1061600071B902A84FF4007204F069F802A8FFF7B1
:10617000A9FC28B10B4804F0CFF96FF0040009E046
:10618000094B4FF400521A60084B1A6822F00402BF
:106190001A6000200DF5037D5DF804FBF089FF1FF8
:1061A000EC89FF1FAFA0010004F00F40B088FF1F73
:1061B0000D4A136810B513F0040401D06CB910E057
:1061C000008B4406094843F004034FF40054046074
:1061D0001360074B58BF49021960BDE81040FFF734
:1061E000ADBF002010BD00BFB088FF1F08F00F40FA
:1061F000F089FF1F10B50B0A8176C3760B0C090ED0
:10620000044603754175C272002104221C3004F05B
:1062100016F8EB22442300206021A075E175227658
:10622000A2746376E374A073E1732274637410BD87
:106230004FF4C07300EB4002B2FBF3F2032330B51E
:10624000B2FBF3F403FB14230A601BB1012B0CBF58
:10625000022301230324B2FBF4F2074D8B60920268
:106260005D43801A04FB005090FBF4F423444B6020
:10627000082390FBF3F030BD00FCFFFF70B54B68C6
:1062800001334B600D46816890F82B20591AB1FB01
:10629000F2F602FB16118AB00446002964D1068B7F
:1062A00006F4005292B2FAB1C2680232934252D05E
:1062B0005AD306A92868FFF7BBFF082186B2226AD5
:1062C00000910699B30011449BB2204604AAFFF73F
:1062D000D9FBE0B9A92E06A804A98CBF002201228F
:1062E000FFF71CFA039027E0760417D5C168023146
:1062F0008B4233D038D32A68016AD3B2022601EB2D
:106300001221009606AA5B00FFF7BCFB10B16FF0EC
:1063100003002AE0BDF8183003930DE02A68016AF3
:1063200002F07F03042601EBD211009603AA9B0022
:10633000FFF7A8FB0028EAD1039B6268934210D9BB
:10634000626A93420DD82B6094F82B10E26803FB2D
:1063500001236B6008E06FF0070006E06FF00800B3
:1063600003E06FF0060000E000200AB070BD0A7A7A
:106370000132D2B20A7210B5048DB2EB541F05D3AC
:1063800000220A72BDE81040FFF778BF002010BD60
:1063900030B5436A90F83E2085B001460BB3144BEC
:1063A000542404FB023401A820310C2203F04FFFD7
:1063B000E525238B029943F0010323832046FFF751
:1063C00073F980B99DF80C3062695B01D15CD554DA
:1063D00021F04003012B04DD204601A9FFF7C7FF90
:1063E000E7E7002001E06FF0030005B030BD00BF1B
:1063F0004488FF1F2DE9F04F89B00D4614460393E2
:10640000029008B1A04800E0A04804F085F82846B2
:1064100004F082F8636ADFF8F8B20BB99C4848E0F0
:106420009C4804F079F89C4804F076F8812194F8AF
:10643000280004F081F8994804F06EF88421606A1D
:1064400004F07AF8964804F067F88421206A04F092
:1064500073F8944804F060F821464FF0540951F85D
:10646000203B93F83A3005A80C2209FB03B903F04E
:10647000EEFE4FF000084646474648460699FFF7AD
:1064800013F9024600287CD19DF81C30D9F814106D
:106490005B01CD1811F803A03FBBBAF1E50F0DD198
:1064A000814804F039F8EA7A02F03F020F2A03D05B
:1064B0007E4804F031F864E016BB12E01AF0400F99
:1064C0000AD00AF0BF0A7A4804F026F8504608219C
:1064D00004F028F8012704E0764804F01DF80126AE
:1064E0000EE095F80D8056460AE0013EF6B256459C
:1064F00005D07148019204F00FF8019A1646012761
:106500006E4804F009F80023E85C0193912104F03F
:1065100013F8019B0133202BF6D1694803F0FCFFEF
:10652000EB7A03F03F030F2B01D066481EE02B7B74
:106530001BB9AB7E0BB9EB7EA3B1634803F0ECFF54
:106540002B7B13B1614803F0E7FFAB7E13B16048CA
:1065500003F0E2FFEB7E13B15E4803F0DDFF5E481F
:1065600003F0DAFF6B7B434502D05C4803F0D4FFB5
:10657000012E06D0484605A9FFF7F9FE07307FF443
:106580007CAF574803F0C8FF8121207F03F0D4FF80
:10659000424803F0C1FF8421A06903F0CDFF4048C9
:1065A00003F0BAFF8421606903F0C6FF3D4803F0A1
:1065B000B3FF2368A16993F83A30542505FB03B56E
:1065C0002846FFF771F80646002840F0CA80277F6A
:1065D0006B693A4803EB471703F09EFFB85D9121C2
:1065E000013603F0A9FF202EF8D13E4803F094FFB6
:1065F000FB7A042B10D005D8012B0BD0022B11D124
:10660000394810E0102B09D0202B09D0082B09D1D4
:10661000364808E0364806E0364804E0364802E0EE
:10662000364800E0364803F077FF364803F074FF41
:1066300000232E21FA5CA2F12000C0B25E2805A83A
:1066400094BFC254C15401330B2BF3D100238DF8F6
:106650001F3003F061FF636A43B12B4803F05CFF16
:10666000039B812193F86C0203F066FF029B002BD1
:1066700050D0264803F050FFA068002103F052FFDD
:10668000E66A246B4DE000BFC8A00100CFA0010066
:10669000DBA00100E5A00100EEA001003EA2010088
:1066A00003A10100EC8401000EA101008F84010010
:1066B0001CA101002FA1010044A1010057A101006C
:1066C0003BAA01005EA1010076A1010011AB01000F
:1066D0008D950100DD7E010090A101009EA10100C9
:1066E000B9A10100D4A10100EBA10100F2A10100B8
:1066F000E1A1010070950100FCA1010006A20100CA
:106700000EA2010012A2010017A2010024A20100A2
:106710004488FF1F039B95F82B40DE68EB6806FB5F
:10672000043411482D6A03F0F7FE8421204603F05B
:1067300003FF0E4803F0F0FE8421304603F0FCFE18
:1067400005EBD6150A4803F0E7FE8421284603F03E
:10675000F3FE084803F0E0FE06F07F00892103F015
:10676000EBFE09B0BDE8F08F35A2010003A10100E6
:106770004AA2010058A201002DE9F04FADF23C4DB4
:106780009046056A90F848A0102204460F4606A8D5
:10679000002110F005FD0AA80021102210F000FDD4
:1067A00018F00C0F07D1238B590703D5676B236BA8
:1067B0009F4200D96768238B9A040DD506A93846F5
:1067C000FFF736FD069B8146EB180AA806A91022A2
:1067D000029303F03CFD0EE05E0407D505EB1725A0
:1067E0005FFA87F902954FF0FF0B06E005EBD7152E
:1067F000029507F07F094FF07F0B02993E46039107
:106800004D46B24A039952F82A300DF1380C6246CF
:10681000CDF800C020469847DDF800C0002840F0C1
:106820006F816346228B90040ED5A92D4FF0010194
:10683000099106A803EB85018CBF00220122019378
:10684000FEF76CFF019B0DE0510409D5022195FB79
:10685000F1F253F82200EA074CBF000C80B201E0CD
:1068600053F82500002840F0378118F0030F11D1AC
:10687000238B13F4005F0DF1380B69D0A92D06A806
:1068800040F6FF710BEB85028CBF00230123FEF75E
:106890007FFF76E094F82B3004930499E36801FBC2
:1068A000063305939C46049B059A1344CCEB0303E3
:1068B00013F0FF03DCD094F82B209A4239D118F062
:1068C000010F36D00DF50E7B00214FF400725846B3
:1068D000CDF800C003F0B3FC20210B22584603F092
:1068E000AEFC2E238BF80030584639461022019317
:1068F000FFF780FC20210B2296A803F0A0FC019B4F
:1069000096A88BF820308BF8213002211022FFF757
:1069100071FCDDF800C06E4A204652F82A30CDF8EE
:1069200000C06246594698470130DDF800C0F2D0F9
:106930000BE06849204651F82A30CDF800C0614686
:1069400098470130DDF800C0F3D00CF1010CAAE744
:106950005B0412D5022295FBF2F215F0010F5BF8F1
:10696000223015BF6FEA03436FEA13436FEA134304
:106970006FEA03434BF8223003E06FF070434BF8AB
:10698000253018F0040F30D0238B03F4005292B25C
:106990006AB1B9F1A90F0AA831460BEB89028CBF85
:1069A00000230123FEF7F4FE4FF000081DE003F47E
:1069B00080439BB2F3B115F001084FF002030AD0F7
:1069C00099FBF3F990465BF829301B0C1B04334309
:1069D0004BF8293009E0A9F1020999FBF3F93BF8DA
:1069E000293043EA06434BF829304FF00009DFF81D
:1069F000E0C017E04BF829609846F6E7E269DDF859
:106A00000CE05CF82A30CDF800C02046594602FB65
:106A100009E298470130DDF800C0EFD009F1010923
:106A20005FFA89F994F82A304B45E7D818F0080F37
:106A300010D1238B5F0747D5626B43F0020323839A
:106A4000236B964228BF721C03F1FF3328BF626399
:106A5000236339E01D4B029953F82A3020465A46E9
:106A6000984700284CD1238B03F4C043A3B1FFB255
:106A700015F0010F4FEA570705D05BF827301B0CC4
:106A80001B04334303E03BF8273043EA06434BF84B
:106A9000273000250E4F12E007F07F074BF82760E4
:106AA000F7E7E269DDF808E057F82A302046594652
:106AB00002FB05E298470130F3D00135EDB294F8BE
:106AC0002A30AB42EDD8B4E730461BE01C88FF1FEC
:106AD000008AFF1F9888FF1F5D4506F1010608DA4E
:106AE000079A01320792099A002A7FF49BAE01357A
:106AF00098E60399013108F0FB080391002580E630
:106B00006FF003000DF23C4DBDE8F08F7FB5038BB5
:106B10000A6803F4C0430D460446016A9BB1D3B230
:106B2000022601EB122100960DF10A025B00FEF72E
:106B3000A9FF10B16FF003002FE0BDF80A300393F6
:106B40004FF6FF730DE002F07F03042601EBD21134
:106B5000009603AA9B00FEF795FF0028EAD16FF08C
:106B60007043039A61688A4201D99A4205D320464C
:106B700029680E22FFF700FE03902A68636A9A4292
:106B800009D8039BE2682B6094F82B1003FB0123C8
:106B90006B60002001E06FF0060004B070BD0000E3
:106BA0002DE9F04F8FB0C2F3C03390E8C0000992D6
:106BB000069391F83A20A64B8B46542101FB0231F3
:106BC0000291044639460BA80C2203F040FB96F9CB
:106BD00000305C2B01D02F2B00D101360023059310
:106BE00004F11E0A2021E66250460B22CDF81CA0BB
:106BF00003F025FB1823002184F82930B1468C4688
:106C00000B4601254FF0050816F8012B50B20D2850
:106C100013D003DCB0B10A280FD016E02F2811D012
:106C20005C280FD02E2810D1002B00F08280082B7A
:106C300066DC01210823B146E6E7002B00F08180E5
:106C40004E4682E0002BF6D0FAE7D0B2202804D8D6
:106C5000002BF0D0202AEED150E07E283AD8DFF881
:106C6000F4A14AFA82F919F8219C19F0210F09D0F0
:106C7000BCF1000F02D019F0200F41D119F0400FE4
:106C80003CD1D8E7BCF1000F3AD119F0040F0CD079
:106C900094F8290021B920F0080084F829002FE099
:106CA00020F0100084F8290041E019F0080F27D0E7
:106CB000A0F12002D2B294F8290029B940F00800CE
:106CC00084F8290003251BE040F0100084F8290017
:106CD00003252CE000F17F095FFA89F9B9F11E0F55
:106CE00003D92030C0B21C28A5D84BB950B21B30F4
:106CF0001FD1012384F81E809C469CE75F22042557
:106D0000072B16DD09B10A2B13DD324612F9013BC0
:106D10000D2B19D003DCBBB10A2B04D114E02F2BAF
:106D200003D05C2B01D01646EFE702250DE0072BC0
:106D3000E9DCDDF81CA04FF0000C0AF80320013359
:106D400079E74FF0FF3500E00425A561013561D0FA
:106D50006663266396F900305C2B01D02F2B00D19F
:106D600001364FF0000902987968FEF79DFC8046D5
:106D7000002847D1029B97F808A05B694FEA4A1A9E
:106D80001D4603935544B9F1000F2FD1059BC3B99C
:106D900004F13803184639460C22089303F057FAD9
:106DA0000398069910F80A3011B9E52B35D1D0E1D6
:106DB0009BB32B7B8BBBAB7E7BBBEB7E6BBB012387
:106DC00064E0059B013B059340F0FE81236D132B8E
:106DD00000F2F5815A1C22650D2202FB0340294670
:106DE0000B2200F5B47003F032FAEDE12846FEF70D
:106DF00085FC94F86C32834240F0DD810120A06173
:106E00008146D9E16FF0030800E296F90030002BCB
:106E100000F0CE806FF00208F8E1EA7A02F03F035A
:106E20000F2B32D0039810F80A1031B9082B0CBF81
:106E30006FF004036FF0010310E0E5290CD1216B22
:106E4000E36A994208D1636B236302235FE000BFCA
:106E50004488FF1FB1A301006FF00203082A00F06D
:106E60007D81226D132A00F27C81511C21650D2148
:106E700001FB024000F5B47029460B22019303F098
:106E8000E6F900210491019B72E10023039A049327
:106E900012F80A3003F0400202F0FF002AB1E52B9D
:106EA00000F0FC80636B012023630D2212F1FF329E
:106EB00080F0FB80002800F0428104F14400089932
:106EC0000C2203F0C4F9002384F86E326B7B84F843
:106ED0006C3294F86E320398226BE16A013384F8C5
:106EE0006E3210F80A3003F03F03012B40F02D8181
:106EF0008A4240F03B81626B2263049A3AB1039864
:106F000010F80A30E52B14BF4FF0FF33012394F83B
:106F10006D2272B1501E0C2202FB00406C3004F155
:106F20006001019303F093F9002284F86D22019B24
:106F30006266DA1C052A00F2478101A151F822F0AD
:106F4000616F00000B6E0000C9710000C971000084
:106F5000C5710000596F00000322A2614FF00109C2
:106F6000A16921F00201012940F02E81039810F857
:106F70000A2012B1E52A1ED024E0636918070BD558
:106F8000BBF83830ABF8362003F00103ABF83830EB
:106F9000DBF8003003B11A70A369002B3FF43AAF5D
:106FA000A38B190704D538460BA90C2203F04FF91F
:106FB0006FF005082AE1069A0AB1DA1C12D0022BFA
:106FC00040F00281B9F1000F0CD1EB7A180700F103
:106FD000FB80284607990B2203F0CDFA002840F0E9
:106FE000F38001E04FF001092B7D6A7D1B0403EB68
:106FF0000263EA7E03EB0223AA7E1344E360CBF82C
:107000000450EA7AD1060CD40298CBF82C3090F8D0
:107010002B10C26801FB0323CBF830304FF002087D
:10702000F4E0A2691AB1A28BD20600F1EF80029AB5
:107030003B6092F82B10D26801FB03237B60022394
:107040003B7296F90030A3B96369022B23D01D0768
:1070500040F1DC800BF1140421460BF108000C22F6
:1070600003F0F5F80BF1200021460C2203F0EFF8B5
:10707000CCE00BA839460C2203F0E9F82660B9F100
:10708000000F01D00423A36104F16C000021FC2255
:1070900003F0D5F8A4E54FF00308B7E0226B636B6B
:1070A0009A423FF4FFAE0020FFE6531E0B2B1FD881
:1070B000DFE803F01C1A18161412100E0C0A08064A
:1070C000AB7F16E02B7F14E02B7E12E0AB7D10E04F
:1070D0002B7D0EE0AB7C0CE02B7C0AE0AB7B08E068
:1070E0006B7A06E0EB7904E06B7902E0EB7800E084
:1070F0006B78591EC9B2FD293FF6D8AE216B01F15C
:10710000FF3CC4F830C011F8011C8B423FF4CEAEF6
:10711000A3F1410C5FFA8CFCBCF1190F02D82033AB
:10712000DBB208E0A3F1610C5FFA8CFCBCF1190F33
:107130001CD82031C9B28B423FF4B8AE16E094F8A7
:107140006C126B7B99420FD1C3E68A420ED30023A7
:10715000DDE6069B04936FF0030309E00020049032
:1071600006E00021049103E0134601E04FF0FF33F5
:10717000626B22630022A264049A42B9591C06D1B0
:10718000039911F80A2002F03F020592BFE61A1D8A
:107190007FF4BDAE94F86D322BB904F1600039462E
:1071A0000C2203F054F894F86D32142B07D80133F5
:1071B00084F86D3208E0C1466FF00203D0E6002388
:1071C000059301E04FF0010902983946FFF7CFF827
:1071D00000283FF4C8ADA369002B3FF41BAEA38B7E
:1071E0001C077FF5E5AE07307FF4DDAE099B58053F
:1071F0007FF5D9AE7B680298013B7B603946FFF78B
:1072000085FC002814BF80466FF0050840460FB08B
:10721000BDE8F08F2DE9F041038B9F048AB004464E
:107220000D46164627D5086806A9FFF701F8236A18
:10723000069A87B202EB0308B6B90822BB00009297
:107240009BB22046414604AAFEF71CFC002862D1EE
:10725000A92F06A804A98CBF00220122FEF75EFA1E
:1072600040F6FF7303903CE020464146FEF71CFACF
:10727000002850D1E1E713F4804F0F68036A19D05A
:1072800003EB172782B92B78022200922046394659
:1072900006AA5B00FEF7F6FB00283CD1BDF81830CB
:1072A00003934FF6FF731CE03946FEF7FDF9002803
:1072B00031D1E8E703EBD71772B92B68042203F04A
:1072C0007F0300922046394603AA9B00FEF7DAFBB3
:1072D00008BB6FF0704304E03946FEF7E5F9D0B91A
:1072E000EBE7039A61688A4201D99A4205D32046A6
:1072F00029680C22FFF740FA03902A68636A9A42D1
:107300000CD8039BE2682B6094F82B1003FB01233D
:107310006B60002004E06FF0030001E06FF00600F6
:107320000AB0BDE8F08100002DE9F0411D4BC76AAD
:1073300090F84880ADF5007D53F8283039466A460C
:1073400004469847064610B16FF0030624E0256B0B
:10735000636B8DF8E8512A0A8DF8E9212A0C8DF823
:10736000EA212D0E1A0A8DF8EB518DF8EC318DF8CB
:10737000ED210D4D1A0C1B0E8DF8EE218DF8EF311D
:1073800055F82830204669463A4698470130F7D0EC
:10739000238B23F00203238330460DF5007DBDE8E7
:1073A000F08100BF1C88FF1F008AFF1F2DE9F04FEE
:1073B000876893B097F8483007925FEAD27905461C
:1073C0000C46089303D1AB69022B2EDD37E008464B
:1073D000FEF7DEFF0028F6D058E240463146FEF7C1
:1073E000C6FFC21D06D17368013B7360404631463B
:1073F000FFF78CFB002840F0498240467168FEF799
:1074000053F9002840F03E82327AD8F814300399BC
:1074100003EB4213059A914280F03E81049921B119
:1074200018460AA9202202F012FF6E6838467168D9
:10743000FEF73AF98246002800F0C08122E2AA460F
:10744000D5F808805AF81E3B6E680593184603F07D
:10745000C1F8059B83460344002150460C22039348
:1074600002F0EDFE2023AB772F2385F8263003F0C2
:1074700017FA009003F014FA009B43EA004000F072
:107480001F300A900028F2D00AA9042205F120003A
:1074900002F0DDFE03F004FA41F61F7303400AA96F
:1074A000022205F124000A9302F0D1FE5046FEF7B5
:1074B00025F90BF1010B0990CDF808B04FF0010A46
:1074C000029B0D2B07DD029B0AF1010A0D3B5FFABF
:1074D0008AFA0293F4E7B9F1000F08D10FFA8AF3A0
:1074E0009A0005EB03139A1A0C2100232FE0636A1C
:1074F000002BF3D094F840305345EFD304F1200B28
:10750000304659460C2202F0A2FE94F84030534512
:1075100058D0CAEB030384F8403094F840303BB1B4
:1075200040463146FEF723FF94F84030013BF2E736
:1075300084F840A0584631460C22009302F087FEA2
:10754000009B40E0013301FB0320406E20B903EBB8
:107550000A0BBBF1140FF5DDB9F1000F02D1CDF824
:1075600010901FE040467168FEF79EF8002840F03A
:107570008981337AD8F814C05B010CEB0301202217
:107580000AA88DE8081002F062FE9DE80810E522C6
:107590000CF80320B8F8183043F00103A8F81830AD
:1075A00001230493BBF1140F04DD304605F15401AF
:1075B0000C2204E00C2202FB0B5130466C3102F02D
:1075C00046FE01E00023049340467168FEF76CF824
:1075D000002840F05781327AD8F814304AF0400A37
:1075E0004FF0FF0B03EB4213CDF818A04FF0FF3222
:1075F000DA4602990D2904D1039991F800A04FF0C1
:10760000000B511C202900F2CA800FF2080E5EF810
:1076100021F000BF99760000DB730000C376000004
:10762000D7760000DF760000E7760000EF760000F6
:10763000F7760000FF760000077700000F77000064
:10764000177700009F7700009F7700009F7700006A
:107650001F770000277700002F77000037770000A2
:107660003F770000477700004F7700005777000012
:107670005F770000677700006F7700007777000082
:107680009F7700009F7700007F77000087770000DA
:107690008F77000097770000184600212022009382
:1076A00002F0CDFD009B069A09991A7002F0BF0204
:1076B000013AD2B206920F22DA72597318461F228B
:1076C00097E780F801A0B8F8182042F00102A8F866
:1076D0001820002264E080F802B0012289E780F8D7
:1076E00003A002225CE080F804B0032281E780F866
:1076F00005A0042254E080F806B0052279E780F85E
:1077000007A006224CE080F808B0072271E780F855
:1077100009A0082244E080F80AB0092269E780F84D
:107720000EA00A223CE080F80FB00E2261E780F83C
:1077300010A00F2234E080F811B0102259E780F831
:1077400012A011222CE080F813B0122251E780F829
:1077500014A0132224E080F815B0142249E780F821
:1077600016A015221CE080F817B0162241E780F819
:1077700018A0172214E080F819B0182239E780F811
:107780001CA019220CE080F81DB01C2231E780F803
:107790001EA01D2204E080F81FB01E2229E7013A36
:1077A00002990D2903D103990139039124E7DDF8EA
:1077B00008E00EF1010ECDF808E01AE77B6996F8B3
:1077C000088003EB4818404605F11E010B2202F029
:1077D0003EFD95F8293088F80C30B9F1000F15D12D
:1077E000384644B931680122FEF7C6FF05462946EE
:1077F0004046102207E049464A46FEF7BDFF0546CF
:10780000294640462022FEF7F5FC00E05546DFF809
:1078100084800899726858F8213079693846984709
:107820000130F6D03B8B23F001033B83B9F1000F0D
:1078300020D104B3216804F1140020310C2202F09D
:1078400006FDE56297F82B20FB6802FB05352563F2
:1078500004F1340004F12C01082202F0F8FC079B2B
:10786000C4F808906360089BC4F80C9084F83E301C
:10787000022400E000243B8B9B0706D53846FFF727
:1078800053FD02E06FF0030000E0204613B0BDE8B6
:10789000F08F00BF008AFF1FF8B507464B69047FD1
:1078A0000D460846B96903EB4414FDF7FDFE064694
:1078B00000BBBB68A0751A0A237762771A0C1B0EEF
:1078C000E3776023E375EB232376A3744423A27745
:1078D0006376E374094C95F84830696954F82330AD
:1078E000BA69284698470130F5D02B8B23F0010365
:1078F0002B8301E06FF003063046F8BD008AFF1FBE
:10790000F8B505460C46164622B92846FEF740FD56
:1079100098B1F8BD03685B686022DA75EB2200213C
:107920001A769A74022E4FF0440219775977997794
:10793000D97799755A76DA74E7D1134F95F83E30B6
:10794000616957F823302268204698470130F5D006
:10795000238B286B23F001032383A368984205D26D
:10796000208B00F0020080B240B9F8BD94F84810B6
:107970003246FDF76FFF0028F2DAF8BD2046BDE879
:10798000F840FFF7D1BC00BF008AFF1F2DE9F04F80
:10799000994DADF5077D0021019028688DF80F10F5
:1079A00010F0020007D09548954B42691B68984734
:1079B000471C00F072872A68D60700F1EA85914ECD
:1079C0003368242B00F2AF80DFE813F02F002F0084
:1079D00025009900B300CE00DD00EC00AD00AD0045
:1079E0000801AD00AD00AD00AD008B019501C201F5
:1079F0008002AD002A03680381049004D504F704D3
:107A00000905AD00AD00AD00AD00280562057C059F
:107A1000D305AD0014037C4A7C48DFF868E20B23F1
:107A20004FF40031FF2417465EE0794A794B7A49DA
:107A30001A607A4A724B1A60794A7A4B1A607A4A0B
:107A40007A4B1A607A4B1A6842F480521A6053F8E3
:107A5000042C42F4006243F8042C4FF410720A60C4
:107A600053F8041C41F4006143F8041C71490A6096
:107A700053F8042C42F4006243F8042C6E4A40F29E
:107A80000321116053F8042C42F4007243F8042CD3
:107A900000204FF400514FF4A0720EF0E7FA674B4C
:107AA00067491A6842F400521A605A6942F4005257
:107AB0005A61644B1A6842F001021A60624A11600E
:107AC000624A1A60013A1A60614B4FF40052022177
:107AD0001A604D20316001229FE2D7F800C01CF4EB
:107AE000003FFAD0DEF800C0013B02D01160046014
:107AF000F3E7584B4FF400521A60032333605648A3
:107B00000DF10F010022FEF7A5F828B1013000F0B9
:107B1000C48600238DF80F309DF80F30012B06D05E
:107B20000020FEF76FF8374C242600F03ABE0423FD
:107B300033604A480DF10F0106AAFEF78BF80028C2
:107B400055D19DF80F30012B09D19DF81B30AA2B80
:107B5000E6D19DF81A30012B1FD0414800E0414882
:107B600002F0DAFC0120DCE73F480DF10F010022B2
:107B7000FEF770F800283AD19DF80F30012B00F283
:107B8000F6850623336039480DF10F010022FEF718
:107B900061F860BB9DF80F3013B1052300F0A2BC63
:107BA0000723336032480DF10F0106AAFEF752F8A1
:107BB000E8B9304802F0B0FC9DF818200F4B02F0F5
:107BC000400202F0FF011AB140221A832A4801E064
:107BD0002A48198302F0A0FC0A23336006AC284827
:107BE0000DF10F012246FEF735F800284CD0013088
:107BF00096D100F052BE00BFB088FF1F4488FF1F1F
:107C00001C88FF1FA488FF1F2CC0024034C0024004
:107C10009D5F00003088FF1F14B00440695E0000C3
:107C2000D95D0000008AFF1FB16100009888FF1F26
:107C30003C80044018B004401CB0044000F00F40E9
:107C40000606003E00C002400CC00240013C3F80DE
:107C500004F00F4008F00F406AA0010064A001008A
:107C600061A2010079A2010015A40100ABA30100EB
:107C70000FA401009EA20100ACA20100BCA2010061
:107C8000A5A3010038C002402278FE2A14BF0222B8
:107C90000122034604EB020E1EF803700821400087
:107CA000C0B287EA000C1CF0800F18BF80F00900FA
:107CB0007F000139FFB2F2D101330F2BECD10F322B
:107CC00000F07F00A35CB0EB530F40F08A85102AD0
:107CD00040F08C850DF11A00611C02F0A3FA00F04F
:107CE00085BDBC4B00221A60FDF76EFF441C00F0FE
:107CF000D48510233360C11C7ED01123336000284B
:107D00007FF40EAFB34A536993F8C2011146E0B154
:107D100093F95200462818D093F93600462814D01B
:107D200093F8C80193F8C911000400EB016093F8BF
:107D3000C71100EB012093F8C61143181360FDF73B
:107D400043FF421C04D100F0A8BD00230B6001E0FA
:107D5000033051D09F494B69DC7D9A7D93F80CA08C
:107D600012EB04244FEA0A2A10D193F8264093F824
:107D70002720240404EB026493F8252004EB02245A
:107D800093F824204FF00109144401E04FF000095A
:107D90001F7DDA7C12EB07270DD193F8227093F840
:107DA000232093F821603F0407EB026793F820201B
:107DB00007EB06271744CC6193F810E0D1F8008058
:107DC00081F82AE0587B834A81F82B0093F80FC092
:107DD0009E7B06EB0C26B6B206EB080CBAF5007FCC
:107DE000C1F820C005D320B10AFB00F1B1F5004F66
:107DF00005DD794802F090FBFDF7CCFE93E60EFB23
:107E000004F4B2F818E0A2F828A02EF0080E1FFA29
:107E10008EFE06EB040A4EF02001CAEB070A11831E
:107E2000BAFBF0FA4FF6F4718A4513D8B9F1000F96
:107E300010D10121516003F1240193F93A30322B22
:107E40000CBF4EF4005E4EF4804E4EF0200EA2F8B1
:107E500018E01CE093F831E093F8301093F82F907D
:107E600001EB0E2193F82EE04FEA0E4E0EEB096E59
:107E700093F82D900EEB092E93F82C9018FA81F1BF
:107E8000CE44D1621160C2F804E003F140015368AE
:107E9000BE1B361B6444B6FBF0F603FB1040138B8D
:107EA000566203F4C0439460D06013B1494B1F3055
:107EB000D86007310B22494802F0C9F9484B122219
:107EC0001A60FDF781FE431C00F0E784414C002856
:107ED0004BD1228B570448D4636993F8FF11AA2928
:107EE00043D193F8FE1155293FD1D97841293CD18E
:107EF0009978612939D15978522936D1197852297E
:107F000033D193F8E71161292FD193F8E611412974
:107F10002BD193F8E511722927D193F8E411722936
:107F200023D193F8EA1193F8EB0193F8EE61090479
:107F300001EB006193F8E90101EB002193F8E801FE
:107F4000014493F8EF012163360406EB006693F8D1
:107F5000ED0106EB002693F8EC01023933188B4251
:107F6000636302D842F0040222831E4802F0D4FA6E
:107F7000238B1D4843F08003238302F0CDFA1B4C72
:107F80004FF0010904F596784FF0030A238FDE07BE
:107F900014D594F83A708FB92668204639463C22A9
:107FA00002F04DF9A4F8389084F83A7036B12660A2
:107FB00030460F4902F004FBA4F836A03C34444597
:107FC000E4D12B6843F001032B60054B13221A60A8
:107FD0001FE000BF4488FF1FC7A201008D88FF1F5C
:107FE000A488FF1FD4A201003BAA0100BC88FF1F88
:107FF000E3A20100C748C84B01681B684269984763
:1080000000287FF48DAD132333602B6843F0010308
:108010002B604D204FF4FA71042202F0F3FC82E54C
:10802000DFF8F082D8F81440D8F8107000214FF42F
:108030000072204602F003F9022384F8BF310C23BA
:1080400084F8C0310B2384F8C231382384F8C3315B
:10805000F82384F8C431B8233F3F84F8C5313F2367
:1080600084F8C6313B0A84F8CB313B0C84F8CC3120
:10807000552384F8FE31AA2384F8FF314046A74BEC
:1080800084F8CA713F0E84F8CD711B6841690022E3
:108090009847002840F07482152333609D4FDFF825
:1080A00090A27C694FF4FE720021204602F0C7F8CE
:1080B000EB232370582363709023A3709849E01C2E
:1080C00002F07EFA4FF400733B85FF210023E37238
:1080D00002223F23A176F821227323766175398B22
:1080E00011F4C04F62D03B69A2741A0A3C20227579
:1080F00001F40052607092B20120E3742074083BD6
:1081000052B140F25518B3FBF8F8B8F1FE0F4FF03A
:108110000603A3730AD815E040F20118B3FBF8F880
:10812000B8F1FE0F4FF00803A3730ED90623E374D2
:10813000FF2323757AB11423E374082323754FF0CA
:108140000C080AE0B8F10C0FF5D8B8F1000F08BF21
:108150004FF0010801E04FF0FE080023E375012312
:1081600084F8168087F82B30552384F8FE31AA2333
:1081700084F8FF3104F136006A49DFF898B108222B
:1081800002F065F83B8BCAF80080980445BF3223A3
:1081900084F83A3008F1080308F10603CBF80830F8
:1081A000BB681F3304F12409FB6059E03869237769
:1081B000A0F13F03190A84F82110190C227484F8E5
:1081C00022102022190EB3F5022FA27384F820305A
:1081D00084F8231001D8012310E0B3F1807F01D887
:1081E00008230BE0B3F1007F01D8102306E0B3F1C0
:1081F000806F02D887F82B2002E0402387F82B30CD
:1082000097F82B10012202EBC111A0F160030B447F
:10821000B3FBF1F3190A84F82510190CCAF80030E1
:1082200084F8243084F82610190E5B005F3384F83C
:10823000271084F830200221062284F82C1084F8BC
:108240003220BB60082204F15200374901F0FFFFE1
:1082500097F82B20BB68A3EB420304F14009FB60B5
:1082600097F82B306373802389F80030292389F82D
:10827000023002F015FB89F8030002F011FB89F8C7
:10828000040002F00DFB89F8050002F009FB89F8F3
:10829000060097F9493033B909F1070023490B2249
:1082A00001F0D5FF11E000232021FA1809EB0300AB
:1082B00092F84920C2712AB909EB030201330B2B52
:1082C000D171F9D101330A2BEFDD16233360114848
:1082D000038B03F4C0433BB9104B41691B683F2239
:1082E0009847002840F04C8117233360DFF8248042
:1082F0000A4BB8F818201B68D8F8141002F4C042D2
:108300004046002A0CBF452200229847074688B104
:10831000471C36E14488FF1F1C88FF1F008AFF1F8F
:10832000E7A20100F0A20100F9A2010002A30100EE
:108330009C88FF1FD8F8144039464FF4007220463D
:1083400001F07DFF08F149010B22204601F07FFF7B
:108350000823E37244236376E3746374A54BA77523
:10836000EB2260211F601823E1752276A274A773A7
:10837000E173227433609F4F9F4C3A6894F82B301E
:108380009A4213D29D49A368D1F800C06169204682
:108390001A44E0470146002835D13B686069013343
:1083A0004FF400723B6001F04AFFE0E119233360B3
:1083B00000233B60924B01221A708F4B1A8B586935
:1083C000510401D58F4902E0930402D58E4904225D
:1083D00001E08E490C2201F03AFF1A2333608649EE
:1083E000844C0B8B226849699F0454BF5F3206227C
:1083F000814F13F4804F814B38461B6818BF082209
:108400009847014608B10131BBE078690C2201F0C0
:1084100016FF2368013323601F23336078487C4CA8
:10842000744B017824681A684C43A2421C4616D348
:10843000012903D801310170192353E06E48018BE3
:10844000CC040AD511F4C04F21F480540CBF5F3224
:1084500008321A600483202344E0212342E0664B63
:10846000198B01F4C04109B95F3200E00832634959
:1084700061480F685969B847002840F08180236837
:10848000013313F0FF0F236040F07181614816E063
:10849000584C5948226803699A4202D32123336019
:1084A00010E0564B41691B689847002868D1236843
:1084B000013313F0FF0F236040F05981564802F05A
:1084C0002BF854E14C4C228B12F4C0420CD0534890
:1084D00002F022F8238B98044CBF5148514802F017
:1084E0001BF80F23336042E1494823690068616942
:1084F00040005F3B1B1A94F82B0081F8ED21B3FB81
:10850000F0F34120013BC87081F8E601722081F848
:10851000E50181F8E401180A81F8E83181F8E90100
:10852000180C1B0E81F8EB31032381F8EC31AA23E0
:1085300081F8FF31552361274FF0520E81F8FE314B
:108540002E4B8F7081F801E081F800E081F8EA019C
:1085500081F8EE2181F8EF2181F8E7711B68204650
:108560004022984760B9238B43F0040323832223DE
:108570003360224B20481B6841694622984730B13E
:10858000013000F08A8132233360FFF7CCBA2648ED
:10859000A5E7D1067FF5C7AA174B2448DF691C6AF7
:1085A00001682744B942814680F0E7807F1ADFF8EE
:1085B00084800A2F28BF0A27002F00F0D880D9F81E
:1085C00000100D4C4B1CC9F80030194B06AE20466C
:1085D00032461B689847002840F0C780238BDFF89D
:1085E00058E013F4804F35D0DEF8003032582ABB03
:1085F000023328E0A088FF1F4488FF1F008AFF1F66
:108600001888FF1F60A001005CA0010099A3010071
:108610009C88FF1FFBA501000EA3010010A3010011
:1086200024A3010028A301002CA301002C88FF1F14
:108630001C88FF1F3888FF1F4088FF1F91B209B1B7
:10864000120C00D101330430B0F5007FCED1CEF84A
:1086500000308AE003F400539BB213B9DEF8001037
:108660007AE0904B1A68236A013AD41A0323B4FBC8
:10867000F3F203FB12441CB1012C0CBF02240124B1
:10868000894ADEF80010D8F80030D2F800C0002285
:108690007F2A59D8012C56F8220013D0022C32D050
:1086A000C0F30B0404B90131012B02D100231C4695
:1086B00034E07E4C044004B90131023BF6D08446DC
:1086C00001243FE000F00F0B0CF07F4A5BEA0A0A3E
:1086D00008BF0131012B20D04FF6F07A00EA0A0AD8
:1086E000BAF1000F00D10131022B16D0DFF8E4A15E
:1086F00000EA0A0ABAF1000F00D10131033B0CD0A5
:10870000844602241EE05FFA80FB0CF0704A5BEAAC
:108710000A0A08BF0131012B03D100234FF4007274
:1087200010E0DFF8B4A100EA0A0ABAF1000F00D1A4
:108730000131022BF1D0000D000500B90131033BDE
:10874000EBD000240132A3E7594ACEF800101360A1
:10875000554BC3F800C008E0F25802B901310433A8
:10876000B3F5007FF8D1CEF80010013F24E74D208B
:10877000042102F015F9FFF7D6B94E494E4C22F00C
:1087800010020A604D4A94F900001268BF211A6372
:1087900001F0DCFE00232370FFF7C5B99DF813300C
:1087A00043B1019B04A9987B052201F051FB0028ED
:1087B000F4D172E09DF81420042AF2D12368132B1F
:1087C00005D12B68266023F001032B6004E04D20C7
:1087D0004FF4FA7102F016F94D20042102F0E0F88E
:1087E000DFE74D20042102F0DBF856E0344F0DF1B5
:1087F0001A01102207F1380001F029FDA378A27AAE
:10880000E17A13F0400F637A07D0120202EB0343C0
:10881000194401318902396118E0207A9B0000F087
:10882000030003EB8023207B03EB921201F0030192
:10883000C009E37900EB41010132023103F00F037B
:108840008A400A2B3A6104BF52003A611D4801F088
:1088500063FE7B692BB94FF4007001F0E9FE184B01
:1088600058610F2304214D20336002F099F8002352
:1088700087F84830144B4FF400521A60134B1A68B3
:1088800042F001021A60124A4FF03E4111601A682C
:1088900022F001021A60FFF746B90DF5077DBDE829
:1088A000F08F00BF2C88FF1F1488FF1F00F0FF000F
:1088B0003888FF1FB088FF1FB488FF1F4088FF1F44
:1088C0004488FF1F3BAA010004F00F4000C0024093
:1088D0000CC002400000FF0F00FF0F002DE9F04127
:1088E000036893F83A70164B0546542404FB07348A
:1088F00020466969FCF7D8FE0646C8B92B7E626936
:108900005B01D018D35CE52B15D10E49DFF8388018
:108910000B2201F09CFC58F8273061696A692046F7
:1089200098470130F7D0238B23F00103238304E021
:108930006FF0030601E06FF009063046BDE8F081F4
:108940004488FF1F3DA30100008AFF1F2DE9F04F5F
:1089500081469FB059F8043B93F83A20A44B4FF05E
:10896000540A0AFB023A00F11003039390F82A30EC
:10897000019300230093019B03F0020780460E46FB
:108980006424FFB25046D8F80810FCF78DFE054667
:10899000002840F0DE8098F80C20DAF8141052011C
:1089A0008B18895C11B1E52906D009E0DB7A1B0739
:1089B00000F1B180012516E1002F00F0AB8002E04C
:1089C000002F40F0A880D87A00F03F0EBEF10F0FC4
:1089D000224654D1002C52D011F0400F13D0E5297B
:1089E00001D1642C0FD1997F0139C9B2FD2905D875
:1089F000621E1EA91144002001F8640C93F80DE0DA
:108A0000CDF800E004E0597BDDF800E0714536D197
:108A10000D2A05DC05A8002101F011FC00242CE042
:108A20001EA9987F1144A2F10D0401F8650C187F6E
:108A300001F8660C187E01F8670C987D01F8680C47
:108A4000187D01F8690C987C01F86A0C187C01F813
:108A50006B0C987B01F86C0C587A01F86D0CD87986
:108A600001F86E0C587901F86F0CD8781EAA01F83D
:108A7000700C22445B7802F8643CE4B24BE082075D
:108A800006D5019901F0200202F0FF0B002A4DD01B
:108A900000F0080202F0FF00002A3CD193F80CE03D
:108AA00006F109020EF0080C02925FFA8CFC195CC8
:108AB000202951D1197A20290AD02E210EF0100E2A
:108AC0001170082001325FFA8EFE195C202958D1FE
:108AD00000211170DA7A32729A7FD97F120402EB88
:108AE0000162597F02EB0122197F0A443260597EEC
:108AF0001A7E02EB0122B280D97D9A7D642C02EBB2
:108B00000122F2804FD04FB91846FCF7F7FD009BC9
:108B1000984203D064244FF0000B07E005A92144DC
:108B2000029801F04DFD64244FF0010B5046494678
:108B3000FDF71DFC073007D1BBF1010F14BF6FF02B
:108B400006056FF00F054EE0BBF1000F3FF41AAFC2
:108B500049E06FF0030546E0052908BFE521BCF1B7
:108B6000000F08D0A1F1410B5FFA8BFBBBF1190F8D
:108B70009CBF2031C9B20130082802F8011B96D1F0
:108B800098E7BEF1000F08D0A1F1410C5FFA8CFC10
:108B9000BCF1190F9CBF2031C9B201300B2802F87B
:108BA000011B92D194E7002FBED07E237372012265
:108BB0003346997A080644BF80399972997A29B95F
:108BC000039849460C2201F042FBADE748B2202849
:108BD000D8BF213102F10102D8BF99720A2A03F1EC
:108BE0000103E6D1ECE728461FB0BDE8F08F00BFD7
:108BF0004488FF1F2DE9F04F00220F684A810C4680
:108C0000097DA7B011F0010F0CBF2C232F23019376
:108C10000DF1310380F82A100546E2810093E189C5
:108C2000A289914280F0518105F1040841460C224D
:108C300002A801F00CFB28460AA9FFF787FE0646AA
:108C400028B110F1100F02D06FF00E003EE1B4F821
:108C50000A90019B0098994401F0BCFC2289484489
:108C6000904207DD404602A90C2201F0F0FA6FF0B5
:108C70000D002BE1BDF82C90217D9DF83020BDF832
:108C80002E80627509F01F0BC9F3431A11F0010F12
:108C90004FEA592909F2BC7907F1010177D0D006D2
:108CA00007D412F0010F0CBF4FF4D2724FF492723E
:108CB00001E040F2ED324FF00B0864204FF02D0E32
:108CC000B8F1010813D0930548BF01F8010C40B278
:108CD00058BF01F801EC722804D077280CBF782027
:108CE000722000E07720520092B20131E8E707F1EC
:108CF0000A00784901F064FC9DF83030DF06024636
:108D00000BD52B68744993F83A30542000FB0313B9
:108D100093F82B10188D484300E00A98414601F063
:108D200085F903462022AAF1020A01301A70BAF12D
:108D30000A0F07D8DFE80AF0080A0C0E1012141602
:108D4000181A1C00654914E0654912E0654910E0F5
:108D500065490EE065490CE065490AE0654908E0AF
:108D6000654906E0654904E0654902E0654900E0BF
:108D7000654901F025FC12210246584601F056F9DA
:108D800010210246484601F051F9074677E0D00726
:108D90004CBF52222D223A709DF8303013F0020F52
:108DA00014BF48222D220A709DF8302012F0040FC3
:108DB00014BF53202D2048704B1C9DF8301011F02B
:108DC000200F14BF41212D215A1C597001325846E1
:108DD000122101F02BF94FF02E0B024680F800B063
:108DE00002210132504601F021F9024680F800B01C
:108DF00000214846013201F019F94FF020090246DE
:108E000080F80090122101324FEAD82001F00EF9CB
:108E10003A23024603700132C8F34510022101F0E3
:108E200005F99DF83030DA0607460AD5237DDB07C1
:108E300003D4364901F0C4FB0746238A0133238259
:108E40001DE00DF1140A52460A98102101F0EEF8C7
:108E5000C0EB0A00113003463A4613F1FF3302D348
:108E600002F8019BF9E73844514601F0A9FB638AF7
:108E70006268013363820A9B13440746636007F10B
:108E8000010920233B704846009901F099FB227D9F
:108E9000C9EB00091107074684F8169006D402466C
:108EA0000D2102F8021B0A21417017462268BA1AE6
:108EB0006281E2890132E281227D120744BF0022F1
:108EC0003A7010367FF4ABAEBEE6002027B0BDE8A6
:108ED000F08F00BF49A301004488FF1F55A3010084
:108EE00059A301005DA3010061A3010065A3010076
:108EF00069A301006DA3010071A3010075A3010026
:108F000079A301007DA3010081A3010085A30100D5
:108F10000F4B70B53C220E46002402FB0435298F0E
:108F200089B901232B8785F83A002EB1F01880B259
:108F300001F07EFB286000E02E60054B3C2000FB2A
:108F40000430868670BD0134052CE6D1002070BD4A
:108F5000BC88FF1F30B5ADF51D7D05460C464FF4AE
:108F60001C720021684601F06AF9684629462246CB
:108F700000F00AF8049B23B1684621460022FDF761
:108F80000FFE0DF51D7D30BD2DE9F843144692F816
:108F90003A308E4A0E46542101FB03230546188BB6
:108FA000020640F1078100226A61002E7BD0E78E25
:108FB00096F900102E2922D196F901102E291ED1E2
:108FC000216829B9268F46F0400626870E4616E00E
:108FD000032F40F2F3800AB1013FBFB211F907C07D
:108FE000BCF15C0F05D196F90210013229B90236A5
:108FF00007E0BCF12F0FEFD1F5E70336D8E7002AE1
:1090000051D0228F032F42F040012187A9833BD901
:109010002368002213F80790DA55238F206823F085
:109020001003238703302146FFF794FF804618B1D1
:10903000236803F80790C1E096F90030BBB1AB8B11
:1090400023F0C00343F08003238730462146FFF717
:1090500081FF18B1A5F81C80804608E0AB8BDB05CA
:1090600005D52068711E384401F0AAFA03E0AB8BE5
:10907000D80503D5E7860520BDE8F883236803F803
:1090800007904046BDE8F883D1050CD5236800223F
:10909000DA700323E38604F1200004F108010C22B6
:1090A00001F0D5F8E7E7218F2E6021F4FC72A98347
:1090B000228736B1327822B152B20A2A01D00D2A63
:1090C00001D1012210E05C2A01D02F2A0DD141F0FC
:1090D0002001A983727822B152B25C2A01D02F2AD2
:1090E00001D1042200E002226A61AA8B12F0020F71
:1090F00004F120062DD15A68D968EA60012A62611C
:1091000093F82B3006D810F4C04F03D01F390B440E
:10911000A36102E002FB0312A261002304F1140721
:10912000237739460C2204F1080001F090F830460C
:1091300039460C2201F08BF8072323876B692068DE
:1091400043F008036B6120B1214901F039FA032390
:10915000E386AB8B13F0E40F1DD05A0603D53046DF
:1091600004F1080112E01F0613D46B6913F0060F17
:10917000304609D004F108010C2201F068F8686952
:10918000042806D1BDE8F88304F114010C2201F093
:109190005EF86E6006E004F11401696030460C224E
:1091A00001F055F86B6913F005000BD101222A611B
:1091B000BDE8F8836FF00100BDE8F8836FF00200AE
:1091C000BDE8F8830020BDE8F88300BF4488FF1F96
:1091D000E3A201002DE9F347002383874368044697
:1091E000884690F83E10D80715464BD5A268E3682C
:1091F000D31A01D1002047E09D4288BF9DB2244B85
:10920000DFF89090542707FB013704F1340A002D52
:10921000F0D0E368C3F308039BB2C3F50076B6B29F
:10922000B54238BF2E4613B9B6F5007F1AD0009666
:109230003846A16B4246FCF725FC80B9A28FE36853
:109240003244A2873A8D3344B3FBF2F1AD1BE360A5
:1092500002FB1133ADB2B044002BD8D10BE06FF05C
:10926000030011E094F83E30A16B59F823303846E2
:1092700042469847E1E738465146FCF7FFFF002891
:10928000C5D001E06FF0080002B0BDE8F08700BF74
:109290004488FF1F1C88FF1F38B50C46096851B170
:1092A000FFF758FE051E09DB2168201D20310C2226
:1092B00000F0CDFF02E06FF0100038BD284638BD49
:1092C000F0B5254B91F83E20542606FB0236ADF54D
:1092D000217D358B05F01005ADB207460C46002DFB
:1092E00031D14B6813F0240F30D029464FF41C7253
:1092F00004A800F0A4FF21680C22203101A800F08E
:10930000A6FF04A839462268FFF73EFE089BFBB182
:109310002A4604A82168FDF743FC851D18D1216861
:10932000069619A820310C2200F091FF206801A9AF
:109330000C22203000F08BFF04A821464FF00042A1
:10934000FEF734F804E06FF0120001E06FF009005E
:109350000DF5217DF0BD00BF4488FF1F38B543687F
:1093600013F00055044608D090F83E20064B5421D7
:1093700001FB0231FEF790FA054620460021442207
:1093800000F05DFF284638BD4488FF1F2DE9F04FEF
:10939000474B90F83E804FF0540B0BFB083B0023EB
:1093A0008387BBF818301546DA06ADF5017D044613
:1093B0000F466ED443689B076ED5DFF8FCA0002DE6
:1093C00059D0E368C3F30806B6B236B9B5F5007FE5
:1093D0000ED2A268D31A9D420AD2364A94F83E3081
:1093E000A16B52F8233058466A46984730B156E090
:1093F000684600214FF4007200F021FFC6F5007CA2
:109400006545CCBF1FFA8CF9A94600A830443946FF
:109410004A4600F01CFF5AF82830A26B58466946AD
:1094200098470130F7D0E368A2684B44934288BF65
:10943000A360E360A38F4E444B44C9EB0505B6F52A
:10944000007F4F44A387ADB2B9DBA26BDBF80830D5
:109450000132A263D21A9BF82B30B2FBF3F103FB6B
:109460001122002AABD1584604F13401FDF7D2FE97
:109470000028A4D017E0A38FA3B16368DE0303D54F
:1094800043F0005363600DE020465946FEF704FAAE
:1094900009E06FF0120006E06FF0090003E06FF0E2
:1094A000030000E028460DF5017DBDE8F08F00BF08
:1094B0004488FF1F1C88FF1F008AFF1F0B8F43F487
:1094C000807370B50B8706460C46CD8EFFF742FDC4
:1094D000031D092B2BD8DFE803F0352A352A082A8B
:1094E0002A05242D0325E5860136236813B396F952
:1094F000002082B1032D02D95C225A5500E001D030
:109500000135ADB220683146284401F059F823688E
:10951000C01AE0860EE0E586022D08BF03255A55E5
:1095200008E00323E38623680022DA7002E06FF08C
:10953000020070BD04F1140004F120010C2200F0BF
:1095400086FE002070BD00002DE9F0472D4B0C4633
:1095500090F83E105426012A06FB01360546C368E2
:1095600005D0022A10D0002A18BF002412E0002CD7
:1095700003DA62429A420CD804E08268D21A94421A
:1095800028BF14461C4405E08268944201D2141B93
:1095900000E000249C4231D005F1340808D2404656
:1095A00005F12C01082200F052FE0023EB6003E0DD
:1095B000AB689C4228BF1C46B6F82890EF68C9F1FA
:1095C000000A0AEA070704EA0A0A574515D2AA6BF5
:1095D000B3680132AA63D21A96F82B30B2FBF3F1CA
:1095E00003FB11234F44002BEFD1304641460122AB
:1095F000FDF710FE0028E8D001E0EC600020BDE897
:10960000F08700BF4488FF1F2DE9F0410C46ADF5FF
:109610001C7D0746154600214FF41C72684600F079
:109620000EFE23681A8F15F0200F14BF42F01C02A3
:1096300042F00C021A87684639462268FFF7A4FCFC
:10964000049B002B00F0AC8015F4804805D0BDF8D9
:109650001C3043F01003ADF81C30684621682A46E0
:10966000FDF79EFA0228064659D1A046264658F82C
:109670002C1B0C22203104F1140000F0E8FD56F8F8
:10968000341B08222C31404600F0E1FD21683046B1
:109690002C31082200F0DBFD22685368D97AC90713
:1096A00048BF25F006056560987FD97F000400EB70
:1096B0000160597F00EB0120197F00264318A36049
:1096C000E66092F83A3011A984F83E3004F12000A7
:1096D0000C2200F0BCFD9DF86E3215F4007184F888
:1096E00040300BD094F83E202F4B542101FB023127
:1096F00020460222FEF704F9A66007E02E0505D5F4
:1097000020460222FFF720FF002849D16D0442D5F0
:109710000120394622466B46FCF76CFE3BE06805AB
:1097200015D5B11D39D121681F4A91F83A3054201E
:1097300000FB0323203168440C22029300F087FDD4
:109740006846214625F00042FDF730FE28E026BBA2
:1097500021680C22203104F1140000F078FD45F05E
:1097600080052368656093F83A3004F1200084F89E
:109770003E3011A90C2200F06AFD9DF86E3284F88B
:109780004030B8F1000F0AD03046394622466B46C9
:10979000FCF730FE01E0022002E0304600E04046E7
:1097A0000DF51C7DBDE8F0814488FF1F30B50A60CF
:1097B00082B10B4C92F83A20542505FB0242128BE1
:1097C000D40602D513F0260F07D11A46BDE8304063
:1097D000FFF71ABF6FF00B0030BD6FF0120030BD05
:1097E0004488FF1F2DE9F0412C4B91F83A2092B0AC
:1097F00012AC542606FB02360B8F44F8441D43F08E
:1098000020030D460B87042221468046FFF7FCFE0D
:1098100048BB04F1140704F12C003946082200F07B
:1098200016FD30460799FBF73FFF58BB9DF82020F7
:10983000736952019B5C43B1E52B26D13046394612
:10984000FCF795FDC31DECD124E02B8F43F03003D2
:1098500004222B8740462146FFF7D6FE0246C8B9B0
:10986000019B5B6807E0022814D1019B5B68DA7AF0
:1098700012F001020CD1E521197020463146FEF7A5
:109880003FF807E06FF0030004E04FF0FF3001E025
:109890006FF0090012B0BDE8F08100BF4488FF1FDF
:1098A000F0B5204B91F83A20542606FB0236ADF570
:1098B0001D7D07460C46684600214FF41C7200F0DF
:1098C000BEFC358B05F01005ADB22DBB238F049582
:1098D00043F008032387684639462246FFF754FBC6
:1098E000049BDBB14FF4806268462146FDF758F9CE
:1098F000821D04D0002808BF6FF011000EE004F1B3
:10990000200115A80C22029600F0A1FC6846294609
:109910002A46FDF74BFD01E06FF012000DF51D7DAD
:10992000F0BD00BF4488FF1FF8B5D30704D4234B14
:1099300053F82030322B3DD1214E542303FB0063DA
:109940001D8B05F01004A4B28CBB1E4F05F0400522
:10995000ADB247F8204012F0040F45F008041C8314
:10996000164C02D045F4804503E0970706D545F430
:10997000005545F008051D83152300E0142344F825
:109980002030140706D5542303FB00631A8B42F4DE
:1099900080521A83542303FB00600B22493000F0ED
:1099A00056FC4D20042100F0FBFF0020F8BD6FF0B5
:1099B0001200F8BD6FF00100F8BD00BFA488FF1FC2
:1099C0004488FF1FB088FF1F8268C3689A4270B541
:1099D000044601D8002070BD43689A073AD590F834
:1099E0003E201F4B057FA169542606FB02363046F8
:1099F000736903EB4515FBF757FE70BBE3681A0A62
:109A0000A3602B776A771A0C1B0EEB776023EB753C
:109A1000EB232B76AB744423AA77A8756B76EB7493
:109A2000104D94F83E30716955F82330A2693046E4
:109A300098470130F5D0338BA06B23F001033383BB
:109A4000B3689842C6D396F848100222BDE8704029
:109A5000FBF700BF6FF0090070BD6FF0030070BD31
:109A60004488FF1F008AFF1F70B5114B1C56E4B9D4
:109A7000104A114E42F82040104A1954542505FB53
:109A800000220421556A46F82050156A0C4A42F813
:109A900020500C4A52F8205045F0100542F8205052
:109AA0004D2000F07DFF204670BD6FF0160070BDA8
:109AB000B488FF1F4088FF1F3888FF1F4488FF1F9E
:109AC0002C88FF1FB088FF1F38B50B465424094966
:109AD00033B904FB00101146BDE83840FBF7E4BD84
:109AE000054D55F8205004FB001011461A46A847B2
:109AF00038BD00BF4488FF1F1C88FF1F2DE9F84FA9
:109B0000DFF84090DFF840B04FF0540808FB00F851
:109B100082460E46174609EB080431465BF82A30A8
:109B200020463A469847411C0546F6D059F8083079
:109B30009F4204D16069228D314600F088FB28469F
:109B4000BDE8F88F4488FF1F008AFF1F024B542294
:109B500002FB0030704700BF4488FF1F0B4670B502
:109B6000014668B9204A214C1088258820EA134014
:109B700080B223EA0006354303432580138031E099
:109B800090F83A201A48542404FB0202128B02F483
:109B900042723AB1154B00221A800B8F03F0010379
:109BA0000B8703E0104A1288134202D16FF00100C4
:109BB00070BD0E4A1088034206D00C8F20EA0300C5
:109BC00004F001040C8710800A8F95070AD4DC0783
:109BD00003D49807EAD5074800E00748FFF7BAF929
:109BE0000028E3DB002070BD2088FF1FA888FF1F2E
:109BF0004488FF1F97A30100178B01002DE9F8434C
:109C0000032B0E4614461D469DF8207043D13FB2EB
:109C1000444A3B0103EB87071368D9199046CD6886
:109C2000002E2FD014B90020BDE8F883B5F81090AD
:109C3000EB8AC9EB03039C42F5DAB9F1000F0ED0B1
:109C4000D8F80030A868DB5931461B69224698478E
:109C5000AB682344AB602B8A23442B825EE00AF07E
:109C6000EFFDD8F80030DB5948469B689847A8605C
:109C70000AF0EEFDD8F80030DB59DB689847002881
:109C8000D1D1DDE7DB59288A5B692E82A968984724
:109C9000AE60BDE8F8830AF0D3FD072D10D0082D83
:109CA00022D0022D37D13FB23B0103EB87071D4B7A
:109CB0001B681F44FB689C68003418BF01242BE01C
:109CC0003FB23B0103EB8707164B1B681F444FF65F
:109CD000FF72BB68013CA4B2944201D09B69F9E7D2
:109CE0001A681C8A326017E03FB23B0103EB87071A
:109CF0000C4B1B68DA19DB5995689B69204698471D
:109D00004FF6FF73013CA4B29C4201D0AD69F9E764
:109D100000242C8200E000240AF09AFD2046BDE8D1
:109D2000F88300BF088AFF1F2DE9F843044628483E
:109D3000217900F0E3F80146002847D100F0DEF871
:109D4000064610B90020BDE8F883471EFFB2214D3A
:109D50003B0103EB87072A6823682046D3511B6821
:109D60009847A9460028EDD10546804623685B68E0
:109D7000984780454FF0200013DA00F059FC002886
:109D8000E0D00DB1A86103E0D9F800203A4490601A
:109D90002289C282227B02B1827708F1010805463E
:109DA000E4E700F045FC0028CCD0D9F80020084BAF
:109DB00017440022F8600260426082606289C282B9
:109DC0007B6023793B743046BDE8F883BDE8F883B7
:109DD000FD9B0000088AFF1F13B50138C4B223B2EF
:109DE000180100EB8303054800680344187C0094C5
:109DF0005C680323A04702B010BD00BF088AFF1FA4
:109E000008B5044B18701423584300F011FC024BA2
:109E1000186008BD048AFF1F088AFF1FFF2837B596
:109E20000D4610D00138C4B223B2190101EB8303EF
:109E3000064909680B441146187C00945C682A4660
:109E40000223A04700E0002003B030BD088AFF1FB6
:109E500013B50138C4B223B2180100EB83030548DF
:109E600000680344187C00945C680423A04702B097
:109E700010BD00BF088AFF1F13B50138C2B213B26C
:109E8000190101EB8303064909680B440021187C82
:109E900000925C680A460523A04702B010BD00BFCF
:109EA000088AFF1F13B50138C4B223B20A4619014C
:109EB00001EB8303054909680B440021187C0094D9
:109EC0005C680623A04702B010BD00BF088AFF1FD0
:109ED00013B50138C4B223B21A0102EB8303064A58
:109EE000126813448AB2187C00945C68002108232D
:109EF000A04702B010BD00BF088AFF1F30B50C4B51
:109F00001D780C4B1B6800221433AA420ED053F864
:109F1000104C844202F1010205D113F8044C8C422A
:109F200001D1D0B230BDD2B21433EEE7002030BD43
:109F3000048AFF1F088AFF1F2DE9F74F824610464B
:109F4000894690469B46FFF7D9FF014608B100209D
:109F50003FE0FFF7D3FF07460028F8D06FF0130368
:109F6000142616FB00361C4B1B681E44BAF8003042
:109F7000A3B1584600F05CFB0446B06070B1BAF87B
:109F800000301846019300F053FB019B0028DED0FF
:109F9000C51820606060A060E560E382BAF8023016
:109FA00093B1584600F044FB0446F06060B1BAF843
:109FB0000250284600F03CFB0028C8D0431920601E
:109FC0006060A060E360E582C6F8048086F81090C7
:109FD000384603B0BDE8F08F088AFF1F07B5052893
:109FE0001ED8DFE800F0111D1D0315191389ADF807
:109FF00004300023ADF8063013680B4A197801A825
:10A000001823FFF799FF0CE0104600F0C1FE08E0AE
:10A010001046FFF789FE04E0104601F053FC00E013
:10A02000002003B05DF804FBD1A200002DE9F0434D
:10A03000CE0604D52023137001F0FB010132CD07B9
:10A0400005D5002803DA2D2313704042013201F0B8
:10A05000020701F0040C2D4B00240A26FFB25FFA20
:10A060008CFC4FF0200810B90A20302526E030255E
:10A0700083420ED9B3FBF6F314B9012BF8D10FB11B
:10A08000157004E0BCF1000FF2D082F800800132BC
:10A09000EEE7B0FBF3F505F13009EDB2002B18BF88
:10A0A000012482F8009003FB15000132B3FBF6F3A4
:10A0B000D9E734B102F8015BB3FBF0F3002BF8D120
:10A0C0008CB911F0040F134602F1010003D00246CF
:10A0D0002020187007E08C0702D502463020187047
:10A0E0003023137001320B0706D513460D2003F8F9
:10A0F000020B0A2050701A4601F0400101F0FF03E4
:10A1000001B913701046BDE8F08300BF00CA9A3B46
:10A11000CB062DE9F04102D52023137001320F0642
:10A1200006D51346302403F8024B782454701A469F
:10A1300001F0400601F0200801F0080C01F00701D1
:10A14000042928BF04214900F6B25FFA88F85FFAB3
:10A150008CFC17460B46013BDBB2FF2B14D09D0055
:10A1600020FA05F505F00F0505F13004392C08D962
:10A17000B8F1000F02D005F1370402E005F15704F1
:10A18000E4B207F8014BE6E75018BCF1000F04D029
:10A190000D2353540A234370023006B90670BDE8FC
:10A1A000F0810246013092F90030202BF9D0013ABB
:10A1B000002012F8013F59B22F290EDDD9B2A1F1CA
:10A1C0003003DBB2092B88BFA1F157034FEA00101F
:10A1D00088BF03F00F031843EBE7704710B5002268
:10A1E000014610F8013BA3F13004E4B2092C04D974
:10A1F000B3B12D2B08BF0122F2E70139002011F87D
:10A20000013FA3F13004E4B2092C06D85BB2303B25
:10A2100003EB400303EBC000F1E712B1404210BD75
:10A22000184610BD534210B51144841819442344F4
:10A2300012F1FF3202D38C5C9C54F9E710BD02444A
:10A240000346934202D003F8011BFAE7704710B5AA
:10A250000023934203D0CC5CC4540133F9E710BD12
:10A260002DE9F843058A4768AA4238BF15460446D7
:10A270000E463DB3C3687A199A42426015D3C7EBC4
:10A2800003081FFA88F80368C8EB05094B444360CC
:10A290000AF0DEFA8EB1394642463046FFF7D7FF64
:10A2A00006EB080021684A4605E00AF0D1FA26B11B
:10A2B000304639462A46FFF7CAFF0AF0C1FA238A18
:10A2C0005B1B23820AF0C4FA2846BDE8F88300002D
:10A2D0002DE9F8431D469DF82030DFF864801F010A
:10A2E00007EB8307D8F800303B44894616469C6844
:10A2F0000AF0A6FA052D0AD0062D0AD0042D16D193
:10A30000204649463246BDE8F843FFF7A9BF258AF3
:10A3100010E0012E03D1D8F800301F44FC6844B18E
:10A320002368258AA36063600023238202E000255E
:10A3300000E025460AF08CFA2846BDE8F88300BF05
:10A34000088AFF1F2DE9F041044615460F460AF022
:10A3500077FA218A628AE38A88182844984202DDC3
:10A360005D1AAD1AADB22A44D4F808806282E26860
:10A3700008EB05069642A66006D3F31A2668A3608A
:10A380009E1BAE1BB6B200E02E460AF061FA4046B4
:10A3900039463246FFF75BFFB54204D02068B91951
:10A3A000AA1BFFF754FF0AF04BFA638AA28AAB425A
:10A3B00006D1238A2B441A4400232282A38202E07E
:10A3C0002A44A2825B1B63820AF042FA2846BDE857
:10A3D000F0810000F8B504460D46002938D1027816
:10A3E00043789A4266D10AF02BFAA178334B34486D
:10A3F0001970FFF783FD33490646087010B90AF05B
:10A4000027FA59E0304B1B68142000FB06362079F0
:10A4100056F80C3C1A8A561D0644D88A864203DD3B
:10A420000D700AF015FA45E006321A8228469A683D
:10A43000511C9960215C1170DA689968914228BFBB
:10A440001A6800F1010028BF9A600628EFD1F8BD14
:10A450001C4B1E7866B9027843789A422CD18778D3
:10A4600017483946FFF74AFD064628B3FFB205E014
:10A47000124A177800221A700AF0EAF96FF01303F3
:10A48000142010FB0636104B1868E3780644032BA3
:10A49000B06804D1C28A038AD01A80B2F8BD2146BE
:10A4A0002A46FFF74FFF0421044678B200F078FAFD
:10A4B0002046F8BD2846F8BD3046F8BD058AFF1F86
:10A4C000D1A200000C8AFF1F088AFF1F30B528B9EF
:10A4D0000846BDE830401146FFF77CBFFF2805D194
:10A4E0000846BDE830401146F7F78CBCBDE8304067
:10A4F000FFF772BC10B503460446E21A14F8010BCC
:10A5000092B20028F9D12AB10846BDE81040194698
:10A51000FFF7DCBF104610BD014B1978FFF7EABF0B
:10A520003782FF1F1FB56A46FFF780FD6846FFF7B9
:10A53000F3FF05B05DF804FB1FB56A46FFF7E8FDC1
:10A540006846FFF7E9FF05B05DF804FB07B5002397
:10A5500070B18DF800308DF801308DF802000123C4
:10A560008DF80410684605218DF80330FFF732FF9F
:10A5700003B05DF804FB30B50023934208D0C45CFF
:10A580000133CD1815F8015CA542F6D0012030BD8D
:10A59000002030BD013810F8013F3BB111F9012B0B
:10A5A0005BB29342F7D008DD0120704791F90000BB
:10A5B000003818BF6FF0000070474FF0FF30704751
:10A5C0000A78034603F8012B11F9012B0AB118464A
:10A5D000F6E770470023C2560AB10133FBE718467D
:10A5E000704700000E4B13B500221A800D4B0E4A27
:10A5F00019600E4B147819601A460378A34202D0F2
:10A6000063B10430F9E74388194411600DF1070381
:10A610005522994202D801F8012BFAE702B010BD89
:10A62000148AFF1F108AFF1F9C82FF1F188AFF1FBA
:10A63000F8B5104A104B11681C880C4414F0030F35
:10A6400017460E4A1CBF24F00304043412681E4649
:10A6500023189A4205460AD92A4620460021FFF7C8
:10A66000EEFD3B68E31A1D4435802046F8BD00200E
:10A67000F8BD00BF108AFF1F148AFF1F188AFF1F32
:10A68000F8B5104A104B05461C8810680444481E53
:10A69000044217461E4602D04B421C400C440B4A53
:10A6A000126863199A420AD92A4620460021FFF708
:10A6B000C6FD3B68E31A1D4435802046F8BD0020E6
:10A6C000F8BD00BF108AFF1F148AFF1F188AFF1FE2
:10A6D000044B1A681346981A13F8011F552980B2C3
:10A6E000F9D07047188AFF1F034B1868034B1B688B
:10A6F000C01A80B2704700BF188AFF1F108AFF1F60
:10A70000044B1868044B1B68C01A044B1B88C01A02
:10A7100080B27047188AFF1F108AFF1F148AFF1F1C
:10A720002DE9F047594F5A4E00233B603360594B97
:10A7300090461A7882460C78002C4DD064B2944230
:10A7400041D10B4693F901405D1AEDB203F10109C5
:10A750000CB14B46F6E7142068430430FFF768FF5E
:10A7600003463060E8434844A14642784AB3514624
:10A7700052B2D1F800E0BEF1000F20D09EF900C027
:10A7800094451AD14A68C3F800E05A600A891A81D0
:10A790000AB10134E4B2B1F80AE08A89A3F80AE008
:10A7A0009A81897BD973BEF1000F00D11AB109F1EA
:10A7B00001095FFA89F9143301E01031D9E701305A
:10A7C000D3E71A600AE04B1C1946013391F90000E7
:10A7D0000028F9D11946AEE7A14625463368002B7B
:10A7E00048D0B9F1000F2FD00C2000FB09F0043045
:10A7F00080B2FFF71DFF264B38601B684FF0000E3C
:10A800004FF0010C4FF6FF7A1A68AAB15A8932B19B
:10A81000524508BFA3F80AE05A89426002E09989CC
:10A8200009B14160012142680AB180F809C009B14B
:10A8300040F80C3B1433E7E70FFA89F94FEA0913A4
:10A8400000EB8900C01A386004EB0800C0B2FFF7C3
:10A85000D7FA7CB13468FF2623685BB123893BB10A
:10A86000032001212246FFF7B9FBA07300B9A673AC
:10A870001434F1E7084809F0D1FF084B00221A60B0
:10A880000AF040FD2846BDE8F08700BF288AFF1F78
:10A890001C8AFF1F9C82FF1F208AFF1F248AFF1F24
:10A8A000064A108840F3000323F4974323F07F0304
:10A8B00083EA500080B21080704700BF208AFF1FDB
:10A8C0001F4B73B51C680025143454F8143CA4F1D4
:10A8D00014069BB314F8053C13F00D0F2CD009F0AF
:10A8E000AFFF34F8083C1BB914F8053CDB071DD456
:10A8F00014F8043C9BB18DF800508DF8015054F8C9
:10A90000142C12788DF803508DF80220002069462F
:10A9100005228DF80430FFF7D9FD04F8045C14F823
:10A92000053C13F00A0308BF04F8053C09F090FF4A
:10A9300054F8103C304698471434C6E702B070BD56
:10A940001C8AFF1F38B50D4B1C68054609F078FFBF
:10A9500004F1140353F8142C72B113F8051C11F010
:10A960000D0F07D092F90020AA4203D009F070FF22
:10A97000012038BD1433EDE7104638BD1C8AFF1F97
:10A98000064B1B681A683AB192F90020824201D145
:10A99000D87B70471433F5E7802070471C8AFF1F6F
:10A9A00038B5154B1C68236823B393F900308342F4
:10A9B0001ED1B1B9114B1D689DB12B688BB19C4262
:10A9C0000DD109F03DFFA3891BB10D4A1268134454
:10A9D0006B600023E373BDE8384009F039BF0C35E4
:10A9E000EBE7480702D5E37B1A0703D4E17338BDD0
:10A9F0001434D8E738BD00BF1C8AFF1F288AFF1F08
:10AA0000248AFF1FF8B5184B1C680D4617464CB337
:10AA1000164B1E6833682BB393F9003083421FD165
:10AA20002368E3B19E4218D109F00AFFF37B23F0BB
:10AA30000203F37327721FB9B58125B9657208E067
:10AA4000002D08BF01250A4B1B681D4401236560CA
:10AA50006372BDE8F84009F0FBBE0C34E0E7F8BDD6
:10AA60001436D7E7F8BD00BF288AFF1F1C8AFF1FD6
:10AA7000248AFF1F124B10B51C68FCB1114B1B68D8
:10AA80001A68CAB192F90020824213D1206880B1BD
:10AA900083420CD109F0D4FE607A20B10A4B64687D
:10AAA0001B68E41A00E0044609F0D2FE06E00C340C
:10AAB000ECE710BD1433E3E7104610BD204610BD8F
:10AAC000288AFF1F1C8AFF1F248AFF1F38B5114BDD
:10AAD0001D68EDB1104B1C682368CBB193F90030B1
:10AAE000834213D12B6883B19C420CD109F0A8FE9C
:10AAF00000232B726B72E37B43F00203E373BDE828
:10AB0000384009F0A5BE0C35ECE738BD1434E3E756
:10AB100038BD00BF288AFF1F1C8AFF1F154A164B2D
:10AB200011681B68013130B5104611600BB30C334E
:10AB3000042453F80C2CE2B113F8031CB9B10568D6
:10AB400053F8081C8D4212D1D17B8D0705D40D0717
:10AB500058BFD47313F8041C117492892AB153F8A6
:10AB6000081C0A4443F8082C01E003F8032C0C33BA
:10AB7000DFE730BD248AFF1F288AFF1F37B590F812
:10AB800033300546B3B1028B8A4213D800248DF8C6
:10AB9000023001238DF803302046DD23694605226B
:10ABA0008DF800408DF801408DF80430FFF78EFCE1
:10ABB00085F8334003B030BD2DE9F04191F83430D1
:10ABC00013F0010C05460C4605D00A8B0B8DD31AE9
:10ABD0000B8300230B8594F830309A0714D0DB07E1
:10ABE00028464CBF112113210AF0C6FDC0B200282F
:10ABF00040F09E8094F8303023F0030343F040038C
:10AC000084F83030BDE8F08103F0200202F0FF0844
:10AC1000002A40F08880268B4EB923F04003284656
:10AC200084F830300AF0C6FD2046314677E0E06A0D
:10AC3000E16810F480600A781BD003F0040000F093
:10AC4000FF0728B123F0040384F83030474611E0B1
:10AC500094F83200824205D094F83180904509D1B1
:10AC6000012E07D043F0040384F830300246012758
:10AC700000E00746BCF1000F33D062698B199A429D
:10AC800004D8521A92B2002A52D000E03246E38B26
:10AC9000284FB6EB530F09D957F82530DB8CB01A83
:10ACA000984203DBB2EB560F88BF520894F830305D
:10ACB00043F0400384F8303028460AF08BFDE36807
:10ACC000626903449342E36024BFA368E36057F8DA
:10ACD00025300646D98C2046FFF750FF2685BDE873
:10ACE000F081284611460AF047FD236801332360AE
:10ACF00094F8303043F0400384F83030C7B9E3684B
:10AD0000626901339342E36024BFA368E360238B4D
:10AD1000013B2383074B53F82530D98C2046BDE8EF
:10AD2000F041FFF72BBF2846BDE8F0410AF042BDD5
:10AD3000BDE8F081388AFF1F38B505463820FFF797
:10AD400077FC044608B9002038BD2846FFF770FCA0
:10AD5000A0600028F7D043192061E0606361E583BB
:10AD6000204638BD10B50C4608310AF05FFD228B35
:10AD7000238DD31A03442383E368181AA368E06081
:10AD8000984202D2E38B1844E0600023238510BD73
:10AD90002DE9F84304460F463F48217AFFF7AEF805
:10ADA0000146054610B1780705D46FE0FFF7A6F815
:10ADB000054600286DD06FF01303142616FB0536E8
:10ADC000364BDFF8E0801B681E44334B17F0020F50
:10ADD000736007D0E08894F80890FFF7ADFF48F85B
:10ADE0002900F06017F0010F2D4F06D0A088FFF763
:10ADF000A3FF237AB06047F82300227A294B58F842
:10AE000022208AB12168D162227A617B53F8222004
:10AE100082F83410227AE18853F82230E27B4A43E8
:10AE2000642192FBF1F2DA84227A1D4B57F822203A
:10AE30002AB3217B82F83310A188227AA77B53F8AA
:10AE400022004F43642297FBF2F78784207AE77B46
:10AE500053F82000794391FBF2F2C284227A53F82E
:10AE600022102268CA62227A617B53F8222082F87B
:10AE70003410217AA27A53F8213083F83220237AD1
:10AE80003374207A21460AF01DFE02E00846BDE830
:10AE9000F8832846BDE8F883DDB00000088AFF1F6C
:10AEA0002C8AFF1F388AFF1F2DE9F0417A4B53F897
:10AEB00021407A4B94F8342053F82150E36A0F462E
:10AEC00002F00201064601F0FF08F1B1E18B258B8B
:10AED000206916074CBF4A080A4615442583DD053C
:10AEE0006369104444BF02F1FF3292B2984228BF16
:10AEF000C1EB0001206128BF2161384621690AF0B9
:10AF0000B9FD238C01332384BBE01A0512D594F8D4
:10AF10003020500704D522F0040284F8302014E0D9
:10AF200094F83210B14205D142F0040284F8302086
:10AF3000BDE8F08113F0800807D094F83180B8EBB9
:10AF40000601D1F1000858EB01089A0625D5132E09
:10AF500012D195F83430DC0703D538462946FFF77F
:10AF600001FF95F8303043F0200385F830306B68EE
:10AF700001336B60BDE8F081112E0ED195F83030B1
:10AF8000980640F1878023F0200385F8303038465A
:10AF90002946BDE8F041FFF70FBE2268D90402F14F
:10AFA0000102226019D52A8BEB8B9A420CD82B69AF
:10AFB0001E702B696A69013393422B6124BFAB6811
:10AFC0002B612B8B01332B8395F8303013F0600FFE
:10AFD00003D138462946FFF7EFFDE28B238BB8F10A
:10AFE000000F3CD19A420BD90133238323691E7091
:10AFF0002369626901339342236124BFA3682361FB
:10B00000E36A13F0600F23D094F83020D2061FD4E7
:10B01000218BA28C91421BD39E060AD595F8303025
:10B0200043F0020385F8303038462946FFF7C4FD67
:10B0300005E038464FF40071EA6A0AF0F9FB94F82B
:10B04000303043F0100384F83030636801336360BC
:10B05000E26A48F2800313409BB1BDE8F081218C85
:10B060009A4201F1010121840BD901332383236921
:10B070001E702369626901339342236124BFA36870
:10B08000236194F8330028B140B20421BDE8F041B7
:10B09000FFF786BCBDE8F0812C8AFF1F388AFF1FAE
:10B0A0000D4B53F8203093F8302041B1910611D563
:10B0B00022F0200283F830201946FFF77DBD42F0D0
:10B0C000200283F8302093F83420D20702D51946A5
:10B0D000FFF748BE704700BF388AFF1F2DE9F843CD
:10B0E000984606460D4614469DF8207009F0A8FBC8
:10B0F000A8F10203082B00F24681DFE813F00900F3
:10B100007C00A3006B001201440144014401EC00E7
:10B11000A04B3FB23A011B6802EB87071F4415F4AE
:10B12000805F14BFFF68BF68002C51D0230605D58F
:10B1300030462146FA6A0AF07BFB49E060050BD5F0
:10B1400021463046FA6A0AF0EBFB0546C5F30021BA
:10B150003046FFF7A5FF17E1E10717D597F8343020
:10B160009A070FD5FA8B1807FB6A48BF5208D90512
:10B1700044BF02F1FF3292B27A84304639690AF054
:10B1800079FC08E030460AF02FFC04E0A30702D562
:10B1900030460AF08DFC600703D530460AF0D4FB38
:10B1A00004E0210702D530460AF014FC14F0100F19
:10B1B000FB6A02D043F4805303E0A20602D523F4D5
:10B1C0008053FB62660644BF05F07F0587F8335065
:10B1D000BD8DD9E03FB23B0103EB87076D4B1B6888
:10B1E0001F4448F28002BB68D96A0A400AB11D8C2C
:10B1F000CAE01D8BC8E03FB23B0103EB8707654BFC
:10B200001B681F44FF683DB9FD8B3B8BED1AA542BF
:10B21000C0F2B980ADB2B7E009F01AFB2946224668
:10B2200007F10800FFF78EF8054609F009FB97F8CB
:10B23000303013F0600F40F0A78030463946FFF7FA
:10B24000BBFCA1E0DFF84C913FB24FEA0718D9F8F8
:10B25000003008EB8708434429469F68224607F1DF
:10B260000800FEF7FDFF97F8343013F0080F05468D
:10B2700048460BD03B8CDC0708D4BA68FB8BF968D6
:10B2800002EB5303994228BF1346FB60FA6A12F09F
:10B29000600F7BD097F83030D90677D53C8BF98C8E
:10B2A0008C4273D823F0100387F8303097060CD502
:10B2B000076847443046F96891F8303043F001039D
:10B2C00081F83030FFF778FC60E030464FF4807151
:10B2D0000AF0AEFA5AE02F4B3FB23A011B6802EB7C
:10B2E0008707012C1F4404D9023CFB68A4B27DB936
:10B2F00002E0BB6865B907E0012C05D91D605D60FF
:10B30000BB681D605D603FE0002543F824503BE0D2
:10B3100003EB84040023E25CEA540133042BFAD1EA
:10B3200031E03FB23B011B4D03EB87071CB12B689B
:10B330001F44FB6820E02A683A44936893F8301071
:10B34000CC0619D521F0100183F83010D168CA6AF3
:10B35000900609D591F8303043F0010381F8303080
:10B360003046FFF729FC04E030464FF480710AF0C4
:10B370005FFA2B681F44BB689A6800251A61DA607F
:10B380001D831D8400E0002509F062FA2846BDE80F
:10B39000F88300BF088AFF1F024B53F82010FFF705
:10B3A0000BBC00BF388AFF1F40B1836993F825208A
:10B3B000501C83F8250003EB42039983704711F07A
:10B3C000010F30B500F1020408D00578134623F8C8
:10B3D000025B407845EA002515801A4611F0020FFD
:10B3E00004F1020008D02578134623F8025B647844
:10B3F00045EA042515801A464B0705D503781380C6
:10B40000417843EA0123138030BD00002DE9F84361
:10B410009946374B089E1B68282404FB09340746CD
:10B42000E38A002B61D1A58AF36822838A4234BF64
:10B4300090468846A84538BF4546A4F816806582E0
:10B440001860B1682B484A6873684FEA054E42F0AD
:10B4500080020EEA0000104318604B68E06883F039
:10B4600040034B608B6883F040038B602946FFF7F5
:10B470009BFF6760E28A638A9A4206D0E3683BB129
:10B480009B6993F82530012B02D9E08ABDE8F88347
:10B490004846314609F0BCFF0028F6D1F36815484C
:10B4A0002F44C5EB0808A58A1F60B16873684A6815
:10B4B0001FFA88F8A84538BF45464FEA054E42F0C6
:10B4C00080020EEA0000104318604B68E06883F0C9
:10B4D00040034B608B6883F040038B602946FFF785
:10B4E00063FF638A2B446382C4E70020BDE8F883CE
:10B4F000488AFF1F0000FF032DE9F04188B01D4678
:10B5000080460E4617469DF8384009F099F9AB1E63
:10B51000042B00F2AE80DFE803F00328781E9B00C6
:10B52000584B24B21B68220102EB84041C4416F41D
:10B53000805F14BFE368A3687C0608D59A6992F817
:10B540002210C80744BF06F07F0682F821609B697D
:10B5500093F8224090E024B2230103EB8404494B8A
:10B560001B681C44A3681C8A86E024B2230103EBF9
:10B570008404444B1B681C44E5685DB903AC404639
:10B58000214609F045FF18B900943046394636E0A7
:10B590002C4671E0AB6993F8224014F001046BD0A3
:10B5A00036B9EC8A2B8AE41ABC4264DBA4B263E0AD
:10B5B00009F04EF931463A462846FEF7C3FE0446E6
:10B5C00009F03EF9AB6993F82230590654D403AE22
:10B5D0004046314609F01CFF00284DD16B68EA68EF
:10B5E000D21AAB6993F8221041F0400183F822107F
:10B5F00092B20096944228BF14466868A1B20A46E7
:10B600004346FFF703FF044636E024B2230103EB71
:10B6100084041C4B1B681C443A46A56831462846E6
:10B62000FEF71EFEAB6993F822305A07044625D573
:10B6300009F006F9AB6993F8222022F0040283F89E
:10B640002220AB69987E09F09BFF0028F9D013E017
:10B650000C4B24B222011B6802EB84041C440FB182
:10B66000E36800E0A3681A6800249A605A601C82AC
:10B6700002E0002400E0344609F0EAF8204608B071
:10B68000BDE8F081088AFF1F2DE9F04F87B007461B
:10B690000DF11600884691461E46F9F787FC0024F6
:10B6A0004FF0010B0178BDF81620521A92B2ADF896
:10B6B000162043780192042B10D0052B20D0022BAA
:10B6C00045D14379BB4205D0D7F1010438BF0024EE
:10B6D000002C3CD001244FF0000B38E0002C36D079
:10B6E000B8F1FF0F02D08378434530D1B9F1FF0F95
:10B6F00002D0C3784B4529D1002E31D0022426E058
:10B700002CB326B3A51ED5F1000C5CEB050C354619
:10B710002B68B3B1BCF1000F11D19A7890F802A058
:10B7200082EA0A0252060AD193F805C01B7943EA5D
:10B730000C23B5F804C09C4509D2AB8007E008355E
:10B74000E6E7BCF1000F02D0286000E00324019B73
:10B750000844002BA6D1BBF1000F0CBF30460020DF
:10B7600007B0BDE8F08F37B5836993F821300546FF
:10B77000BBB1028A8A4214D800248DF8023001231A
:10B780008DF803302046DD23694605228DF804300C
:10B790008DF800408DF80140FEF798FEAB6983F804
:10B7A000214003B030BD0000F8B504468078E7784A
:10B7B00066790B4600F07F010AB2550105EBC20223
:10B7C0000A4D2D681544227920F07F00384342EA63
:10B7D000062209F053FEE3780BB9112303E095F834
:10B7E000233043F0010385F82230F8BD488AFF1F5B
:10B7F00000F07F0138B5104A0BB25C0104EBC303C3
:10B8000014681C4400221346E568FF2009F036FE48
:10B81000002384F82230E38284F825301DB12B8286
:10B820002B68AB606B60A36823B100221A821A6890
:10B830009A605A6038BD00BF488AFF1F70B5022861
:10B84000C0B004460D46164606D11D4B012218789D
:10B850000023FFF719FF31E0684600214FF48072A2
:10B86000FEF7EDFC14B1012C11D026E0144B294653
:10B870001878FF226B46FFF707FF083400AB23441C
:10B8800053F8083CCBB19878FFF7B2FFF5E70C4BC3
:10B890002946187832466B46FFF7F6FE08B10024B9
:10B8A00001E020460AE0083400AB234453F8080CBA
:10B8B00018B10021FFF778FFF5E7002040B070BD18
:10B8C000468AFF1F2DE9F04105462B4FA97B2B4AE5
:10B8D0003C6804301C23FEF72FFBAE7B80466EB124
:10B8E00036B2730103EBC6063444AB89A3826B897D
:10B8F000DE0614D5202384F8233010E06B7C28204A
:10B9000001335843FEF794FE08238382AB7C3860F2
:10B91000044680F820302946304609F071FE6FF069
:10B920001303142212FB0832154B1B681A44D36808
:10B93000E36013B19C612B892382AB7BA376AB7B45
:10B940006BB1EB7B5BB119B24C0104EBC1013C68FC
:10B950000C44A376AB7B84F82430AB89A382936834
:10B96000A3601BB19C61AB7C84F820302B684046FF
:10B970002360BDE8F08100BF488AFF1FF9B40000D2
:10B98000088AFF1FF8B51546194A0E461168282285
:10B9900050430C180F5817B9A06838B9F8BD304695
:10B9A00029461A46B847072820D1F5E794F8200021
:10B9B00018B140B20421FEF7F3FF94F82220A368E7
:10B9C00002F0040101F0FF0779B9D88A198A411AF7
:10B9D000A94206DB184631462A46FEF7B3FC384634
:10B9E000F8BD42F0040284F822200120F8BD00BF17
:10B9F000488AFF1FF0B5C1B00E464FF48072002197
:10BA000005466846FEF71BFC3046FF2100226B46C8
:10BA1000FFF73AFE40B3164F00245DF8040020B350
:10BA200055B91EB98078FFF7E3FE1BE000AB234455
:10BA30009988FFF7B9FE15E0837803F07F035A0178
:10BA400002EBC3033A681344012D93F822200BBF85
:10BA500022F0010222F0020242F0020242F0010250
:10BA600083F822200834D8E7012041B0F0BD00BFA0
:10BA7000488AFF1F2DE9F043944687B00D461E46C5
:10BA800006282AD8DFE810F009014E024902070013
:10BA90005502630269029F4B1B68282707FB0C377E
:10BAA000FC8AFD681CBBC5B12C8AC4B16A68EB680E
:10BAB0009A4202D3E98A521A6A606868191A89B2EE
:10BAC000A14228BF214600960A466346FFF79EFC26
:10BAD000AB692846198AFFF746FE002446E2AB69A7
:10BAE00093F8222022F0400283F822203EE27B8A53
:10BAF000A342C0F09780002D75D02A8A002A72D008
:10BB0000AB6993F82500998B012800F1FF30C8BF7D
:10BB1000B3F81EE083F82500C1EB020189B2AA69DF
:10BB2000C8BFA3F81CE0298292F825306FF0010EFF
:10BB3000581C02EB430800230EFB00F09E46023B1C
:10BB4000834207D008EB0309B9F81C90CE441FFAD2
:10BB50008EFEF4E7714530D10029B9D197F8223033
:10BB600013F0300F15D0BB8AB4FBF3F003FB104386
:10BB70009BB273B9B3687068596841F0880101607D
:10BB8000596881F040015960996881F040019960DD
:10BB900001216B681C44EB686C609C4202D3EB8A09
:10BBA000E41A6C600023FB82002991D192F82230C4
:10BBB00023F0400382F822308AE76B681C44EB686C
:10BBC0006C609C4202D3EA8AA41A6C6068681B1AF3
:10BBD000CEEB010E99B28E454FF00003B8BF1FFAAD
:10BBE0008EF1FB826FE7BB8AB4FBF3F203FB1243D7
:10BBF0009BB2A3B93B8BA34203D197F8223098069E
:10BC00000DD5B36871685A6842F088020A605A68B4
:10BC100082F040025A609A6882F040029A600024E2
:10BC2000FC82A3E1E41ABA8AA4B2944228BF144663
:10BC3000A5B1AB6993F82520998B012AC8BFD88B91
:10BC400002F1FF3283F82520C8BF98832B8A5B1A44
:10BC50002B82AB692846198AFFF785FD798A7A68B5
:10BC6000F3680A441A60B36871685A6842F0800049
:10BC7000294A2604324002430A605A6882F0400290
:10BC80005A609A6882F040029A6021462846FFF77F
:10BC90008BFB7B8A1C447C821FE70C781D4B24F0B5
:10BCA00080041F684FF00008012CA7F81680994601
:10BCB00000F08E80022C00F0E680002C40F0DA804C
:10BCC0004B78092B7CD8DFE803F0767B7B7B7B43CA
:10BCD000057B72468B78C87891F8078043EA00208C
:10BCE0008B7943EA082800F47F43B3F5007F17D02F
:10BCF00006D8B3F5807F25D104A8F9F751F912E0F1
:10BD0000B3F5407F17D0B3F5C06F1BD10096034841
:10BD10000A210BE0488AFF1F0000FF031BA401005B
:10BD200004A8F9F743F9BDF8101000964246002325
:10BD3000FFF76CFB1AE1C0B204A9F9F73DF900283E
:10BD4000F1D112E13B68002B00F00F81681C3CE050
:10BD50008B78B37429E08978864E00203170FFF724
:10BD600049FE044610B100233370FEE0D9F80030DC
:10BD700093F82060CEB1A91C01220DF11600FEF748
:10BD800066FA75238DF8133002238DF8143020469F
:10BD9000FE2304A907228DF810408DF811408DF87C
:10BDA00012608DF81530FEF791FB0324DEE000965B
:10BDB0007048012102E07048009602210A46B6E769
:10BDC0003B68002B00F0D1800846318A002257E002
:10BDD00091F80190B9F10A0F01F1020021D0B9F1F7
:10BDE0000B0F03D0B9F1000F44D135E0614B1B7844
:10BDF000002B00F0BA80032104AAFFF7E0FA9DF8B7
:10BE00001210FF224046FFF719FD20469DF8121040
:10BE10009DF81020FFF712FD00280CBF0324042416
:10BE2000A4E0544B1B78002B00F09F80022104AA51
:10BE3000FFF7C5FA02209DF810104246FFF7FEFCFE
:10BE4000002800F0928021462246009603304346A7
:10BE5000FFF7DCFA444689E0464B1B78002B00F0E4
:10BE600084800221009645480A464B46FFF7CEFAE9
:10BE70004C467BE03B68002B77D0318A284642460F
:10BE80009847044672E091F80180B8F1010F3ED85E
:10BE9000881C04AA2146FFF792FA364BBDF8100021
:10BEA0001B780BB9002860D1282300F01F0203FB88
:10BEB0000272B8F1010F92F8223017D119077FF5FD
:10BEC0000CAE23F0080382F822303B68002B3FF4CD
:10BED00004AE06ACC0B204F8090D09F055FAD9F861
:10BEE000003020461B6800210422C9E703F0080245
:10BEF00002F0FF03009622B1022121480A460023E6
:10BF000002E002211D480A46FFF780FAE5E53B689A
:10BF10005BB3084603220821B2E71A8A12B96046C9
:10BF2000022303E0328A604629460123FFF72AFDF7
:10BF3000A7E79B7C33B1134B1B68CC2193F92000FE
:10BF4000FEF704FB00200146FFF754FDC5E50D4B4D
:10BF50001B68CB2193F9200004E00A4B1B6893F97E
:10BF60002000CA21FEF7F2FAB7E50424204607B004
:10BF7000BDE8F083468AFF1F448AFF1F28A4010002
:10BF800026A40100488AFF1F054B1B68282202FBDC
:10BF9000003090F82230194380F82210704700BF1B
:10BFA000488AFF1F034B1B68282202FB003090F8D1
:10BFB00024007047488AFF1F2DE9F0410546012003
:10BFC0000F46164609F007FF044638B909F003FF8B
:10BFD000002808BF412080F00304E4B22B0404D5FC
:10BFE00064F07F04E4B284F00304C5F30E0120463C
:10BFF0003A463346BDE8F04109F032BF70B5154608
:10C000000204044649BFC0F30E0401200020A4B27C
:10C010000E4609F0E0FE30B1214632462B46BDE81F
:10C02000704009F002BF4FF0FF3070BD022810B51C
:10C0300004D003280DD0012816D10BE0002009F010
:10C04000CAFE88B1002160F07F00C0B20A460B46EC
:10C0500006E0002009F0BFFE30B1002201211346A6
:10C06000BDE8104009F0FCBE4FF0FF3010BD402885
:10C0700001DC303803E06028D4BF37383D3840B2A7
:10C08000C0B2704708B590F90000FFF7F0FF1B2819
:10C0900028BF1B20000300F5103008BD13B5042293
:10C0A00001A9044609F092FE019B53B1591C0BD023
:10C0B000C4F57F3000F2FB30984238BF0190019800
:10C0C00003E04FF4805000E0002002B010BD0000FB
:10C0D000F8B50D461646074650B1FFF7DFFF0430AE
:10C0E00020F47F6323F00F0303F580543C4401E008
:10C0F0004FF410340A4FBC4202D900202860F8BD2A
:10C100002046FFF7CBFF286030B1201D31460122C9
:10C1100009F05CFE2046F8BD04F58054EBE700BF53
:10C12000FEFF030008B509F0E5FD003818BF6FF009
:10C13000000008BD2DE9F74F884614464A4E002AF4
:10C1400000F08C803568DFF8309185BB471DFF21FA
:10C1500008224648C9F80070FEF771F8284601A980
:10C160000DF10302FFF7B4FF0546002853D00199F3
:10C1700001F58051043121F47F6121F00F01AF42BC
:10C18000019109D36B189F4206D22846FFF7CAFFD8
:10C19000019BA3423FD21F44284601A90DF103028F
:10C1A000FFF796FF0546B0B3B842E0D933E0D9F8BF
:10C1B00000302B44A3F5103BCBF30F370BF1FF3BC3
:10C1C0009344CBF30F3BBBF11B0F05D91B2F47D873
:10C1D000C3F580244FF01B0B4FF0000A07EB0A0554
:10C1E000ADB25D4517D02D03214B05F514359D42A9
:10C1F00011D82846FFF752FF014648B11C4B2A18B8
:10C200009A4288BFC5F5802128460431FFF78AFF8E
:10C210000AF1010AE2E73368134F022B0FD8C3F18A
:10C2200003051448AC4238BF2546184441462A4607
:10C23000FEF70DF83B682B443B60A844641B14B91F
:10C24000B8F1000F0AD13368D9F80000224618442B
:10C25000414609F069FD33681C443460306800E0F1
:10C26000284603B0BDE8F08F4C8AFF1F548AFF1F99
:10C27000FFFF0300598AFF1F508AFF1F2DE9F0417D
:10C2800006460D4617469846FFF708FF044650B18C
:10C29000441B08D0444528BF4446681D30443946F5
:10C2A000224609F093FD2046BDE8F08173B5124A9D
:10C2B0001368064601930024D3B10B780F4D146028
:10C2C000214622462B7109F02FFD01A904222846A0
:10C2D000FDF7BDFF29460822304609F025FD30460E
:10C2E0002146224609F020FD00B10194019800E0AA
:10C2F000184602B070BD00BF4C8AFF1F548AFF1F52
:10C3000000234FF41432824204D80133DBB202F529
:10C310008052F8E7092B01D8303303E0232B94BF78
:10C3200037333D33D8B240B2704709F013B800003C
:10C330000C4B70B5002203F13C0513F9064C991F14
:10C3400054B133F8044C844206D822B15688A64230
:10C3500088BF0A4600E00A460633AB42EDD11046DC
:10C3600070BD00BF648AFF1F10B5094B03F13C028A
:10C3700093420CD013F9064C3CB19C1FA04204D050
:10C3800033F8044C641A23F8044C0633F0E710BD6C
:10C39000648AFF1F38B51B4B044603F13C029342ED
:10C3A00007D013F9061C11B1991F8C420AD106332C
:10C3B000F5E7012270206188FEF724FB6288124BAA
:10C3C0001A8038BD08F03CFA7020FEF753FB6388F2
:10C3D0000D4D98420ED92988081A81B211B1204614
:10C3E000FFF7C2FF702061880122FEF70BFB638814
:10C3F0002B8003E02A881344181A6080BDE8384077
:10C4000008F026BA648AFF1F5C8AFF1F2DE9F043FB
:10C41000877B87B0384600A90522FDF719FD002863
:10C4200041D09DF80350002DF4D1DFF880808DF8C5
:10C4300008508DF809508DF80B504FF6FF76A9463D
:10C440003046FFF775FF0446B8B1B8F8003066888B
:10C45000B34203D2ADF8123004AD0FE023788DF86B
:10C460000A30237900208DF80C3002A984F800905E
:10C470000522FEF72BF82546E2E725B1698811B1C0
:10C480002846FFF771FF4FF6FF70FFF751FF044694
:10C490000028BFD0012270206188FEF7B3FA6288BD
:10C4A000024B1A80B6E707B0BDE8F0835C8AFF1F35
:10C4B00070B5154E0546A6F13C03B342A3F1060044
:10C4C0000AD013F8024C944203D113F9064CAC4243
:10C4D00001D00633F1E708B90C4C05E041800DE0CE
:10C4E000063414F90C0C20B1B442A4F10603F7D1C0
:10C4F00070BD3BB11D7059801A711846BDE870407F
:10C50000FFF748BF70BD00BFA08AFF1F648AFF1FEE
:10C5100010B513680C68A3420CD852684968E31A36
:10C520008A42036002D88A1A426010BD13B1013BEF
:10C53000036010BD00230360436010BD38B5144D87
:10C54000044608F07DF92B6823600023636008F03F
:10C550007FF92B68236008F073F908F079F92168F6
:10C560000C4B0B4423600C4B1A6863681344002B7C
:10C57000636004DD094A0A442260013B04E003D001
:10C58000074A0A44226001335B42636038BD00BF42
:10C59000A08AFF1F807EAA83B88AFF1F817EAA839C
:10C5A0007F7EAA83F8B50668446805468421304634
:10C5B000FDF7C2FF2948FDF7AFFF68688421FDF74A
:10C5C000BBFF274B27493344B3FBF1F001FB10338A
:10C5D0004FF46161B3FBF1F601FB16333C21B3FB71
:10C5E000F1F501FB15371021FDF79CFF1B48FDF706
:10C5F00093FF00213046FDF795FF1848FDF78CFFAB
:10C6000002212846FDF78EFF1448FDF785FF3846C6
:10C610000221FDF787FF1448FDF77EFF41F2C603B4
:10C62000B4FBF3F40CB9114807E0114B9C4203D85A
:10C630002546104E0A2704E00F48BDE8F840FDF7F4
:10C640006BBFB54204D80D48FDF766FF7D43F8E7A0
:10C6500020460821BDE8F840FDF764BF4E85010083
:10C660008064DB3180510100F1AA010058A401006F
:10C670003F420F009F86010061A4010011AB010041
:10C680006120B721FDF762BFF0B57A4D2B68588C59
:10C6900091B04604169C40F1EA80012940F0E78001
:10C6A000010407D563788BB9734B744A1B78012159
:10C6B000D154DCE07049097803EB81005530114614
:10C6C0000422FDF758FF0028ECD0D0E0237803F0D7
:10C6D000C003C02B00F0CB8004F128006849082279
:10C6E000FDF749FF002800F0C280237803F007031C
:10C6F000043B012B00F2BB800023019302930393C0
:10C70000049394F829E02B6894F82870B3F9223048
:10C7100094F82B6094F82A0094F82C2094F82D10AB
:10C720004FEA0E4E4EEA0767002B47EA060694F8DA
:10C730002F3046EA00200ADA090441EA0262134374
:10C7400094F82E20059043EA0223069367E009043B
:10C7500041EA0262134394F82E20079043EA022331
:10C76000089394F8213094F820201B0443EA0263D4
:10C7700094F82320134394F8222043EA02230993D8
:10C7800094F8253094F824201B0443EA026394F8BB
:10C790002720134394F8262005A843EA02230A938E
:10C7A000FFF7CCFE3748FDF7B7FE09A8FFF7FAFE02
:10C7B0003548FDF7B1FE07A8FFF7F4FE3348FDF753
:10C7C000ABFE05A8FFF7EEFE03A805A9304AFFF768
:10C7D0009FFE01A807A909AAFFF79AFE03A8014630
:10C7E00001AAFFF795FE0399049A4B08B1EB430F9A
:10C7F0004FEA520218BF02F100420799049219440D
:10C800000393049A089B05919A1824BF013105915E
:10C8100006926B204BF620710322FFF749FE2B682E
:10C82000059993F854201B4B1B480B4402F03F0121
:10C8300012064156194A4FF4617000FB013348BF9C
:10C8400003F561630F93069B1360154B01221A6079
:10C850000BA821238DF8383009F074FB1148FDF73F
:10C860005BFE05A8FFF79EFE0F4B03221A60002017
:10C8700011B0F0BDEC82FF1FC48AFF1FA78AFF1F03
:10C88000C8A401006AA4010078A4010084A40100E6
:10C89000B08AFF1F8081557C36A40100B88AFF1F33
:10C8A000C08AFF1F92A40100BC8AFF1F5F4B1A6859
:10C8B0002DE9F041528C02F44042B2F5804F90B025
:10C8C00004461F4640F0AD8002A8002138220AF03D
:10C8D00067FC574B5CB11A680132042A1A6007DD05
:10C8E000544B02221A606B2043F6982193E01C609F
:10C8F0000426514DDFF8588154B12B780133DBB257
:10C90000032B88BF0023013E2B7000F0878000249A
:10C910002A783B68494903EB820055300422FDF731
:10C920002AFE0028E9D02B7818F80330002BE4D138
:10C93000DB238DF810300A238DF81230FA238DF89E
:10C94000133001238DF819303D4D8DF81840032325
:10C950008DF81A30FE238DF81B302B68394C8DF87A
:10C9600023301A0E8DF820201A0C8DF821201A0A77
:10C970006B688DF822201A0E8DF824201A0C8DF881
:10C98000252020461A0A8DF826208DF82730FFF73B
:10C99000D5FD23681A0E8DF838201A0C8DF8392031
:10C9A0008DF83B301A0A63688DF83A201A0E8DF81C
:10C9B0003C201A0C8DF83D208DF83F301A0A224B8E
:10C9C0008DF83E2093F900001B4B1978174B1B681C
:10C9D0006B2703EB810130238DE8880055317B22E2
:10C9E00002AB07F0A3FA002808DD22682B689A4200
:10C9F00004D9284621460822FDF729FC1348FDF7F3
:10CA00008BFD1048FFF7CEFD0A4B01221A606B2008
:10CA100040F2EE210322FFF74BFD02E04FF0FF3022
:10CA200000E0002010B0BDE8F08100BFEC82FF1FE5
:10CA3000AC8AFF1FBC8AFF1FC48AFF1F24AB010002
:10CA40003882FF1FB08AFF1F4182FF1F9FA4010091
:10CA5000A78AFF1FF8B5404B1A6804460D4622B15D
:10CA60003E4952420A6000221A603D4B1A68013268
:10CA70001A603C4B1A780132D2B23B2A1A701E4619
:10CA80004AD9394B1A780132D2B23B2A1A701F4662
:10CA900036D9364B1A780132D2B2172A1A7023D9F6
:10CAA00000221A70324A3348117803780131C9B232
:10CAB00011700133DBB2062B01D9073BFAE71D29C0
:10CAC000037007D12C490B78022B03D1012313707B
:10CAD00003230B702B0707D5E3682BB107F0B0FEDB
:10CAE000E368984707F0B4FEA80607D563692BB141
:10CAF00007F0A6FE6369984707F0AAFE00233B7083
:10CB0000A90707D563682BB107F09AFE63689847B9
:10CB100007F09EFE00233370EA0507D5A3682BB10A
:10CB200007F08EFEA368984707F092FEAB0507D585
:10CB300023682BB107F084FE2368984707F088FE2E
:10CB400023693BB107F07CFE23699847BDE8F840B4
:10CB500007F07EBEF8BD00BFC08AFF1FB88AFF1F66
:10CB6000A08AFF1FA48AFF1FA68AFF1FA58AFF1F96
:10CB70004682FF1F4082FF1F4282FF1F0D4B1B7822
:10CB8000C3720D4B1B8883800C4B1B7883710C4B3D
:10CB90001B78C3710B4B1B7803720B4B1B784372D2
:10CBA0000A4B1B7883720A4B1B6803618023037353
:10CBB000704700BFA48AFF1F4482FF1F4282FF1FED
:10CBC0004682FF1F4082FF1FA58AFF1FA68AFF1F04
:10CBD000A08AFF1F2DE9F04708B94C4B19604C4D56
:10CBE0004C4E0A4640F2B374042304F1FF3C1FFA92
:10CBF0008CFC1CF0030F0ED1B24210D9A2F1F172DD
:10CC0000A2F505420233DBB2062B02D80134A4B2EE
:10CC1000EBE7073BF7E7AA420AD8002500E0012529
:10CC20000024DFF81481DFF8F090DFF810A10CE0A9
:10CC300002F17E4202F5F61202F548620133DBB2E0
:10CC4000062BE3D9073BFAE702246DB1012C0BD187
:10CC5000524519D9A2F51812A2F56E521D33DBB256
:10CC6000062BF1D9073BFAE718F8046009FB06F731
:10CC7000BA4209D9D21B3344DBB2062B01D9073B98
:10CC8000FAE70134E4B2E0E70134234DE4B20127CE
:10CC9000AA420BD9A2F5A8320137A2F5C072FFB2A1
:10CCA0000133DBB2062BF3D9073BFAE7002540F648
:10CCB0000F66B24204D90135A2F56162EDB2F8E720
:10CCC00000263B2A03D901363C3AF6B2F9E7D2B244
:10CCD00050B18471C7710372C27286724572A0F836
:10CCE00004C00161BDE8F0870C490C700C490F705D
:10CCF0000C490B700C4B1A700C4B1E700C4B1D70BA
:10CD00000C4BA3F800C0BDE8F08700BFA08AFF1F4E
:10CD10008033E1010085E201805101004282FF1F62
:10CD20004682FF1F4082FF1FA48AFF1FA68AFF1FA3
:10CD3000A58AFF1F4482FF1F2AA40100803B260012
:10CD40002DE9F04387B005460C4601A800211422C6
:10CD50000AF026FA042D0FD10B238DF8103074B190
:10CD600001A809F0EFF8059B4BB920467849FDF77B
:10CD700027FC001BC0B2E7E001A8FFF7FFFE15F09B
:10CD8000070641D0002C3BD015F0060718D0002133
:10CD900022469DF80B00FDF749F92E260246067043
:10CDA000022101329DF80A00FDF740F902460021F8
:10CDB00002F8016BBDF80800FDF738F9024600E003
:10CDC000224615F0050F1CD017B120231370013235
:10CDD00002219DF80D00FDF729F93A25024605705C
:10CDE000022101329DF80E00FDF720F902460221D2
:10CDF00002F8015B9DF80F00FDF718F9024600E00C
:10CE00002246141BE0B29FE0002C00F09080102D11
:10CE100040F2CF7953D194F900302B2B07D1631C0A
:10CE20001C46013394F90020202AF9D0012620461F
:10CE3000FDF7D4F923465FFA80F81C4613F8017B0E
:10CE4000A7F13002D2B2092AF7D977B118461C46A9
:10CE5000FDF7C4F92346C7B21C4601332278303AA5
:10CE6000D2B2092AF8D906B1013694F9003053BB81
:10CE7000102D14D122461178A1F13000C0B209283A
:10CE8000144602F10102F6D92029204607D145783F
:10CE9000303DEDB21446092D8CBF10253025AA0671
:10CEA0001AD54B458DF80B808DF80A70ADF8083017
:10CEB00003D803F5FA63ADF80830302D37D1302DA3
:10CEC00008BF1025B3E701342046FDF787F983B288
:10CED000002ECDD00136CBE7032E21D8DFE806F0B7
:10CEE00002090C138DF80D808DF80E708DF80F303F
:10CEF000E3E7059B434411E0059B3C2202FB08331A
:10CF00001F4405970EE0059A4FF4616101FB08226A
:10CF10004FF03C0818FB072757FA83F3059301E00D
:10CF2000002ECAD001A80599FFF754FEC5E7102DC1
:10CF30000ABF084B0123019301A808BF06238DF8FF
:10CF4000103008F0FFFF002007B0BDE8F08300BFFD
:10CF5000B4A4010081C60000B0F804C02DE9F04778
:10CF6000042340F2B2740022644504F0030617D291
:10CF700001344EB902F1F17202F505420233DBB21F
:10CF8000062BF1D9073BFAE702F1F07202F599326C
:10CF900002F5C0720133DBB2062BE5D9073BFAE795
:10CFA0008579DFF8C080DFF8C0906C1E54B1013C79
:10CFB00014F8087009FB07223B44DBB2062BF5D9B5
:10CFC000073BFAE75EB9022D09D902F5A83202F54E
:10CFD000C0720133DBB2062B01D9073BFAE790F8A8
:10CFE000078008F1FF394B44DBB2062B01D9073B20
:10CFF000FAE7867A477AC47A30B24FEA800A80012B
:10D00000CAEB00004FF4616A0AFB0700DFF858A082
:10D0100020440AFB0900104489B10A4AA2F800C062
:10D02000094A1570094A82F80080094A1770094AAE
:10D030001670094A1470094A1370094B1860BDE84C
:10D04000F08700BF4482FF1F4282FF1F4682FF1FFE
:10D05000A58AFF1FA68AFF1FA48AFF1F4082FF1F09
:10D06000A08AFF1F2AA401008051010038B5104B8F
:10D070001B685B8C5904054619D50E4C94F9003099
:10D08000002B0ADA10200C49032206F079FE002852
:10D09000207002DB7B2106F099FE084B00221A600B
:10D0A00029466B200222BDE83840FFF701BA38BD9F
:10D0B000EC82FF1F4182FF1F89C60000BC8AFF1F50
:10D0C00010B586B0044606A8422340F8144D8DF8EA
:10D0D000103008F037FF0128024605D1064B6B20BF
:10D0E00032211C60FFF7E4F96B2032210622FFF7A2
:10D0F000DFF906B010BD00BF9C8AFF1F30B5284D78
:10D10000847B8FB0204606A90522FCF7A1FE0028EB
:10D1100043D09DF81B3013B1412B25D0F2E79DF889
:10D120001C30013B052BEDD801A252F823F000BFC3
:10D1300049D1000081D1000051D1000005D100008B
:10D1400005D1000055D100002868FFF7B9FFD9E7E5
:10D15000012016E0122301A88DF8103008F0F2FE2D
:10D160006B203221062215E0204606A99DF81C20DE
:10D17000FCF76EFE9DF81830032B05D0042BC1D1AF
:10D180000020FFF793FBBDE7064B02221A606B20DD
:10D1900043F69821FFF78CF9B4E70FB030BD00BF1C
:10D1A0009C8AFF1FBC8AFF1FF8B51D4B1D4D1E68D2
:10D1B0003223B6FBF3F6B6FBF5F402460021204617
:10D1C000FCF734FF442141706121817005FB146636
:10D1D00079214FF461652023B6FBF5F4C170024656
:10D1E0007321037043710171063220460021FCF760
:10D1F0001DFF05FB14663C253A27B6FBF5F40246F5
:10D200000770022120460132FCF710FF024607702A
:10D21000022105FB14600132BDE8F840FCF706BFAF
:10D22000248AFF1F8051010008B56C20FDF78AFB9E
:10D2300018B9BDE8084009F033BD08BD000900F089
:10D240000E00062810B522D8134B1A7882421A46CF
:10D250001FD0124B196841F480611960A0F140049D
:10D260000F49E4B2D96244F0C0540E4944F480340A
:10D270002C330C601C4621680B4B8903FBD50B49F2
:10D280000968196841F400311960107001E000204C
:10D2900010BD012010BD00BF5891FF1F00C002400B
:10D2A00000000A1A34C002402CC0024038C00240BC
:10D2B000204B1A6842F4806210B51A601E4A40F092
:10D2C0001040DA621D4A40F480302C33106018465A
:10D2D00002681B4B9403FBD51A4A10681868CCB23D
:10D2E00040F40030186044F01044144844F4803492
:10D2F00004601C462068124B8003FBD514681A6832
:10D30000090A42F400321A6041F0C0510B4A41F45C
:10D310008031E4B211601968094A8803FBD5094BD2
:10D3200018681368C0B243F40033136044EA002065
:10D3300010BD00BF00C0024000000A1A34C0024005
:10D340002CC0024038C002402B4B1A6842F4806265
:10D3500030B51A60294A40F01040DA62284A40F499
:10D3600080302C33106018460268264B9403FBD59E
:10D37000254A10681868C1F3074440F4003018606B
:10D3800044F010441E4844F4803404601C46206875
:10D390001C4B8003FBD514681A68C1F3072042F4C4
:10D3A00000321A6040F01040154A40F4803010609E
:10D3B000E4B218460268134B9503FBD5124A156870
:10D3C0001868C9B240F40030186041F0C0510C48F0
:10D3D00041F48031EDB201602D0211461868094A0E
:10D3E0008003FBD508681368C0B245EA004043F4E7
:10D3F00000331360204330BD00C0024000000A1A11
:10D4000034C002402CC0024038C002401E4B2DE9FF
:10D41000F0411C6844F480641C601C4C40F01040D7
:10D42000DC621B4C2C3340F4803020601C462068AA
:10D43000184B8503FBD5184D184F28681868DFF87E
:10D4400060C040F40030186011484FF6FF761C466B
:10D45000013A92B2B24214D012B9C0F800C000E052
:10D460000760D3F8008018F4003FFAD0D5F80080A8
:10D4700001F8018BD4F8008048F40038C4F800802B
:10D48000E6E7BDE8F08100BF00C0024000000A1AD4
:10D4900034C002402CC0024038C00240FF0001905E
:10D4A000FF000118012070470020704700207047DE
:10D4B0007047000008B545200421FDF771FA024BC2
:10D4C0001A6801321A6008BD0891FF1F38B504467A
:10D4D0000D46FFF7B3FE40B96DBAA9B241EA044167
:10D4E0002220BDE83840FFF72FBF04F01F00294677
:10D4F00040F04000BDE83840FFF7DABE10B5044602
:10D50000FFF79CFE28B921042020FFF71DFF80B201
:10D5100010BD04F01F004FF6FF71BDE81040FFF78B
:10D52000C7BE0000F8B50E461446014610B9882063
:10D53000FFF7CCFF1A4B1B491A6842F480621A604D
:10D54000194ADA62194A2C33116019460A68184BD5
:10D550009203FBD5174D2A681A6842F400321A600C
:10D56000124A711C18464FF6FF76013CA4B2B44231
:10D5700014D011F8017C14B947F0C05701E047F00E
:10D58000104747F4803717601F68BF03FCD52F682A
:10D59000076847F4003707600131E6E7F8BD00BFD0
:10D5A00000C002402A00019000000A1A34C0024064
:10D5B0002CC0024038C0024038B504462146022043
:10D5C000FFF784FF47F61C60FFF798FF000524D59E
:10D5D00047F61C60FFF732FE4FF40061BC20FFF7F6
:10D5E00067FE4220FFF78AFF054647F61A60FFF7FD
:10D5F00085FF10F4806F4FF0440005D01521FFF730
:10D6000065FF45F0010504E01221FFF75FFF25F0FB
:10D610000105A9B24220FFF759FF47F61A60FFF74C
:10D620006DFFC10506D51E20FFF708FE9E200221D2
:10D63000FFF73EFE204638BD7D4B1A6842F480520B
:10D64000F0B51A6053F8042C42F4006243F8042C3D
:10D65000784A40F24321116053F8042C764942F491
:10D66000006243F8042C4FF410720A6053F8041C53
:10D6700041F4006143F8041C70490A6053F8042C1B
:10D6800042F4006243F8042C6D4B40F203221A600E
:10D690006C4A6D4B1A606D4A85B004461A610B25C1
:10D6A00041F23427013D00F0BF80652647F6166041
:10D6B00041F23421FFF70AFF013E00F0B58047F642
:10D6C0001660FFF71BFFB842F0D1652647F61A60D7
:10D6D000FFF714FFC30402D4013EF7D1A4E047F6DC
:10D6E0006E60FFF7ABFD10218E20FFF7E1FD584B78
:10D6F000002223201A7007F0A1F847F61660FFF702
:10D70000FDFE06460028CDD14FF4967007F096F83E
:10D7100047F66E604FF44041FFF7D8FE4D4B304660
:10D72000314641F2EE751D80FFF7D0FE04202946F8
:10D73000FFF7CCFE062045F6FE71FFF7C7FE47F661
:10D7400016604FF4C041FFF7C1FE182046F20101F8
:10D75000FFF7BCFEE3889E0604D547F634605E21E1
:10D76000FFF7B4FEE3881D0515D547F66460FFF7A3
:10D77000C5FE6073000AA07347F66260FFF7BEFE45
:10D78000E073000A207447F66060FFF7B7FE60742C
:10D79000000AA07417E0637BA17B47F6646043EA4C
:10D7A0000121FFF793FEE37B217C47F6626043EAA9
:10D7B0000121FFF78BFEA17C637C47F6606043EAA2
:10D7C0000121FFF783FE54204FF48271FFF77EFEA4
:10D7D000662040F2E151FFF779FE6A20FFF78EFEE6
:10D7E00010F00104F9D11E20FFF728FD01219E2031
:10D7F000FFF75EFD184B8DF80440009306238DF86B
:10D80000053002238DF80E30082302936846122358
:10D81000ADF80C3008F04CFC47F6726048F240015D
:10D82000FFF754FE204601E04FF0FF3005B0F0BD99
:10D830003C80044010B0044014B0044018B00440D0
:10D840001CB00440000C3F8000C00240000A0DB82C
:10D850005891FF1F0C91FF1FB5D400002DE9F04136
:10D86000644E357888B08DBB0DF11507F2F78CFE4C
:10D870006149624C06223846FCF7E9FC45238DF8E5
:10D88000143040F2EA53ADF81030ADF812300C23EA
:10D8900022888DF81B305A4B8DF80C5002930321CF
:10D8A00042F40063042002AAADF80E30ADF81C501B
:10D8B000FCF794FB394630700622A01CFCF7C7FC2D
:10D8C00023886FEA43436FEA534323804D4FDFF8C9
:10D8D0003881042447F61C60FFF710FE41064FD53F
:10D8E00047F67260FFF7AAFC4FF40041B220FFF741
:10D8F000DFFC47F61C60FFF7A1FC4021BC20FFF7CE
:10D90000D7FC8A203988FFF7E1FD2C2069460822E0
:10D91000FFF77CFDBDF800503B493D80BDF802207B
:10D920002C20ADF81020FFF771FD41F2EE739D42FF
:10D9300018BF023D4FF01E0014BFADB245F6FE7594
:10D94000CDF80880FFF77AFC4FF480719E20FFF736
:10D95000AFFC29460620FFF7B9FD47F67260FFF7D6
:10D960006DFC92204FF40041FFF7A2FC019B1A06C8
:10D9700006D5BDF81030043BADF81030002301E0AF
:10D980004FF0FF3393BBBDF8103023B3029B1A7BDB
:10D99000082A20D15B7B062B04D002A803F08CFA66
:10D9A000C8B105E002A800F099FA0028F5D012E00D
:10D9B000029BDB7D062B0BD0112B05D0012B0AD14E
:10D9C00002A803F09FF806E002A806F015FA02E0AC
:10D9D00002A805F03BFA30780021FCF779FA013C07
:10D9E0007FF478AF45200421FCF7DAFF08B0BDE8EA
:10D9F000F08100BF0591FF1FF382FF1FF182FF1F1F
:10DA0000D0A401000C91FF1FC58AFF1F12220D4BED
:10DA100002FB010210B553F822400B2804F1010467
:10DA200043F8224005D8482251435A5801325A50EF
:10DA300010BD102805D8482202FB01331A6B0132B1
:10DA40001A6310BD1091FF1F112806D8122303FB83
:10DA50000100034B53F8200070470020704700BFBF
:10DA60001091FF1F06280FD011280BD0012801D1DB
:10DA70000E200AE0064B482202FB01310B6B0133FA
:10DA80000B6370470F2000E01020FFF7BFBF00BFFF
:10DA90001091FF1F20F0C003062B024612D0112B5D
:10DAA0000ED0012B01D103200DE00A4B4822514337
:10DAB0005A18D0690130D0615A5801325A50704713
:10DAC000042000E00520130644BF0630C0B2FFF773
:10DAD0009DBF00BF1091FF1F034B482202FB003087
:10DAE0000021FCF7ACBB00BF1091FF1F70B5094CC3
:10DAF00000231919C65C0A7B0D7A164086EA0501D7
:10DB00000A4203F1010303D1042BF2D1012070BDBD
:10DB1000002070BDF182FF1F144B1968F0B5044658
:10DB200001F169050846A84204D010F80F3F002B08
:10DB3000F9D119E00A46002301F10F06AA4211D0DB
:10DB40000F32501A304410F80F7C17F0450FF5D102
:10DB500033B110F80B7C1879874238BF1346EDE7D4
:10DB60001346EBE7184603B10470F0BD5C91FF1F4C
:10DB700013B542788DF8051000248DF8022041225B
:10DB800003468DF803200DEB0402991C901D012221
:10DB90008DF801408DF80040FCF759FB0223204628
:10DBA000694607228DF80430FCF790FC02B010BDE6
:10DBB00070B5062204460E460968FCF748FB1C496E
:10DBC0000622A01DFCF743FB0625082323732A46E3
:10DBD0006573184904F10E00FCF739FB2A46144915
:10DBE00004F11600FCF733FB1349042204F11C0076
:10DBF000FCF72DFB2A467168104D04F12000FCF75C
:10DC000026FBB168042204F12600FCF720FB2878EB
:10DC100021462A22FCF75AFC20B1002128780A4626
:10DC2000FCF754FC0D200021BDE87040FFF7EEBE6C
:10DC3000F382FF1FECA40100F982FF1F0591FF1F73
:10DC400000B58FB000238DF8203001238DF82130EE
:10DC5000064B0B300193064B0290694603A80093D4
:10DC6000FFF7A6FF0FB05DF804FB00BF24AB010077
:10DC700038AB0100F8B50D4617461E46FFF74CFFBE
:10DC80000446E8B1294604220B30FCF7E0FA0D49BE
:10DC90000622601DFCF7DBFA02250423E370204610
:10DCA0002571FFF7CDFF2378677043F04003A6701E
:10DCB00023702A4641201921BDE8F840FCF7A2BE96
:10DCC000F8BD00BF38AB01002DE9F04F4A4F90F886
:10DCD0000E903B6893B0D3B97820FCF7A9FC892358
:10DCE0003860464900F80B3B0422FCF7B0FA38686C
:10DCF000424905300622FCF7AAFA412040F6B83125
:10DD00000122FCF77FFE02E09DF80B203AB1484665
:10DD100002A90522FCF79CF80028F5D169E09DF8DE
:10DD20000C30012B3BD1D7F80080022108F1690BA0
:10DD3000464608F10F054FF0410C5E4529D006F12B
:10DD40000F0AC8EB0606735D180620D574192079F2
:10DD5000E8B10138C0B22071C8B913F0010301D194
:10DD6000735514E0E3780BB1013BE370E37863B1E2
:10DD700050460191CDF800C0FFF762FFDDF800C00A
:10DD800006F805C00122019900E07355217156463D
:10DD9000D3E7002AB1D0412019210222B1E7022B9A
:10DDA000B5D13C68924604F16908234604F10F0599
:10DDB00043451AD003F10F061B1B5A5D520612D5BC
:10DDC0005A19D17839B10139D1703046FFF738FF8F
:10DDD0004FF0010A07E0595592F901301BB1304666
:10DDE0000321FFF7C5FE3346E2E7BAF1000FD2D1B7
:10DDF00083E713B0BDE8F08F5C91FF1F38AB0100E3
:10DE00002DE9F84F324B1678D3F800800746894643
:10DE100008F1690A454608F10F0B554526D005F172
:10DE20000F04C8EB04035B4413F80F3CE3B105F1A6
:10DE30001A0039460422FCF79EFBA8B906F0040339
:10DE400003F0FF07002B41D1EB7B5B0607D595F96B
:10DE5000103023B120460421FFF78AFE2F74EB7B9C
:10DE600003F03F03EB731CE02546D6E73846FFF787
:10DE70003DFE58B3384617490422FCF77CFB30B905
:10DE8000144815490422FCF776FBF8B10126304608
:10DE9000FFF742FE0446C8B10B3039460422FCF7B6
:10DEA000D6F9601D49460622FCF7D1F9750705D45D
:10DEB00016F0010F0CBF1423052300E0002323718B
:10DEC0000423E370237863F07F032370BDE8F88FA9
:10DED0005C91FF1F0183FF1F24AB01002DE9F04F70
:10DEE000046894F80C80B8F1080F91B040F08F806E
:10DEF00003891B2B40F28B80227D637D43EA022342
:10DF0000012B04F1160502D0022B21D07FE002275D
:10DF100041488DF8047004F126010422FCF72BFB24
:10DF2000064698B91C348DF8280002A905A88DF87A
:10DF30002970029503950494FFF73AFE204629467E
:10DF400001AAFFF75DFF384631465CE0404659E0E4
:10DF500031488DF8143004F12601042204F11C0725
:10DF6000FCF709FB002841D12C4B1E6806F1690A19
:10DF7000344606F10F0B544536D004F10F08C6EBBA
:10DF800008035B4413F80F3C63B3384604F11A01ED
:10DF90000422FCF7F0FA814620BB294604F1140064
:10DFA0000622FCF754F9E37B590706D413F0010F5E
:10DFB0000CBF4FF014094FF0050904215A0684F8EC
:10DFC0001390A17407D594F9103023B14046FFF7A0
:10DFD000CFFD00232374E37B03F03F0363F07F0353
:10DFE000E37301E04446C6E702200BE038460C49E3
:10DFF0000422FCF7C0FA20B13846294605AAFFF7EB
:10E00000FFFE08200021FFF701FD012000E00020B5
:10E0100011B0BDE8F08F00BFF982FF1F5C91FF1FB8
:10E0200038AB01002DE9F04788463549354C174695
:10E0300004230A1D0546266802F028FFA146002891
:10E040005AD106F10B0406F1830A5445A4F10B06DC
:10E050000DD014F80B3C43B1204629460422FCF7AE
:10E060008AFA10B996F900303AE00F34EDE7284605
:10E07000FFF73CFD88B1284623490422FCF77BFAD0
:10E0800008B1022007E0204820490422FCF773FA77
:10E090000028F6D00120294627E01B481B4904220E
:10E0A000FCF769FA28B3D9F8005005F169092C4644
:10E0B00005F10F0A00E034464C4514D004F10F0678
:10E0C000731B534413F80F3C002BF4D004F11A00D7
:10E0D0000D490422FCF74FFA0028ECD194F90F30D7
:10E0E000002B09DB05E00849012042463B46FFF7CB
:10E0F000C1FD0020BDE8F0873046BDE8F08700BFD5
:10E10000F982FF1F5C91FF1F0183FF1F24AB0100F9
:10E110000C4B1A6870B5134602F16904002102F134
:10E120000F05A3420CD00F339E1A2E4416F90F6C24
:10E13000002EF6DA0131C9B28142F2D1184670BD23
:10E14000002070BD5C91FF1F054B1B68002203F18E
:10E1500069018B4203D0DA731A740F33F9E7704701
:10E160005C91FF1F02681378591C11440160002064
:10E17000013BDBB2FF2B04D012F8011F41EA002063
:10E18000F6E7704710B503681A78541C1C44033A2C
:10E1900004600846BDE8104099180422FCF757B8FF
:10E1A000F0B5D1B000214FF49672054605A8FCF7F2
:10E1B00046F85049504C514F0C2205A8FCF747F83F
:10E1C000FCF76EFB2070FCF76BFB6070FCF768FBE4
:10E1D000A070FCF765FB2146E070042206A8FCF75E
:10E1E00036F83B7813F0E00F04D008A84449042225
:10E1F000FCF72DF8434906220CA8FCF728F840A8A4
:10E2000041490622FCF723F8012D8DF806512AD04A
:10E2100033D3EB1E012B4FF004022ED83B7813F0C2
:10E22000C00F0DD132238DF8073103AB03F1FD0090
:10E2300036498DF808210DF20D14FCF708F802E0BC
:10E2400003A800F1FB043B7813F0C50F08D1362377
:10E25000042223706270A01C2D49FBF7F8FF0634DE
:10E26000042D03D10CE003AB03F1FB042046294944
:10E270000922FBF7ECFF093402E003A800F1FB04DC
:10E280000DF10B00F2F73EF9014690B19DF80B201D
:10E290007AB1D31C234450A883420AD226460C23C9
:10E2A00006F8023B62703046FBF7D1FF9DF80B4049
:10E2B0003444FF2323703B78174A13F0600F4FF468
:10E2C000967392F9000000934FF04403019309D034
:10E2D0000F49432203AB05F029FE013007D10F4B54
:10E2E0001D7004E00E49432203AB05F01FFE51B040
:10E2F000F0BD00BFFBA401006091FF1F7891FF1FDC
:10E30000F982FF1FF382FF1F07A501007C91FF1F09
:10E310006591FF1FF2A401004782FF1F7991FF1F43
:10E3200038AB010038B504460D46FCF7B9FA40F2A7
:10E330003333B0FBF3F083B2322B86BF643C13FA65
:10E3400084F31B1999B22A464420BDE83840FCF7F3
:10E3500059BB0000092810B5104B04D00A2814BF7F
:10E3600002460B2203E01A68013215D008221B680E
:10E370000A4C93B140F21D518B4205D9A3F21E53B2
:10E3800023604FF6FF7104E032214B4399B2002322
:10E3900023604420FCF736FB002010BD7091FF1F66
:10E3A00010B5094C4420FCF791FB08490422204693
:10E3B000FBF74DFFFFF7C8FE204644210022BDE8D1
:10E3C0001040FFF72FBE00BFF982FF1F7C91FF1F97
:10E3D000F8B57D4D2B78082B04462E4600F0818041
:10E3E0000CD8022B78D0042B15D0012B40F0EB80F9
:10E3F00004232B70754BC8221A800CE0202B77D099
:10E4000002D8102B0AD0F8BD402B00F08380802B5F
:10E4100000F0B180F8BD062C00F0D180072C0AD0A6
:10E42000042C16D12046FFF7BBFE694BDB2193F984
:10E430000000FCF78BF802230021664833700422A9
:10E44000FBF7FDFE40F226200121BDE8F840FFF772
:10E4500069BF052C26D1604A604B106819680A30E4
:10E4600081421D4603D88B080320434313605C4858
:10E4700013680468A3F10A07BC4204D30324B3FB66
:10E48000F4F464000460C91A2960016820245B1A4E
:10E49000092013603470FFF75DFF4D4BDC2193F9C9
:10E4A000000015E0494C0320FFF77AFE2088032185
:10E4B000FFF738FF23885B009BB2B3F5486F2380DA
:10E4C00040F28180C8232380414B93F90000D92179
:10E4D000BDE8F840FCF73AB808232B703B4BC82244
:10E4E0001A803A4C0120FFF75BFE20880221DFE70B
:10E4F000FFF730FF002866D0082C64D140230320AA
:10E500002B70FFF74DFE344A13685B081360344AE2
:10E5100013602BE008281BD1FFF71CFF002852D006
:10E520002D4A13685B0813602D4A3B2B136007D8F4
:10E530002A4980232B700B685B080B60136038E05E
:10E540000920FFF707FF0320BDE8F840FFF728BECA
:10E55000062838D1202321492B701F4B08681A68E0
:10E56000801A08601E490968521A1A600920BDE81D
:10E57000F840FFF7EFBE0B281DD1FFF7EBFE10B3FD
:10E58000164A13685B081360154A3B2B136010D8BA
:10E590000223002104220F482B70FBF750FE40F2AB
:10E5A00026200121FFF7BEFE094BDA2193F9000076
:10E5B0008EE70A20C5E7062805D110232B70BDE899
:10E5C000F840FFF7EDBEF8BD7891FF1F7A91FF1F6D
:10E5D0006491FF1FF982FF1F6C91FF1F7491FF1F51
:10E5E0007091FF1F2DE9FF41A84B0A9D93F9003060
:10E5F0008342174640F06C81012940F06C81BDF8E0
:10E600002C30E32B40F269812B78022B40F065819E
:10E61000281D9F490422FBF7AEFF002840F06081CF
:10E6200005F11001042201A8FBF711FE05F1180104
:10E63000042202A8FBF70BFE05F11C0095490622F7
:10E64000FBF799FF002840F04B8105F1EC0092495F
:10E650000422FBF790FF0446002840F036818F4EDD
:10E660003378102B05F1F00514D033780395102B77
:10E6700027D009D8042B27D0082B40F00381002590
:10E680002F46DFF824822CE0402B1DD0802B40F059
:10E69000F98019E001A882490422FBF76CFF0028E9
:10E6A00040F01E817F4839460422FBF764FF0028B2
:10E6B000DBD002A839460422FBF75DFF0028D4D046
:10E6C0000EE1794D794E5DE00025784E784FA4E05B
:10E6D0004B1C03930B78062B2BD00CD8012B25D089
:10E6E00004D203990B78FF2BF2D12BE0032B25D119
:10E6F00003A870491FE0352B09D0362B0BD0332BE4
:10E700001CD103A8FFF72EFDC8F80000E9E7CB1CD9
:10E7100003938D78E5E70231624803910422FBF709
:10E7200096FD039B043303930127DAE703A86249AC
:10E7300001E0624903A8FFF725FDD2E703A8FFF730
:10E7400011FDCEE7002F00F0BD80022D40F0BA8011
:10E75000102301A9042252483370FBF778FD0320EF
:10E76000FFF71EFD564BC82003211880FFF7DAFD86
:10E77000B8E04B1C03930B78332B31D00ED8012B10
:10E780001CD004D203990B78FF2BF2D1AAE0032B03
:10E7900017D0062B36D103A8484914E0362B15D0E4
:10E7A00002D8352B21D02DE03A2B26D03B2B29D176
:10E7B00003A8FFF7D7FC3E4B1860E3E703A83E49E8
:10E7C00001E03C4903A8FFF7DDFCDBE702313548F7
:10E7D00003910422FBF73BFD039B04330393D1E732
:10E7E00003A8FFF7BFFC2860CCE7CB1C03938B7812
:10E7F000052B72D1FFF7D4FDC4E703A8FFF7B2FCE5
:10E800003060BFE703A8FFF7ADFCBBE75A1C0392DB
:10E810001A78352A17D00DD822B9039B1A78FF2A07
:10E82000F4D12AE0332A24D103A8FFF79BFC1E4B26
:10E830001860F2E73A2A17D03B2A1AD103A8FFF74B
:10E8400091FC3860E9E79A1C03929A78062A05D170
:10E850000720FFF7BDFD4FF0FF3443E00333052AE7
:10E8600008BF01250393D8E703A8FFF77BFC3060BE
:10E87000D3E703A8FFF776FCCFE79DB30620FFF7A9
:10E88000A7FD2FE06FF006042CE000BF4782FF1FBA
:10E890006091FF1FF382FF1F07A501007891FF1F02
:10E8A0007C91FF1F6591FF1F7491FF1F7091FF1FE7
:10E8B0006C91FF1F0183FF1FFD82FF1F0583FF1F58
:10E8C0007A91FF1F6FF003040CE06FF0090409E078
:10E8D0006FF0070406E0002404E06FF0050401E097
:10E8E0006FF00804204604B0BDE8F08110B5847BC9
:10E8F0008AB0204669460522FBF7AAFA00B39DF8C4
:10E9000003309DF80420412B17D120466946FBF7C0
:10E910009FFA9DF800300B4C042B06D1207810B1E3
:10E92000FFF73EFC06E0184602E0032B02D105206B
:10E93000FFF74EFD0023237002E01046FFF748FD6D
:10E940000AB010BD7991FF1F70B51C4C94F90030CE
:10E95000002B054626460CDB96F90000184C442196
:10E9600005F034FA174B05F07F02002D1A700BDA10
:10E9700017E010201449032205F002FA0028207045
:10E98000EADA6FF0010070BD104811490422FBF76C
:10E99000F2FD30B10F480D490422FBF758FC01236A
:10E9A00000E002230422002108482370FBF747FC03
:10E9B000C8200121FFF7B6FC002070BD4782FF1F71
:10E9C0007891FF1F6491FF1FE5E50000F982FF1FAA
:10E9D00024AB01007C91FF1F08B54420FCF776F8BA
:10E9E000044B0548054900221A70BDE8084004227E
:10E9F000FBF72DBC7891FF1FF982FF1F7C91FF1F51
:10EA000008B5024B00211B68984708BD8891FF1F7D
:10EA10002DE9F043454B1A78012ACBB0074602D0C6
:10EA2000032A0FD072E002221A70414B1860414B4A
:10EA30004148196004224149FBF709FC404B05227B
:10EA40001A7003E03A4B1B6883425FD140F2111207
:10EA5000002105A8FBF7F3FBFBF722FF394B8DF8EC
:10EA60001400188000220123000ADFF8E0808DF8EE
:10EA700015008DF816308DF817208DF818208DF8B8
:10EA8000193008AC0C2540F2131997F90000002842
:10EA900047D0C5F5887001343E4600230130F95C4B
:10EAA0004AB22E2A08D039B10133834231D216F846
:10EAB000012B04F8012BF2E7591E3E292CD81D44E6
:10EAC000AFB27D1CADB24D4529D82E2A6FEA0301A5
:10EAD00008BF0136635496F90030ABB91A490522D4
:10EAE0002046FBF7B4FB642001460122BD1DFBF765
:10EAF00089FFADB26423019398F9000000950E4997
:10EB0000352203AB05F012FA3746BEE74FF6FF7029
:10EB100007E04FF6FC7004E04FF6FE7001E04FF6A0
:10EB2000FD7000B24BB0BDE8F08300BF8791FF1FBE
:10EB30008C91FF1F8891FF1F8091FF1F0583FF1F8E
:10EB40008691FF1F8491FF1F11A501004882FF1FBE
:10EB500008B5094A094B117859B103201870084BC0
:10EB60001868084B013911701968FFF751FF002030
:10EB700008BD0120187008BD8691FF1F8791FF1FF7
:10EB80008C91FF1F8891FF1F10B51F4B847B1A7853
:10EB90008AB072B901221A70102003221B4905F0B5
:10EBA000EFF81B4A002810702BDB352105F00EF919
:10EBB00027E0204669460522FBF74AF908B39DF88D
:10EBC0000330412B16D1204669469DF80420FBF7FF
:10EBD0003FF99DF80030032B04D1FFF7B9FF80B156
:10EBE0000A200CE0042B0CD10A4B06221A70FFF706
:10EBF000AFFF06E02BB9FFF7ABFF10B10B20FFF71B
:10EC0000FFFE0AB010BD00BF8791FF1F19EC000086
:10EC10004882FF1F8691FF1F2DE9F84F5B4B0A9D2D
:10EC200093F9003083420E4640F0AB80584B197880
:10EC3000012900F0A680104656490422FBF79BFCF0
:10EC40000446002840F09D80012E40F09C80BDF8D5
:10EC50002C30072B40F295804F4B29781B88DAB275
:10EC6000914240F08E806A78B2EB132F40F0898099
:10EC7000AB78190640F1858013F07A0F0DD1EB784F
:10EC80005A0605D01B0603D50D20FFF7B9FE78E024
:10EC90002B7913B96B79012B01D00C20F5E73F4B91
:10ECA00095F806A01C68EF7995F808906E7A0C35F7
:10ECB00095F800B005F10108BBF1000F11D04046F6
:10ECC00021465A46FBF757FC00285AD15C4408EB12
:10ECD0000B052378002BEBD02E2B04F10104E7D099
:10ECE0004FE02F4829460522FBF745FC0446002843
:10ECF000D3D147EA0A2746EA0929691DB9F1000F6D
:10ED00003CD00B780E46013123B103F0C003C02B79
:10ED1000F7D10E46711C04222248FBF72CFC727AB4
:10ED2000B37A054606F10B0143EA0222C8B9042A68
:10ED300017D11848FBF78BFA67B16420FBF7C6FEC2
:10ED4000194B14491B6801209847114A012313707D
:10ED50002C4618E0154B06221A703C46FFF7F8FEC9
:10ED600011E0114417B1013FBFB2C7E7B9F1000F7D
:10ED700009D009F1FF391FFA89F9BFE7002FC0D187
:10ED800001E04FF0FF342046BDE8F88F4882FF1FB6
:10ED90008791FF1F8091FF1F8491FF1F8C91FF1FA0
:10EDA00011A501000DA501008891FF1F8691FF1F8D
:10EDB00003461A46013392F900101F29F9DC00239B
:10EDC0001370704738B5094C2468248FA40709D5FF
:10EDD000074CA56835B1114620461A46FAF7FAF9EC
:10EDE000A08F38BDFDF74AFA80B238BD0092FF1FF0
:10EDF0009091FF1F2DE9F04F0C46ADF2EC5D0D78C0
:10EE0000002800F01582022804D801D1887F07E08D
:10EE1000087E02E0272802D90876657800E0887726
:10EE20000A381F2800F20482DFE810F02000F60103
:10EE30002300260028002B002E0030003300600045
:10EE400062000401A600AD0068006500020207012F
:10EE5000A800AA0002020202020202020202020248
:10EE600002020202020202020B01C100A0491A249E
:10EE7000D6E1A0491124D3E19F4908E09F490E241F
:10EE8000CEE19F490B24CBE19E4935E09E490D24FC
:10EE9000C6E19E4F3B681B8F9E0740F1BF8108AEC5
:10EEA0009B49052206F11400FBF7D1F93B6818686D
:10EEB000FBF790FB84B2022C06D9023CA4B240F2CC
:10EEC000AC539C4228BF1C463B681968224602315D
:10EED00006F11900FBF7BBF90444204603228D49D3
:10EEE000A41BFBF7B4F9A4F111023AE08A4996E1B8
:10EEF0008A49122494E18A49132491E108AE0F2231
:10EF000006F114008749DFF84882FBF7A0F90027D3
:10EF100006F123024FF02C0907EB08030021187AB1
:10EF2000FBF784F80137042F00F1010280F800900C
:10EF3000F2D1E08A0021000AFBF778F82C23037055
:10EF400002460132A07D0021FBF770F829230370EF
:10EF50002E2343700D2383700A23C370801BA0F1FE
:10EF6000100268B2314692B2082303F07DFB0028FC
:10EF7000D4BF0020012061E16B4988E76B494EE175
:10EF80006B4908244CE10DAE6A4904223046FBF778
:10EF90005EF900210EAA6068FBF748F80D230370A4
:10EFA0000A2343700230821B08A968B2DBE76DB206
:10EFB000284603F001FB438C40F2B45293420646CC
:10EFC00004D840F2D922934201D833E113460DAA66
:10EFD000E0686168FFF7F6FE02462082002800F034
:10EFE0002781284608A9082303F03EFB071E40F3AB
:10EFF0002481228AF38C1344F384738C9B1A9BB272
:10F0000040F2B4518B4201D80BB916E10B4661684E
:10F01000E06811440DAAFFF7D5FE0246002800F073
:10F020000C81238A03442382284608A9082303F07D
:10F030001BFB03E140490C24F2E0042323773F4902
:10F04000EDE0324B1B681E8F06F00206B6B2FEB131
:10F050003B4E3C493C480DAB3360012333752C22B9
:10F0600040F2B4533381FBF7F2F836483146F9F7F2
:10F07000C1FD0F30F08904BF0023B38130B10123FB
:10F08000A3822F4B68B208A95A896DE7A082D5E008
:10F090000DF1180A2D4907225046FBF7D8F83046E3
:10F0A0000DF1130205A9FDF713F80AF10202334628
:10F0B0003746B04681460DAE0392059A002A00F00D
:10F0C0009A80A28A03F1010B5FFA8BFB9342CDF881
:10F0D00008B0C0F087800FFA88F303F284539F4290
:10F0E00038D90BF1FF3B6282A4F814B088E000BF6E
:10F0F00052A6010089A601007BA6010043A60100DB
:10F1000034A5010016A501002AA601000092FF1FE8
:10F1100080A5010086A50100B4A6010059A5010043
:10F120006CA5010040A501009BA601002AA50100D5
:10F13000A3A5010077A601008AA501004FA5010043
:10F140000492FF1FD491FF1F1C92FF1FACA501006A
:10F15000F182FF1F30463C490A22FBF778F806F19E
:10F160000A003A490B22FBF772F806F1150C6246C9
:10F1700000210598CDF804C0FAF758FFDDF804C067
:10F180003349C0EB0C0C0C2208F108088346E0441C
:10F19000FBF75DF89DF813202E4B03980A2A84BFD5
:10F1A0000A228DF813209DF813200BF10C0C53F854
:10F1B0002210CDF804C00322FBF749F84846FDF7BA
:10F1C0009FF88AF80000DDF804C051466046072227
:10F1D000FBF73DF80BF113039E1B37441FFA88F829
:10F1E000BFB21E46484605A90DF11302FCF770FF99
:10F1F000029B814661E71BB1A28A13446282A3820B
:10F200001FB168B208A93A46AEE6A38A83B90123C2
:10F21000A38211490A2403E0104900E0104909249F
:10F2200022460DA8FBF713F868B208A922469BE610
:10F23000002003E04FF6FF7000E0384600B20DF208
:10F24000EC5DBDE8F08F00BF20A60100A9A601007B
:10F2500097A50100A082FF1F38A601006DA601003E
:10F2600080A5010038B58D7F0C461DB9FFF7C2FDA2
:10F27000E57738BDE07738BD38B50446214629200A
:10F28000FFF7B8FD054618B107236377002038BDA6
:10F2900021460B20FFF7E6FF657794F9010003F0A4
:10F2A00079FD082038BD00002DE9F341A14C154639
:10F2B00004F1400294F90030984203D02034944283
:10F2C000F8D3DDE20139072900F2D682DFE811F038
:10F2D0002D00080018003600D4022D00CD02CF0208
:10F2E0004FF002110020FAF739FC934B0221186805
:10F2F000FAF734FC012323770023A3770A2031E0B7
:10F30000637F0025012BA57700F0B882237F042BB3
:10F3100005D103F03FFD012323770820B1E2E07F10
:10F32000E5772146FFF766FDA8E20025184615217E
:10F330002A462577657703F05BF99FE2237F012B4F
:10F3400014D128467D4901F033FD78B17C4B1B7800
:10F35000DF0704D52844092104F0CCFF607602239E
:10F3600023770C202146FFF745FD8AE2237F022BFD
:10F3700019D12846734901F01BFDA0B1704B1B78D1
:10F38000DE070CD528440A21667E04F0B3FF304323
:10F39000C0B2607618B1042323770E20E2E703237E
:10F3A00023770D20DEE7237F032B40F05C82284685
:10F3B000654901F0FDFC08B11020D3E728466349F8
:10F3C00001F0F6FC002840F0CC812846604901F0AD
:10F3D000EFFC002840F0288228465E4901F0E8FC56
:10F3E000F8B1A27E12F001050ED094F9000003F0EE
:10F3F000D1FCA37E980703D594F9010003F0CAFC61
:10F400000023A37610203CE203F09EF8012301467E
:10F41000E0822A4694F90100A37603F0E9F8182067
:10F42000A0E728464C4901F0C3FC00284FD12846EC
:10F430004A4901F0BDFC88B13F4B1E68338F9907E4
:10F440000AD5474B281D1E60FFF7B2FC3146FAF77C
:10F4500035F8002840F08581142083E7284641498B
:10F4600001F0A6FC98BB28463F4901F0A1FC80B3FF
:10F4700004F108062844314601F063FC03461D46AA
:10F480001A1A95F900102F2903F10103F7DC2B2339
:10F490002B70A81AFAF7A2FE0002E0822B465A1C33
:10F4A000581B93F901302F2B01DD1346F7E700239A
:10F4B0001370101AE58AFAF791FE2844E08231466B
:10F4C0002A480422FBF757F808B919204AE7132005
:10F4D00048E72846264901F06BFC00285FD0164B10
:10F4E0001B681A8F92070ED51D4E681D3360FFF7FB
:10F4F0005FFC3146F9F7D0FE002840F032811D4B09
:10F500004FF6FF729A81A57E15F0010534D00F20C9
:10F510002146FFF76FFC00236382A382A37E0028AD
:10F52000D4BF002501259B0737D521462820FFF7AA
:10F5300061FC32E04C82FF1F0092FF1FB4A5010066
:10F540004892FF1FBAA50100C0A50100C5A5010092
:10F55000CAA50100CEA50100D3A50100D8A50100D0
:10F56000D491FF1FDCA50100E2A5010024AB01003E
:10F57000E8A501000492FF1F20786378E28A0095D5
:10F5800020F01F001843607004F1080140B21423FA
:10F5900003F094FB0028C0F2E480012304E1284634
:10F5A000A24901F005FC00283BD02078637820F0C8
:10F5B0001F001843A37E607013F0010308D09C4B1A
:10F5C0001E68338F13F0020F05F105050BD116E00D
:10F5D0000093E28A40B204F10801142303F06EFBA9
:10F5E0000028ECDABDE02846FFF7E2FB91493246FD
:10F5F00040F20263FAF7DAF8022808D0B1E02846B0
:10F60000FCF740FDE060284601F0ECFBE076A07ED0
:10F6100010F0010003D0032363770F20A2E602233A
:10F6200085E028468449824E01F0C2FB48B3376822
:10F630003E8F06F002060535B6B2284636B1FFF712
:10F64000B7FB3946FAF7CEF8C8B18AE07B4901F03A
:10F65000AFFB38B14FF410304FF4E031FCF762FDEE
:10F6600066600CE02846FCF70DFD0546FCF716FD2C
:10F67000411D2846A5F51035FCF754FD65601620A0
:10F6800070E628466E4901F093FB0746E0B1366804
:10F69000338F9F070DD5681D664DFFF789FB2946FF
:10F6A00032460123FAF782F802285AD1AB68636028
:10F6B00008E06B792F2B54D0681DFCF7E3FCA0F514
:10F6C0001030606017204DE628465E4901F070FB5F
:10F6D00000286BD020786378D6F8008020F01F00D7
:10F6E00018436070B8F8386006F00206B6B26EB320
:10F6F000681DFFF75DFB01234E494246FAF756F8B5
:10F700000228A37E04D09E0729D594F9010024E0A5
:10F7100013F0010567600CD003F0020303F0FF0053
:10F7200023B12046FFF7A8FD3846AAE006236377F9
:10F73000A7E094F90100E28A009504F1080114237E
:10F7400003F0BCFA00280CDB06232DE06B792F2B8D
:10F7500009D1A37E9D0702D540B203F01BFB002315
:10F76000A3761120FEE5681DFCF78CFCE060FCF739
:10F7700095FC78B194F90100E28A009604F1080141
:10F78000142303F09BFA002804DB062363776660EA
:10F79000304676E0A37ED907E3D50025292021460F
:10F7A0006560FFF727FB0723637767E033681B8FEC
:10F7B0009A0710D52846244901F0FAFA58B1681D75
:10F7C000FFF7F6FA1B4932682023F9F7EFFF00280C
:10F7D000C7DB1C20C6E533681B8F9B070ED5284668
:10F7E0001A4901F0E5FA48B1681DFFF7E1FA11493D
:10F7F000F9F766FD0028B4D11D20B3E533681B8FEF
:10F800009F0729D52846124901F0D2FA20B9284687
:10F81000104901F0CDFAF8B12844FFF7C9FA316870
:10F82000FAF73EF800289CD112209BE5EDA50100D7
:10F830000092FF1F9091FF1FF3A50100F9A50100A1
:10F84000FDA5010003A6010009A601000FA6010005
:10F8500015A6010016A6010028460B4901F0A8FADA
:10F8600008B11B207EE515207CE502207AE5237F88
:10F8700033B92070184604E0002002E0284600E07A
:10F88000022002B0BDE8F0811BA601002DE9F04185
:10F890007A4C1E4605468846174604F1400394F903
:10F8A0000120AA4205D020349C42F8D30220BDE8B2
:10F8B000F08194F9000002F0D0FEA8F102010629BF
:10F8C00000F2D980DFE811F0070034008000C900A1
:10F8D0005B00A500D200A27E02F0FB03D007A37656
:10F8E00003D543F00203A37603E00F202146FFF780
:10F8F000B9FC637F012B03D100236382A3821AE04A
:10F90000022B02D103236377B5E0062B0BD12146EE
:10F910000F20FFF76FFA00282046D4BF00250125ED
:10F92000FFF7AAFC69E0A37E43F00403A376A2E0FC
:10F93000637F012B13D128202146FFF75BFA054690
:10F94000002840F0988021460B20FFF78BFC65775C
:10F9500094F9010003F01EFA0820BDE8F081072B9E
:10F9600040F08980464B1B680022DA846368228A53
:10F97000134463602046BDE8F041FFF77DBC637F20
:10F98000032B14D13F4B1B681B8F990703D53E48AF
:10F99000F9F7E4FC04E0E06804F11B01FCF786FCE5
:10F9A0000B202146FFF75EFC0023637708E0A37F6E
:10F9B00013B9E07FE37700E000202146FFF71AFA51
:10F9C0000020A076BDE8F081637F032BA37E17D1D2
:10F9D00023F00403A3762B4B1B681D8F05F0020553
:10F9E000ADB22DB1394632462748F9F7CFFC42E097
:10F9F000E06839463246FCF79DFB2846BDE8F081B9
:10FA000003F0040303F0FF00002B35D01020BDE805
:10FA1000F0811C4B1B681B8F9A0712D5A38A4BB130
:10FA20002C221A481A49FAF712FC1A4B4FF6FF72A9
:10FA30009A8108E0218A144849420122F9F784FD9D
:10FA400001E0638AA3820E4B1B680022DA84214600
:10FA50000120FFF7CFF9BDE8F081A37E03F0040396
:10FA600003F0FF00002BD1D1BDE8F081A37EDB07BE
:10FA70007FF51CAF65700020BDE8F0814C82FF1F50
:10FA8000D892FF1F0092FF1F9091FF1FD491FF1F7C
:10FA90001C92FF1F0492FF1F70B51B4B93F900309F
:10FAA000013306460C462ED1184D286858B98021DE
:10FAB000F9F72EFA04F00203286003F0FF0013B9EF
:10FAC0000221FAF74BF8124B1C70124C04F120057E
:10FAD0003146114A102002F005FD1521002204F8DC
:10FAE000200C02F085FD002304F8043C0820782156
:10FAF0000A4A02F0F7FCAC4204F81F0C04F12003A0
:10FB000001D21C46E4E770BD4C82FF1F0092FF1F2C
:10FB10004892FF1F6C82FF1FA9F200008DF80000C1
:10FB200070B50A4CFF2504F1200614F9200C02F0F0
:10FB300051FD14F91F0C02F04DFDB44204F8205C95
:10FB400004F1200301D21C46EFE770BD6C82FF1F59
:10FB50002DE9F04F8FB00C460790089315462AB94F
:10FB60008D8B81F84120CD878A8304E091F8413064
:10FB7000013381F8413094F84230DFF8309323F0BC
:10FB80002103002284F84230AA460392A38B94F802
:10FB90002260A4F81CA02B449BB20993CAEB050376
:10FBA0009BB20493049A079BADF830A013440D93C5
:10FBB000002E40F00D81079B089A1344059304F131
:10FBC0001C030693BDF83020002A00F001810D9B34
:10FBD000581C0D901978A32940F0F480032A44D9C9
:10FBE000991C0D915B78642B0AD004D8442B07D064
:10FBF000482B2DD0C2E0732B02D0762B1BD0BDE05A
:10FC0000A54A126822B1732B08BF084690470646E2
:10FC1000002E00F0B580022E04D10723ADF832305B
:10FC20009E4FAEE0032E4FF00803ADF832300CBF0C
:10FC30009B4F9C4FA5E0D9F80070002F00F0A180E9
:10FC400008460DF1320200212346B847074698E0E6
:10FC5000D9F80070002F00F0948094F842309F068D
:10FC600007D543F0010384F84230A38B9B1AA3838A
:10FC7000A5E094F841300DF12C0B04EB43035846FA
:10FC80000222B3F80C80FAF7E2FA0D9B02330D93CF
:10FC9000BDF8303008F10108033B1FFA88F8ADF8D1
:10FCA0003030D9F800702346584641460DF13202F3
:10FCB000B84794F842300746002851D0580705D578
:10FCC000BDF83230043BADF8323006E0BDF832000A
:10FCD000202138440422FAF7B2FABDF83210059A0E
:10FCE0000CAB04310093019289B2069B38460DAAF1
:10FCF00004F07FFA94F84230990704D503F0080322
:10FD000084F8423064E00D9AC0EB0A0CB2B1E28B89
:10FD10001FFA8CFA92451EDD94F8412004EB420252
:10FD200043F00103A2F80E8084F84230A38B043B19
:10FD3000A383AAF1040C1FFA8CF64AE094F8412040
:10FD400004EB420208F1FF3843F00103A2F80E80F1
:10FD500084F84230EFE708F101081FFA88F8A0E7BD
:10FD600043F0200384F842300D9B2082023B0D9328
:10FD7000BDF830300333ADF8303002E0002700E04A
:10FD800037460D9B02330D93BDF83030033BADF881
:10FD90003030BFB10CAB0093059BBDF8321001931E
:10FDA0000DAA069B384604F024FA03B202464BB172
:10FDB0000D9B23B1C0EB0A0C1FFA8CFA02E0C2EBD8
:10FDC0000A0CB8E7BDF83030013BADF83030F9E649
:10FDD0005646B4F81CC0039A049FCCEB050C1FFADE
:10FDE0008CFCC2EB0C0C099A1FFA8CFA3744CAEB54
:10FDF0000203BFB2A383BAF1000F3ED0DFF8B08098
:10FE0000D8F800301B8F9A0708D5236D33B104F161
:10FE10004800CAF100010122F9F796FB6EB3089B76
:10FE200007EB0A059D4228DA94F84230DB0724D418
:10FE3000D8F800301C4A1B8F13F0020F07F1100393
:10FE40000AD0216D41B11268D11804F14800043183
:10FE50005246F9F7BFF90AE0A08BA1691268014484
:10FE60006068134408445246191D05F0AFFFA38B88
:10FE70000397DB1BA383ADB288E694F8423003F00E
:10FE8000080384F84230E38F3846CAEB030CA4F829
:10FE90003EC00FB0BDE8F08F6492FF1F22A70100A3
:10FEA00029A70100A6A701006C92FF1F4C92FF1F1B
:10FEB0007492FF1F38B50C4D0C4904462868372250
:10FEC0001430FAF7C4F93722032384F82130A283CF
:10FED00094F920002968082302F0C6FB0028D4BF4B
:10FEE0000020012038BD00BF6C92FF1F9EA90100B9
:10FEF0002DE9F8433A4E0F4613460446316890F90F
:10FF000020003A4602F0B0FB0028D4BF4FF00008B2
:10FF10004FF00108B8F1000F5ED094F84030013383
:10FF2000DBB2012B84F8403056D82E4BA1691A68F9
:10FF3000A08BE389D4F81490558C238243189945FB
:10FF40004AD9ED1BADB2002D46D0C0EB0909D784CC
:10FF5000C1EB0909E78B1FFA89F2BA4228BF3A467A
:10FF6000954204D3BD4238BF2F46154600E02F46C8
:10FF70001D4A1268128F920709D5226D3AB1316875
:10FF800004F1480014312A46F9F724F906E06068C4
:10FF90003168184414312A4605F018FF134BE587E1
:10FFA0001B78DB0708D530682A46143021463B46CB
:10FFB000FFF7CEFD054602E0A38B2B44A383E38F1E
:10FFC0004B452CBF0823002335B1A58794F92000A9
:10FFD00031682A4602F048FB4046BDE8F88300BF7E
:10FFE0006C92FF1FD892FF1F7492FF1F5092FF1F49
:10FFF00038B50D4608490446FAF7E2FA2946FAF7F9
:020000021000EC
:10000000DFFA0649FAF7DCFA05490238FAF7D8FAB6
:10001000001B023880B238BD06AA010039AA0100CF
:1000200015AA01002DE9F0410C4690462E491322F5
:1000300007461E46FAF70BF994F82220013A07F119
:100040001100082A16D8DFE802F00D110B07091578
:1000500005150F0025490AE0254908E0254906E075
:10006000254904E0254902E0254900E02549FFF73C
:10007000BFFF00E00020133085B22EB163682B442F
:10008000636063695B1B6361E68B6369761BB6B271
:10009000B34296BF9EB20023082388F800301A4B63
:1000A0001B681B8F13F0020F2F440ED0236D63B11A
:1000B00004F1480800210A464046F9F745FA40464F
:1000C00039463246F9F786F804E060683946324628
:1000D00005F07CFE63685B1B6360636970192B44E9
:1000E000636180B2BDE8F081B2A701003EAA0100C1
:1000F00049AA010052AA010069AA010073AA0100DD
:100100007DAA010087AA01007492FF1F73B508231E
:100110000C468DF807300546002846D03E4E01219A
:100120003068F9F71BFD94F8213000BB022B08D88A
:1001300095F900302F2B04DD2846294604F014F9E8
:1001400000E0364D284604F1480132680123F9F7F2
:100150002DFB022802D0002565611DE0236D284695
:10016000636100F03FFE002584F8220014E0022BBA
:1001700003D895F900302F2B01DC30232B70284653
:10018000FBF780FF0A2384F822300546FBF786FF41
:100190000223606184F82130636943B94FF4DB7254
:1001A000626184F822301E4D01E04D68053D94F8EF
:1001B00022300A2B06D12DB1281D04F12201012283
:1001C00005F004FE174E30680535656021460023B2
:1001D00014300DF10702FFF725FF134BA0831B78A6
:1001E000124D13F0010F01460CD02A683068E38BE2
:1001F000568C2146143000229E4238BF3346FFF70A
:10020000A7FC01462B680022DA8420469DF80720CF
:10021000FFF76EFE02B070BD7492FF1F91AA01003D
:10022000E3A701006C92FF1F5092FF1FD892FF1F9F
:10023000F8B54769BA4204460D4607D20E2380F846
:10024000213022B3BF1A4261FA2606E0022380F869
:100250002130104B0027DF73FB2663690020E85430
:10026000294604F081F80C4B401B013860611B6883
:100270003046294622469847FA2E01D1676106E0AA
:1002800004F144002146BDE8F840FFF73FBF0020DD
:10029000F8BD00BF5492FF1F6892FF1F2DE9F74F72
:1002A00090F82130052B04460E4615460CD19B4B89
:1002B000DA7B002A40F02C81062180F821100121F0
:1002C0001860D97380F8432094F82130062B4FF042
:1002D000000800F2C980914FDFF85092002D00F025
:1002E000C3808E48C37B980602D56269013A626179
:1002F00003F0080101F0FF02E9B132780D2A05D1BF
:1003000023F008025907FA73E8D4A9E094F84330BF
:10031000013384F84330A3E00CF1010C5FFA8CFC4C
:1003200081F804C009EB0B010879604512D0013255
:100330000B2A00F09580B91859F8320091F804C0E2
:1003400096F800A010F90C0082454FEAC20B40F06D
:100350008380E1E74A79013A06F1010B05F1FF3AA2
:100360000A2A6CD8DFE802F0060B133B463F3F3FFA
:100370003F3F3F0023F0020343F0480331E043F0E6
:100380000403B01CFB73F9F729FF606157E05A07BB
:100390000AD594F8432022B9204659461FFA8AF21A
:1003A00069E043F02003FB73FB7B13F0120F46D090
:1003B000636994F84320083B9B1A6361584BFF2004
:1003C0001B6800212246984728B9544AD37BD80697
:1003D00001D5092300E00A2384F821302FE043F0FF
:1003E0000203FB732BE0990729D523F0020343F0A6
:1003F0001003F6E74B4BDFF838C1186801930CF196
:10040000010115221430CDF800C0F9F720FF1621A4
:10041000019B6161DDF800C094F92000C4F804C0BC
:1004200001211522A1610A2184F82210A2831968F2
:10043000082302F019F90028C8BF4FF001083A4814
:1004400000210B22F9F7FBFE94F82130082B07D985
:100450005E461FFA8AF507E04FF00000087166E774
:10046000013D0136ADB239E794F821300E2B07D1AA
:10047000204631462A4603B0BDE8F04FFFF7D8BE0C
:10048000002D47D06769AF4238BFBDB20A2B16D0E6
:10049000236843B9224B65611B68FC203146224624
:1004A0009847676104E0606831462A46FBF742FEE0
:1004B0002DB194E80C00934204BF05336360666974
:1004C0006368761B1D44666165601EBB04F12201F2
:1004D0002068FBF7EBFE114BDE732268104B666061
:1004E00001461B6802B110B1FE20002100E0FD2092
:1004F00022469847022384F8213008B1002001E009
:1005000004F14400214603B0BDE8F04FFFF7FEBD03
:10051000102000E0404603B0BDE8F08F5492FF1F6A
:100520006892FF1F6C92FF1F5892FF1FC0A6010028
:1005300079A701002DE9F7431E46A14B1C68074629
:10054000154604F50C7394F92000B84240F003827C
:100550004B1E0B2B00F20782DFE813F0350055002D
:1005600066000101050235007C000C000502050251
:100570006200A00094F82130002B40F0F481914BF0
:100580001B781E0711D5904B1B682BB9012384F8EB
:10059000213084F82070E6E12846612200F8012D20
:1005A00098470128F2D00220FDE1D806EED5864B0F
:1005B0001B68002BEAD02846622200F8012D9847DC
:1005C0000128E3D1EFE7A5683DB1804B1E6826B155
:1005D0000020012102462346B0478C2220460021FC
:1005E000F9F72DFE7A4BA560DA7B84F8207022B1F2
:1005F0001A68944204BF0022DA73002138460A4682
:1006000001F0F6FFAFE1022384F82130714B1B6843
:100610009B8CB3F5AF6F88BF4FF4AF63E383A2E168
:10062000A369002B00F09F8194F82130032B00F088
:100630009280A28BA3691344A36103294FF00003A6
:10064000A38307D1228A04F10E00A2811946042255
:10065000F9F7F5FD5F4A1268002384F84030D3842F
:1006600094F82110032900F06A81012940F27B816E
:100670006069A16988426CD98DF80730E58B411A11
:10068000A94203D808238DF807300D46508C8542C7
:100690000AD9002800F08781054605E001250023DE
:1006A00084F840508DF80730A0694B4EAFB2A78355
:1006B00048B93068214614300DF107020123FFF7D5
:1006C000B1FC05461DE0454A1268128F12F0020F78
:1006D000626810D0216D71B104F14808411F1144C6
:1006E00040460022F8F730FF3168404614313A4660
:1006F000F8F770FD05E03168104414312A4605F022
:1007000065FB304B1B78D9071CD5324AE38B126846
:100710003068558C14309D4238BF2B46214600224C
:10072000FFF716FA054668B994F842301A0704D460
:10073000294B1B6820221A7501250023A383A38956
:10074000E38123822046A9B29DF80720FFF7D0FB62
:1007500029E194F9200002F01DFB082023E16268E2
:1007600094F82130002A40F0EE80032B18D8284658
:100770001B490322F9F7FFFE50B12846194904220C
:10078000F9F7F9FE08B110200DE1052384F82130B6
:10079000002EF8D015F8013B013E2F2BB6B2F7D151
:1007A00094F82130042B30D9052B40F0CE802B78E3
:1007B0002A2B19D02846FBF765FC074615E000BF39
:1007C0007092FF1F5092FF1F6492FF1F4C92FF1FF9
:1007D0005492FF1FD892FF1F6C92FF1F7492FF1F4D
:1007E0009FA70100A2A7010000276B78284684F884
:1007F000443000F0F7FA276084F8220067600FB9F0
:1008000001236360002363619FE0002104F10C0079
:100810000622F9F714FD94F821102B78DFF8908167
:10082000032901D8202B66D198F8003094F83B00BA
:100830005B0760D5DFF87CC1032998BF04216B1CDE
:100840003246002A50D00F1F042F49D8DFE807F0A6
:100850000309101F270013F8017C0D2F08BF052185
:100860003EE013F8011C0A2914BF0421062137E0D9
:1008700013F8017C0D2F2FD01CF80090B9452DD115
:100880000130C0B214282BD90020082128E013F829
:10089000011C0A2923D1022384F8213065E013F8D2
:1008A000017C0D2F0ED1204480F8237004F1230722
:1008B0003846394603F048FC3846072103F01AFD54
:1008C000C8B15AE0172850D800F10109204480F837
:1008D00023705FFA89F003E0072101E00020042182
:1008E000013A013392B2ACE784F83B0084F821105E
:1008F0006FF0020041E098F800309F0738D52B4F89
:1009000000203B68294622469847B846002834D143
:100910002F467B78202B2BD0013EB6B246B3262B38
:1009200003D03F2B01D00137F3E7B878D8F8003077
:1009300003373946224698470028EAD01DE0204672
:10094000FFF7B8FA2FE0042B0DD92046294632468E
:10095000FFF7A4FC27E08C349C427FF4F4AD22E640
:100960000C2384F8213000201DE04FF0FF3004E01C
:1009700028462146FFF7CAFB15E0031D032B0DD8BF
:1009800001A252F823F000BF6109010067090100CC
:10099000990901003F0901000020EAE702AB03F8D2
:1009A000010D1846E5E703B0BDE8F0836892FF1F2C
:1009B0005092FF1F5AA701002DE9F0472E4D2C68D9
:1009C0008146884617461E46002C34D14FF40C70E1
:1009D000F9F72EFE286040F28C50F9F729FE274BDC
:1009E000042418607821264AD5F800A0082001F0D8
:1009F00079FD2B688AF8200093F92000002250210D
:100A000001F0F6FD2B68013C03F18C022A60E9D16C
:100A1000194A1C4DA3F5D27313602B68FBB920460D
:100A20002146F8F775FAB306286018D4204601214C
:100A3000F9F794F813E004F58C6594F92030002B55
:100A40000ADA78210E4A082001F04CFD502184F882
:100A50002000002201F0CCFD8C34AC42EDD10A4BD9
:100A60001E700A4BC3F80090094BC3F80080094B75
:100A70001F60BDE8F08700BF7092FF1F6C92FF1FE0
:100A8000350501007492FF1F5092FF1F6892FF1FEF
:100A90006492FF1F4C92FF1F084B70B51C685CB13D
:100AA00004F50C75FF2694F9200001F093FD8C34B9
:100AB00004F86C6CAC42F6D170BD00BF7092FF1FA1
:100AC0002DE9F3410E4B02AE1C6806F8010D04F54A
:100AD0000C7700254FF0020894F821300C2B07D139
:100AE000013584F8218030462146EDB2FFF70EFB38
:100AF0008C34BC42F0D1284602B0BDE8F08100BF82
:100B00007092FF1F2DE9F043B0F804800768B0F839
:100B1000069008F10808B84408F1060489B00646B2
:100B2000214600204A4600F08BF94FF6FF739842A9
:100B30006ED198F80650032D51D0082D02D0002D0B
:100B400066D11DE0002588F80650A570E570B388D1
:100B50003168F288194428460E3100F071F9C0431B
:100B600080B2030AA370E07001218DE810020295A3
:100B7000039507F11A002A46802300F023FA47E084
:100B800023798DF8155001228DF8163008F10C01EB
:100B900003230DF11A008DF817308DF819208DF808
:100BA0001450F9F754FB062307F11A0104220DF142
:100BB0001B008DF81830F9F74AFB0522284605A9D5
:100BC000F9F784FC9DF818200532904220D969235A
:100BD000284605A98DF81730F9F778FC18E06378F6
:100BE000032B15D1637C112B12D1227A02F00F0254
:100BF00092000832A318A05C99785A78DB7842EA10
:100C0000002043EA0121022207F11E0303F01AFA31
:100C100009B0BDE8F0832DE9F04190B007AC16466D
:100C2000804622220F46204600218DF81730F9F722
:100C300006FB0823A01D0DF1170101228DF81C30C1
:100C40008DF82060F9F703FB002505F161020135FD
:100C500063191A2DDA71F8D121462222002000F002
:100C6000EFF8C04382B2130A8DF81E30222301939D
:100C70009DF917308DF81F2003930094029640468B
:100C8000012100223B4600F09DF910B0BDE8F08143
:100C900030B504460D4685B021462A46002000F0B6
:100CA000CFF8C04380B20022030AA370E0708DE841
:100CB00030000292039204F114000121802300F01D
:100CC00081F905B030BD2DE9F7430024054688467B
:100CD000A1462A46501B164612F8017B79B22F29ED
:100CE000F8DCB0B1022813DC86F80090301AF9F76E
:100CF00058FA0DF804000134062C06F1010537708E
:100D0000E7D1404669462246F9F7A1FA284600E0B5
:100D1000002003B0BDE8F08370B50A460546002404
:100D20002D26285D4121F9F7F3F90134052C00F156
:100D300001020670F5D168790121BDE87040F9F72C
:100D4000E7B92DE9F04100240F46A0460246131AE8
:100D5000154612F8016BA6F13001C9B20929F6D97E
:100D600073B1032B0CDC85F80080E81AF9F736FA2A
:100D700038550134042C05F101002E70E6D100E055
:100D80000020BDE8F08170B50A46054600242E26F5
:100D9000285D4021F9F74AF90134032C00F10102E2
:100DA0000670F5D1E8780021BDE87040F9F73EB94A
:100DB00030B50023CA5C9CB282B1C55654B2A5427C
:100DC0000AD0602C01DD203A02E0402C08DD203200
:100DD000D2B252B2954203D10133EBE7204630BD87
:100DE000002030BDF8B50023014610F9012B1F2A61
:100DF00016DC9BB10B461846013B90F900202E2AC9
:100E0000F9D10E4D0024471C384655F82410E6B29F
:100E1000FFF7CEFF78B901340A2CF5D10A20F8BDCE
:100E20003F2AE6D0202A02D1002BDDD0E2E72E2A8D
:100E300008BF0123D8E73046F8BD00BFA082FF1FDE
:100E400010B5C3B2000A0231E2B111F8024C2044DD
:100E5000C0B2A04205D2013313F0FF0304BF01303A
:100E6000C0B2012A0ED011F8014C2344DBB2A342D8
:100E700005D2013010F0FF0004BF0133DBB2023AAB
:100E800092B2E0E703EB002080B210BDF0B5002481
:100E9000E5B2AB420CD0065D155D45EA0607FF2FB3
:100EA00008D10F5D7E40354204F10104F0D001E02D
:100EB0000120F0BD0020F0BD2DE9F34704680223B6
:100EC0008DF80430637B05460BB1002070E0038988
:100ED0000D2BFAD9212BF8DDA27B02F0F002402A7B
:100EE000F3D194F81080627C02EB08281FFA88F88E
:100EF0000D3B4345E9DD04F11E0738462E49042227
:100F0000F9F739FBE8B12C4938460A1D0423FFF7ED
:100F1000BDFF0646A8B9384628490422F9F72BFB3D
:100F200078B1E07D314640F08000FCF7B3FDE37D11
:100F3000012BCAD1286822490622F9F71CFB20B1EF
:100F4000C3E7E07D0021FCF7A5FDA67B06F00F06B8
:100F5000B600143EF6B2282EB7D82B89213BB342F7
:100F6000B3DD06F1140729681FFA87F900200E3156
:100F70004A46FFF765FF4FF6FF739842A5D104F18B
:100F80001A0A50460D490422F9F7F5FA28B12968E2
:100F90005046063101AAFCF733FF237D9B0694D40B
:100FA000A8F11408C6EB0806A5F80490EE803846B0
:100FB00002B0BDE8F08700BFF982FF1F38AB010027
:100FC000F382FF1F2DE9F0418AB00D4614469DF9CA
:100FD00048109DF94C20BDF8446007469846FDF73F
:100FE00021F80146002865D00531062201A8F9F74D
:100FF0002EF9334906220DF10A00F9F728F9314993
:10100000022204A8F9F723F945238DF8123006F1DE
:1010100014031A128DF814202B4A8DF813401488EB
:101020008DF81530230A8DF816308DF81740631CA3
:10103000002413800DF112010A2220468DF81B5066
:101040008DF818408DF819408DF81A80FFF7F8FEDA
:101050001E490422FFF7F4FE39460422FFF7F0FE92
:10106000C04380B2030A8DF81D0018498DF81C306A
:1010700004220DF11E00F9F7EAF8042239460DF1B9
:101080002200F9F7E4F82846114D2146FCF7EAFC66
:10109000287801A92222F9F719FA68B1109928785D
:1010A0003246F9F713FA287821462246F9F70EFA64
:1010B00080B201E04FF6FF7000B20AB0BDE8F081E7
:1010C000F382FF1FA5AA01007892FF1FF982FF1F7C
:1010D0000591FF1F10B5084B044693F9000001F07D
:1010E00059FE064B01221A70054B20461B68002151
:1010F0009847082010BD00BF8C82FF1F7A92FF1F07
:101100008092FF1FF0B5794E3378053BD3B00A2BA0
:1011100000F2E980DFE813F00B001D0024002F002F
:101120003300400058005B00A700A700C90007A8D3
:101130006F49F9F745FA6F4B00211B68012098476A
:1011400001460DF12100F9F73BFA07A8F9F742FA39
:101150000FE007A86849F9F733FA0A240823AAE040
:10116000644B1B6806200021984707A9002202F063
:1011700098FF84B275E05F4B07201B68F3E707AD6B
:101180005E492846F9F71CFA5A4B00211B680220D9
:10119000984701460AA80CE007AD59492846F9F7D7
:1011A0000FFA544B00211B680320984701460DF1AC
:1011B0002600F9F705FA2846F9F70CFA80B23E2323
:1011C000441C2B54A4B24CE007A84E496FE0494D93
:1011D0004D4907A8F9F7F4F92B6800210320984737
:1011E0000446214608A8F9F7EBF92046F9F7F2F989
:1011F00084B207AA201D12FA80F04449F9F7E0F9F9
:101200002B680021042098470F34A4B2074607A892
:1012100039462044F9F7D4F93846F9F7DBF9204488
:1012200084B207A820443A49F9F7CAF92B6800218B
:10123000022098470834A4B2054607A8294620444E
:10124000F9F7BEF92846F9F7C5F9204484B207A892
:1012500020443049F9F7B4F92F4B02340022A4B2EC
:101260001A80082327E02C4B1B88ADF80630214B51
:101270000DF106011B6805209847BDF806400146A0
:1012800044B907A82549F9F79BF90E2333700324C5
:10129000082310E0B4F5967F28BF4FF4967407A892
:1012A0002246F8F7D4FF002305E01D4907A8F9F707
:1012B00087F90424082332780D2A08D0611C07AA74
:1012C0000D2089B210550A2002345054A4B2154A98
:1012D00002A992F90000224601F0C6F90028D4BF05
:1012E0000020012000E0002053B0F0BD7A92FF1FE3
:1012F000A7AA01008092FF1FADAA0100B8AA0100B1
:10130000C5AA0100D0AA0100D5AA0100DAAA0100ED
:10131000E6AA01003BAA01008492FF1FEFAA010088
:101320001BA601008C82FF1F37B51C4D02282870B8
:101330000DD0042828D0012822D15320F9F7C6FB6C
:10134000174B08201B6800219847002423E0154C08
:1013500094F9000001F01EFD94F9000012490024E8
:1013600000941922234601F0A9FCA0420DDB0323BF
:10137000532040F2DC5101222B70F9F743FB04E0CB
:10138000FFF7C0FE044600E00024532040F2DC5189
:101390000122F9F737FB204603B030BD7A92FF1FD8
:1013A0008092FF1F8C82FF1F7C92FF1F80B102780A
:1013B0004378303A92B21201303B92B21A4492B260
:1013C0008378120192B2303B13449BB2033000E0A9
:1013D0000346354A1278043A0B2A63D8DFE802F054
:1013E000060B1A2914373C474C4E565BB3F5087F61
:1013F00058D1052054E0B3F5147F53D12B4B1B7803
:10140000DB0705D506204BE040F23522934218D188
:10141000092045E0B3F54D7F05D14378562B08BF31
:1014200007203FD13CE040F2015293423AD10E20D6
:101430001BE0B3F54D7F35D14378552B32D10820D1
:101440002EE002F5407293422CD10D200DE0B3F551
:10145000147F27D10A2023E0B3F5147F08BF0B20A7
:101460001ED0B3F5AA6F1DD10F20FFF733BEB3F521
:10147000557F17D10C2013E0A3B905E093B90C4BAD
:101480001A8802F596721A800D2009E0B3F5147FD0
:1014900008D10F2004E040F22122934202D1012022
:1014A000FFF742BF002070477A92FF1F7B92FF1F19
:1014B0008492FF1F10B5204C94F90040844239D12A
:1014C0000139082936D8DFE801F016070D282F1F4B
:1014D000243505000A2013E0184B1B78032B23D179
:1014E000042012E0154B1B780B2B4FF000001DD988
:1014F000FFF75CFF18E0114B1B78012B04D90C207F
:10150000BDE81040FFF7E6BD0120BDE81040FFF741
:101510000BBFBDE81040FFF7F5BD022B07D9104601
:10152000BDE81040FFF742BF002010BD10BD4FF0D6
:10153000FF3010BD022010BD8C82FF1F7A92FF1F6A
:1015400000B5094B807B1B788BB053B169460522EF
:10155000F8F77EFC28B19DF8033013B90B20FFF794
:10156000B9FD0BB05DF804FB7A92FF1FF8B5144C7F
:1015700094F90030002B07460D46164611DB114B3F
:101580001B78012B18D8394604220F48F8F75FFE64
:101590000E4B1E600E4B02201D70FFF7C5FE002093
:1015A000F8BD102078210B4A00F09CFF0028207025
:1015B000E5DA4FF0FF30F8BD6FF00100F8BD00BF75
:1015C0008C82FF1F7A92FF1F7C92FF1F8092FF1F69
:1015D0007B92FF1FB514010010B5034601301C7843
:1015E00014F0800F11D004F07F04012C08D0022CDD
:1015F0000AD15C78D81C9B7843EA0424042305E0D4
:10160000981C5C78032301E0002402230C8012B1B3
:101610001188CB1A138010BD70B50378022B13D13B
:101620004278541EE4B2032C10D8851C83782846D7
:10163000013A12F0FF0204D010F8016F46EA0323CA
:10164000F6E72819013000E000230B6070BD0000B0
:1016500038B50446144B94F86950186891F9003075
:10166000002BACBF0831014691F900309D421ADAD7
:1016700023444A7883F824204B68002BEED00B7863
:101680000133DBB284F864302344002283F8242041
:10169000A02384F86B304B682046984794F8643058
:1016A000013384F8643038BDCC92FF1F2DE9F3413B
:1016B0000F4690460A300C465CB30178302901D0C1
:1016C00041450ED190F90120002A06DA043CA4B26B
:1016D000220A8270C4700430EEE7023CA4B20230E9
:1016E000EAE7461C30460DF106010022FFF774FFC1
:1016F000BDF806507F2D03D9EB1CF018043C02E026
:101700006B1CF018023CA4B2A54204D8641BA4B21E
:10171000D2E7384601E04FF0FF3002B0BDE8F0817B
:10172000F8B5444B0D4614461F6898B103782B2B2F
:1017300001D00220F8BD352978D84D1E461CADB227
:1017400002F1240031462A462E44F8F780FD266037
:1017500084F86450002284F8662084F8682007F139
:10176000080313F9081C0029A3F1080653DB94F8B9
:1017700068208A424CD1A11891F8240013F8071C64
:10178000884246D153F8041C29B394F86B30A32B3C
:1017900017D1B378DA0708D5274B94F864201D6871
:1017A0000D2004F12401002308E0A36873B9224A44
:1017B000156894F864200E2004F12401A847042041
:1017C000F8BDA12B02D1B3789B071CD520468847D2
:1017D000002820DA17E0511CC9B2A94284F8681029
:1017E00017D394F86B10A5290BD184F869202046F3
:1017F0003146FFF72DFF94F86930013384F86930E2
:1018000009E0A12905D120463146FFF721FF02E07A
:1018100001DC0833A5E794F8660048B994F8653010
:10182000002B86D0802384F86630F8BD0120F8BDF7
:101830000020F8BDCC92FF1FC092FF1FFF2810B5FB
:1018400003460A7004D801224A70C81C8B7010BD70
:10185000B0F5803F4FEA102205D2022048708A700E
:10186000081DCB7010BDB0F1807F4FEA104006D24A
:10187000032488704C70CA700B71481D10BD04247D
:101880004C701C0EC8708C700A71881D4B7110BD95
:10189000F8B50E4C94F90030002B07460E4615465D
:1018A0000ADA10200A49032202F06AFA002820709E
:1018B00002DBA12102F08AFA064B94F900001F60B6
:1018C000054B1E60054B1D60F8BD00BF8D82FF1FDC
:1018D000C5220100C092FF1FB892FF1FCC92FF1FCC
:1018E00012B1136813B949E04FF480737F2902D80D
:1018F0000170013070470A0605D501F07F024900EA
:1019000021F0FF011143B1F5803F09D2012B41F4D1
:10191000004135DD03460A0A03F8022B41702DE031
:101920000A0406D4C1F3CF3289B241F4004141EA3E
:101930000241B1F1807F0AD2022B41F400011FDD88
:101940000B0C03700B0A43708170033070470A025E
:1019500007D44A0021F07F4102F07F4241F40001A8
:101960001143032B41F000410ADD0B0E03700B0CF9
:1019700043700B0A8370C17004307047184670477B
:10198000002070472DE9F04F0F4609880546406852
:1019900001F10806421C3E446A6085B0C1F5FA7345
:1019A00006F1020895F8642098B902F108009842FF
:1019B00002DB4FF0FF30FFE06FF00800801A0344B5
:1019C0003944039330238B72822388F80130063622
:1019D00008E0111D9942ECDA6FF00401891A0B44FA
:1019E00003934646B146302309F8013B0623B37002
:1019F00095F864304FF02B0B0133F37006F1050AB4
:101A000086F804B095F86420504605F12401F8F7F3
:101A10001EFC95F8662095F864C0402A0AEB0C0479
:101A200030D00AD8022A17D002D8012A1AD0B4E03E
:101A3000042A3AD0062A6CD0AFE0432A09D002D853
:101A4000422A09D0A9E0A2F18003022B40F29A8039
:101A5000A3E0039B002BACD02146E869FFF7EEFE24
:101A600004469AE0296A95F86750039A6B1C9342E2
:101A70009FDA6FF001035B1B1344039304230AF8FE
:101A80000C300DE0296A95F8675003986B1C83426F
:101A90008FDA6FF001035B1B03440AF80C200393F9
:101AA00004F1020A657050462DE0D5F820B0BBF174
:101AB000000F0AD05846CDF804C0F8F78BFD85B268
:101AC0007F2DDDF804C003D800E05D46AB1C00E0CC
:101AD0002B1D039A93423FF76CAFD31A03937F2DCC
:101AE0004FF004030AF80C3004D804F1020A6570C0
:101AF00065B106E0822363702B0AA37004F1040A27
:101B0000E570504659462A46F8F7A1FB0AEB050452
:101B100043E003992B6A012902DC4FF0000A2FE011
:101B200004AD023945F8041D0AF80C2084F802B00F
:101B300004F1030A4FF0000B93F900202F2A0EDC6A
:101B4000504659462A460193FFF7CAFE019B82463A
:101B50000028E2D093F900207AB10133ECE718466F
:101B60000193F8F73BFB019B83461A46134601326B
:101B700093F900102F29F9DCDEE7A31CC31A637068
:101B800054460AE0039B012B7FF713AF00230AF8AA
:101B90000C20023404F8013C02E0002C3FF409AFB1
:101BA000C9EB040909F1FF3986F801903B88C8EBBD
:101BB00004041C443C80002005B0BDE8F08F000008
:101BC0002DE9F04FADF5337DDFF804C303911446E2
:101BD0001D464FF00101302383464FF0820A4FF03B
:101BE0002B004FF002084FF00409DCF800608DF87C
:101BF00010008DF8C6308DF8CB102346CDF808C004
:101C00008DF8C7A08DF8CA808DF8CC508DF8CD9096
:101C100003200DF1CF010022B047C7B28DF8CE707E
:101C200007F10903DDF808C015B1012D60D035E1D9
:101C30002FAE33446FF05B00987233463B4407F19C
:101C40000E061F4683F814A02FA90623FB750F4626
:101C500037444FF02B02FA72DCF800C007F10C0198
:101C60002A4623464046E0470130C0B206442FAB27
:101C700033444022B872DA722FAB334403F10D00C3
:101C80008C4983F80C904A46F8F7E1FA2FAB3344BD
:101C90004FF0010083F811802FAB334403999874FF
:101CA0002FAB3344844A83F813B02FAB334412680C
:101CB00083F814802FAB334458752FAB3344432043
:101CC000997506F10D012FAB0B4414214A43642191
:101CD000B2FBF1F2110E1973110C5973110A9973B9
:101CE000A421987283F80B90DA731336039146E0BF
:101CF0002FAA1344A7229A722FAB3B4407F10F027D
:101D000083F814A02FAB3B4483F817802FAB3B44E0
:101D10001D766A4B195D01B91D552FAE32441B5D0E
:101D2000DFF8AC81937233463B444FF0020A83F8EC
:101D30001AA033463B4400214FF001090A4683F8BC
:101D40001B90D8F8006023460420B0472FAB3B44DB
:101D5000002118772FAB3B440A4683F81DA02FAB18
:101D60003B44D8F800C083F81E9005202346E04786
:101D70002FA907F116060F44A722F87703922FAB7D
:101D8000334430229A722FAB33448222DA72A0237A
:101D900004368DF8BB30DFF838A1ADF8BC60012304
:101DA00015938DF8BAB000260DF11108012D16D14A
:101DB00016B94046424903E0012E07D14149404649
:101DC000F8F7FEFB0023C14647461CE0B21E4BEA73
:101DD0000222DAF800700620414692B205E0DAF8F5
:101DE0000070062041464BEA06222346B8470028E9
:101DF000E8D12BE017F9012B2E2A03D097F9002008
:101E0000002AF7D1814697F9002072B13846029333
:101E1000F8F7E4F9002201464846FFF761FD029B0E
:101E2000C9EB000C6344DBB2E4E763B1591C04A8BE
:101E3000C9B214AAFFF774FC28B914A82FA9FFF798
:101E4000A1FD002802DB0136F6B2AFE72FA8BDF8EE
:101E5000BC10039AFFF72AFC031E22DD1A4A1268FF
:101E6000062101FB0421194A087912789BB210431C
:101E700004F0030240EA421000936E23019340B243
:101E8000A2220DF1BE0302F051F8411C0DD0012D2C
:101E90000AD10A4B1A5D01321A5505E06FF00100B4
:101EA00003E06FF0020000E000200DF5337DBDE897
:101EB000F08F00BFF982FF1F248AFF1FC492FF1F0B
:101EC000F3AA010001AB0100B892FF1F8D82FF1F32
:101ED000C092FF1F2DE9F0474FF00609DFF840A040
:101EE00080460F46164609FB02F900240125DAF860
:101EF00000304B445B791D4208D10134E4B26D00DF
:101F0000022CEDB2F3D10020BDE8F0872346404615
:101F100039463246FFF754FE431CEED1BDE8F08748
:101F2000B892FF1FF8B5C0F34114174B09B1002256
:101F30001A551B5D144A042B1FD80133134D13553A
:101F40002301EA18E85C51782246FFF7C3FF01300D
:101F500001D10020F8BD0E4E05EB04170025335DBE
:101F6000013BDBB233550235002BF2D07B19785D93
:101F700059782246FFF7AEFFF1E700231355044AD4
:101F800013550120F8BD00BFC792FF1F8692FF1FA7
:101F9000BC92FF1F70B58CB0847B0DF10905204603
:101FA00002A90522F7F754FF50B39DF80B30412BDF
:101FB000F5D102A99DF80C202046F7F749FF0DF155
:101FC000070029460122F8F742F99DF80830032B53
:101FD0000ED19DF907000021FFF7A4FF0028DED0F5
:101FE000084B00211E680A460B460A20B047D6E778
:101FF000042BD4D19DF907000121FFF793FFCEE711
